:100000000C94A2080C94C1080C94C1080C945109DA
:100010000C9487090C94C1080C94C1080C94C10875
:100020000C94C1080C94C1080C94C1080C94C1082C
:100030000C94C1080C94C1080C94C1080C94A70C32
:100040000C94C1080C94C1080C94C1080C94C1080C
:100050000C9412660C94C35D0C94C1080C94C108F6
:100060000C94C1080C94985E0C94C1080C948C5E9E
:100070000C94C1080C94C1080C94C1080C94C108DC
:100080000C9445710C94C1080C94C1080C94C108DF
:100090000C94D65E0C94C1080C94CA5E0C94C108F2
:1000A0000C94C1080C94C1080C94C1080C94C108AC
:1000B0000C94C1080C94C1080C94C1080C94C1089C
:1000C0000C94C1080C94C1080C94C1080C94C1088C
:1000D0000C94C1080C94C1080C94C1080C94C1087C
:1000E0000C94C1080C94CB650C94D5650C94C16537
:1000F0000C9481650C9406660C94F7650C94EB6582
:100100000C94DF650C94C1080C94C1080C94C108D0
:100110000C94C1080C94C1080C94C1080C94C1083B
:100120007E7A9D7A1C7B0B7C2B7C4B7C537C007CE9
:10013000084AD73B3BCE016E84BCBFFDC12F3D6C4E
:1001400074319ABD56833DDA3D00C77F11BED9E4B4
:10015000BB4C3E916BAAAABE000000803F076342E1
:1001600036B79BD8A71A39685618AEBAAB558C1D4E
:100170003CB7CC5763BD6DEDFD753EF6177231BFD0
:10018000000000803F08000000BE922449123EABF0
:10019000AAAA2ABECDCCCC4C3E00000080BEABAAA1
:1001A000AAAA3E00000000BF000000803F0000003F
:1001B0000000084178D3BB4387D1133D190E3CC3DF
:1001C000BD4282AD2B3E68EC8276BED98FE1A93E5E
:1001D0004C80EFFFBE01C4FF7F3F00000000002500
:1001E000730A005854414C5F5452494D3D256400F8
:1001F00025730A0025730A00546573742036202580
:10020000730A005465737420352025730A00546501
:10021000737420342025730A0054657374203320CE
:1002200025730A005465737420322025730A005424
:1002300065737420312025730A006368616E3D2563
:10024000640A0074787077723D25640A0035303096
:100250006B0A003235306B0A003131356B0A0035DC
:10026000366B0A0033386B0A0025730A0073656E1B
:10027000743D252D75206475703D252D75206967A9
:100280006E6F7265643D252D752074746C5F7A65A0
:10029000726F3D252D750A0025372E3366202537D0
:1002A0002E33660025352E326620004572726F723D
:1002B000203020566F6C74004E6F74207375707010
:1002C0006F727465640A004572726F722030205636
:1002D0006F6C74004572726F72203020566F6C74B0
:1002E0000025630074746C3D252D64200074746CCB
:1002F0003D252D6420004E65772074746C3D252DBE
:100300006420002563004D533536313120503D25A2
:100310002D372E326620252D372E32666D0A00428B
:100320004D5030383520256C642050612020252D1B
:10033000372E32666D00256300545F484541545F97
:100340004944583D252D352E32662000545F4445E2
:10035000573D252D352E3266200041483D252D354F
:100360002E32662000545F53485432583D252D35B7
:100370002E3266200052485F53485432583D252D96
:10038000352E32662000545F52483D252D342E31E3
:1003900066200052483D252D342E3166200025630D
:1003A00000256300256300256300256300726570E6
:1003B0006F72745F616C6C3D007265706F72743D3A
:1003C00000256300256300256300256300204F534B
:1003D0004343414C3D2564200020467573653A2017
:1003E00065653D253032782068663D2530327820BD
:1003F0006C663D25303278206C623D2530327800C5
:100400004D43553D2530366C780025630074785F88
:100410006C656E3D252D6C752C6C6F775F766F6CFF
:10042000746167653D252D6C750A002563004F4B8F
:100430000A0025630025630025630025630025630A
:100440000025630064656275675F616C6C3D0064E4
:10045000656275673D0064656275673D0025730AD6
:1004600000646565700A006E6F6E650A00707772D1
:10047000733D00696E74725F7365635F70313D2513
:100480002D372E33660A00696E74725F70313D2518
:100490002D6C640A00696E74725F7365635F7030FF
:1004A0003D252D372E33660A00696E74725F7030F9
:1004B0003D252D6C640A00765F6D63753D252D35F5
:1004C0002E32660A00745F6D63753D252D352E3220
:1004D000660A00707077723D25730A006465627564
:1004E000673D0025730A006175746F0A006C6F67C1
:1004F0005F6D6F64653D007573625F7077723D2557
:10050000730A0072656C61793D25730A0074746C1E
:100510003D252D640A0052494D455F616464723D7A
:10052000252D642E252D640A006E65696768626F4B
:10053000725F7461626C655F73697A653D25640AF8
:10054000006C6F775F766F6C746167653D252D3346
:100550002E32660A00747870773D25640A0063685D
:10056000616E3D25640A006932633D0069643D00A7
:100570007478743D25730A0053797374656D205344
:10058000756D6D6172790A006D61736B3D002C00B1
:10059000696E74657276616C3D252D750023252D7D
:1005A000642C00745F686561745F69647800745FCF
:1005B00064657700616800705F6D733536313100B6
:1005C00072685F736874327800745F73687432782D
:1005D0000070610070006164340061643300616424
:1005E00032006164310061330061320061310076B4
:1005F0005F696E00726800757074696D65007031B6
:100600005F6C73740070315F740070310070305F24
:100610006C73740070305F7400703000765F6D63CF
:100620007500745F6D637500743100740069640057
:1006300065363400747874002D002B006175746F7A
:10064000006E6F6E6500706F7765725F73617665BF
:100650005F6C656472790072656C61795F6C65646A
:100660007900636F6D7061737300616363656C0023
:100670007072657300705F707772006165730070EF
:10068000315F6C6564790070305F6C656472006521
:1006900076656E74006C6564006F7700706B740033
:1006A00074785F6C6564790072785F6C6564720061
:1006B0006F706572006E6F6E65002530327800765F
:1006C0005F6164343D252D382E3666002000765F4C
:1006D0006164333D252D382E3666002000765F613B
:1006E00064323D252D382E3666002000765F616429
:1006F000313D252D382E3666002000765F6C696707
:1007000068743D252D382E3666002000765F6132F4
:100710003D252D372E3366002000765F61313D2563
:100720002D372E3366002000765F696E3D252D350E
:100730002E326600204E657665722D7573656420D5
:10074000737461636B203E20256420627974657345
:100750000A00757074696D653D252D642D6461799D
:10076000732D253032643A253032643A25303264B4
:100770002D686F7572730A0074657374205B6F6601
:10078000667C317C327C337C347C355D20202020BB
:10079000202020202D2074657374206D6F64657394
:1007A0000A0D00263A205B545820504B5420434FEA
:1007B0004E54454E545D2020202020202020202D06
:1007C0002073656E6420706B742066726F6D206399
:1007D0006D646C696E652F636861740A0D007764DF
:1007E00074205B6F6E7C6F66667C746573745D20CD
:1007F000202020202020202020202D2077617463BD
:1008000068646F670A0D00757067722020202020D1
:1008100020202020202020202020202020202020D8
:100820002020202D207265626F6F74207669612010
:10083000626F6F746C6F616465720A0D007561722E
:1008400074205B33386B7C35366B7C3131356B7C97
:100850003235306B7C3530306B5D202D2073657404
:10086000207465726D2F7561727420737065656494
:100870000A0D00626F6F742020202020202020208D
:100880002020202020202020202020202020202D5B
:10089000207265626F6F740A0D0070777273205B4F
:1008A000646565707C6E6F6E655D20202020202061
:1008B0002020202020202D206D637520736C65651D
:1008C00070206D6F64650A0D007265737420656534
:1008D00070726F6D202020202020202020202020DA
:1008E00020202020202D20726573746F7265206592
:1008F0006570726F6D0A0D0070707772205B6F6E9D
:100900007C6F66665D202020202020202020202073
:10091000202020202D2070726F6772616D6D6162E2
:100920006C65207077720A0D00747874205B7374A4
:1009300072696E675D20202020202020202020204A
:1009400020202020202D20536574207265706F7246
:1009500074207465787420737472696E670A0D0070
:1009600074787077205B31352D305D202020202079
:100970002020202020202020202020202D205458FE
:10098000205077722E204869676865737420302084
:10099000283364426D290A0D0074746C205B302D7D
:1009A00031355D20202020202020202020202020E4
:1009B00020202020202D2074696D652D746F2D6CF2
:1009C00069766520666F72207061636B6574730A67
:1009D0000D007373202020202020202020202020A4
:1009E00020202020202020202020202020202D20FA
:1009F00073797374656D2073756D6D6172790A0D0D
:100A00000072732020202020202020202020202061
:100A1000202020202020202020202020202D207277
:100A20006164696F2073746174730A0D00726920C8
:100A30005B236E5D205B696E745D2020202020208A
:100A40002020202020202020202D207265706F7211
:100A50007420696E74657276616C0A0D007265208F
:100A60005B236E5D205B2B7C2D5D205B6D61736B6A
:100A70007C6175746F2C6D61736B5D202D206D6FC3
:100A80007465207265706F7274207365742F6D6F5A
:100A9000646966790A0D006F7720202020202020CD
:100AA0002020202020202020202020202020202046
:100AB0002020202D206F6E652D776972652073656B
:100AC0006E736F72730A0D006C6F67205B617574D3
:100AD0006F7C6F6E7C6F66665D202020202020205A
:100AE000202020202D206D6F746573206461746157
:100AF000206F6E205553420A0D006E65205B666CB8
:100B00007573685D202020202020202020202020B8
:100B10002020202020202D206E65696768626F727A
:100B2000207461626C650A0D0065727220202020BD
:100B300020202020202020202020202020202020B5
:100B400020202020202D206572726F722073746126
:100B500074730A0D006D6375202020202020202052
:100B60002020202020202020202020202020202085
:100B7000202D206D637520696E666F0A0D00696413
:100B8000205B72657365745D20202020202020206A
:100B9000202020202020202020202D206964206873
:100BA000616E646C696E670A0D0068756D202020A7
:100BB0002020202020202020202020202020202035
:100BC0002020202020202D2068756D6964697479AB
:100BD0002073656E736F720A0D0072656C61792007
:100BE0005B6F6E7C6F66667C73746174735D2020CE
:100BF0002020202020202D2072656C6179206E65D8
:100C000074776F726B207265706F7274730A0D0067
:100C10006465205B6D61736B5D20202020202020A7
:100C20002020202020202020202020202D2064652E
:100C30006275670A0D006368616E205B31312D3289
:100C4000365D202020202020202020202020202051
:100C500020202D206368616E2031312D323620280E
:100C6000322E3430352D32343830204D687A290A0E
:100C70000D0063616C69205B5B765F696E7C61313E
:100C80007C61325D20766F6C747C72657365747CF8
:100C90006E6F6E655D202D2063616C696272617498
:100CA000650A0D0061646320202020202020202080
:100CB0002020202020202020202020202020202034
:100CC0002D2073686F7720765F696E2C2061312C40
:100CD00020613220766F6C74616765730A0D007550
:100CE0002020202020202020202020202020202004
:100CF00020202020202020202020202D20757074EE
:100D0000696D650A0D0076202020202020202020FB
:100D100020202020202020202020202020202020D3
:100D200020202D2076657273696F6E0A0D00682091
:100D300020202020202020202020202020202020B3
:100D4000202020202020202020202D2068656C706D
:100D50000A0D00256300756E6B6E6F776E20636DF4
:100D6000640A00484D433538383300257300257335
:100D700000202573002025362E32662000253032D3
:100D8000780074656D705F65787465726E3D252DB1
:100D9000362E326600202573002025362E3266203E
:100DA0004F6E2D426F617264002530327800746599
:100DB0006D705F626F6172643D252D362E32660064
:100DC0000A00503A20256C642050612020252D37E0
:100DD0002E3266206D0A00256300256300493243E8
:100DE0003A2000452025642E256420636C6F636BD8
:100DF00020256C752063707520256C75206C706DD6
:100E000020256C752069727120256C7520676C65D2
:100E10006420256C7520796C656420256C752072C2
:100E20006C656420256C7520747820256C75206CA9
:100E3000697374656E20256C752073656E736F72AF
:100E40007320256C752073657269616C20256C7543
:100E50000A00532025642E256420636C6F636B2089
:100E6000256C7520747820256C7520727820256C8F
:100E7000752072747820256C752072727820256C2C
:100E800075207265786D697420256C752061636BBF
:100E9000747820256C75206E6F61636B74782025E3
:100EA0006C752061636B727820256C752074696D98
:100EB00065646F757420256C752062616461636B75
:100EC000727820256C7520746F6F6C6F6E672025AB
:100ED0006C7520746F6F73686F727420256C752049
:100EE00062616473796E636820256C752062616449
:100EF00063726320256C7520636F6E74656E746910
:100F00006F6E64726F7020256C752073656E6469F6
:100F10006E6764726F7020256C75206C6C7478201D
:100F2000256C75206C6C727820256C750A00257311
:100F300025730A004F6E6C696E650A000A002C204A
:100F4000636865636B207261746520257520487A3B
:100F50000025732025732C206368616E6E656C20FC
:100F6000257520706F776572202575000A00257839
:100F70003A004D41432061646472657373200052EE
:100F8000616E646F6D20455549363420616464722A
:100F90006573732067656E6572617465640A000A23
:100FA0002A2A2A2A2A2A2A426F6F74696E67202504
:100FB000732A2A2A2A2A2A2A0A00454550524F4DC6
:100FC00020697320636F72727570742C207265775C
:100FD000726974696E6720776974682064656661F8
:100FE000756C74732E0A006C6F63616C686F737438
:100FF0000041544D4547413132387266613100023B
:101000000000FFFE0000016E616E00696E66000068
:10101000407A10F35A00A0724E18090010A5D4E8C7
:101020000000E87648170000E40B54020000CA9A5A
:101030003B000000E1F505000080969800000040AC
:10104000420F000000A086010000001027000000F1
:1010500000E803000000006400000000000A000037
:101060000000000100000000002C76D888DC674FEB
:101070000823DFC1DFAE59E1B1B796E5E3E453C61B
:101080003AE651997696E8E6C28426EB898C9B6213
:10109000ED407C6FFCEFBC9C9F40F2BAA56FA5F4BD
:1010A00090055A2AF75C936B6CF9676DC11BFCE0E5
:1010B000E40D47FEF520E6B500D0ED902E03009438
:1010C0003577050080841E080000204E0A000000CD
:1010D000C80C333333330F986E12831141EF8D21D7
:1010E00014893BE65516CFFEE6DB18D1844B381B3E
:1010F000F77C1D901DA4BBE424203284725E228103
:1011000000C9F124ECA1E53D274E414E494E49541A
:1011100059494E46CDCCCC3D0AD7233C17B7D138E0
:1011200077CC2B329595E6241FB14F0A0000204161
:101130000000C84200401C4620BCBE4CCA1B0E5AD0
:10114000AEC59D7411241FBECFEFD1E4DEBFCDBF6D
:1011500019E0A0E0B2E0E2EFFDE101E00BBF02C068
:1011600007900D92AA34B107D9F710E3AAE4B9E0C9
:1011700001C01D92A63FB107E1F70E94227D0C94A9
:10118000F78E0C9400008DE694E09F938F930E945D
:10119000FF8B80914A0290914B020F900F9093FF2A
:1011A00003C087E694E002C081E694E09F938F93AA
:1011B0000E94FF8B0F900F900895E091031BEF7139
:1011C000F0E0E85AF44E80838091031B8F5F809398
:1011D000031B8091302888608093302844E352E0DC
:1011E00061E1CA010E94B24D80E090E00895CF9382
:1011F000DF93EC01809151099091520986FF1DC047
:101200008E811F928F938D811F928F938C811F925D
:101210008F938B811F928F938A811F928F938DE47E
:1012200093E09F938F930E94ED8B8DB79EB70C96A2
:101230000FB6F8949EBF0FBE8DBFBE0188E899E03F
:101240000E94E44EBE0184E092E0DF91CF910C94C5
:10125000594E87EE93E08115910511F00197F1F752
:1012600008958823B9F052985A981DBA8091690060
:10127000806280936900EA9A53985B98EB9A809118
:101280006900806880936900809168008160809324
:1012900068000895109269005A9AEA985B9AEB9850
:1012A00008951F920F920FB60F9211248F939F9360
:1012B000AF93BF938091680080FF20C08091102879
:1012C00090911128A0911228B09113280196A11D88
:1012D000B11D8093102890931128A0931228B093E9
:1012E0001328809151099091520987FF07C0749883
:1012F00082E090E09093710280937002BF91AF9171
:101300009F918F910F900FBE0F901F9018951F9275
:101310000F920FB60F9211248F939F93AF93BF93A9
:101320008091680080FF20C080911428909115283A
:10133000A0911628B09117280196A11DB11D809388
:10134000142890931528A0931628B09317288091FD
:1013500051099091520990FF07C0739882E090E084
:101360009093710280937002BF91AF919F918F9182
:101370000F900FBE0F901F90189580937C00809166
:101380007B00877F80937B0080917C00806C8093C2
:101390007C0085E080937A0080917A008068809359
:1013A0007A0080917B0087FFFCCF80917B0085FFD6
:1013B000FCCF80917A00806480937A0080917A00DB
:1013C00086FDFCCF109279001092780084E090E0C6
:1013D00060E070E020917A00206420937A002091F0
:1013E0007A0026FDFCCF2091780030917900620FC1
:1013F000731F0197009771F710927C0080917A001B
:101400008F7780937A00769567957695679580E0DB
:1014100090E00E947882089580E00E94BD092091AA
:101420006C0230916D0240916E0250916F020E94E9
:10143000588421EE3AE744E95EE30E941181089561
:1014400080E18093510160E16093510180915101ED
:1014500085FF03C06F5F6F31B9F78BE4689FB00100
:101460001124882777FD8095982F0E947A8220E0AA
:1014700030E64FE954E40E94118120E030E04AE771
:1014800054E40E94DB810895CF93DF93EC018881BF
:101490009981009799F088339F4021F01982188232
:1014A00083E011C0623171F40E94200A6093AB2383
:1014B0007093AC238093AD239093AE2388E39FE099
:1014C0009983888381E0DF91CF91089580917B009B
:1014D000886080937B0089EC80937C0085E080931A
:1014E0007A0080917A00806880937A0080917B00F6
:1014F00087FFFCCF80917B0085FFFCCF80917A0035
:10150000806480937A0080917A0086FDFCCF809180
:101510007A00806480937A0080917A0086FDFCCF07
:10152000609178007091790080917A008F77809334
:101530007A0080E090E00E94788227ED33EA40E96B
:101540005FE30E94588426E636E648E853E40E94AA
:1015500010810895BF92CF92DF92EF92FF920F9386
:101560001F93CF93DF93CDB7DEB729970FB6F894CB
:10157000DEBF0FBECDBF6C0110924A098FEF898785
:1015800004E11BE1B12C7E0189E0E80EF11C8985A4
:101590008823E9F1E8E0BE16E1F1BE016F5F7F4FFD
:1015A000C7010E944D5789858F3F11F08E3F19F476
:1015B00080934A092CC0CE010196C114D10471F464
:1015C0000E94665780932D28FE013196A5E2B8E26D
:1015D00081918D93EE15FF05D9F71DC00E946657C6
:1015E000F8018083FE01319620E030E0A8014850E8
:1015F00051098191DA01A20FB31F8C932F5F3F4FE6
:1016000028303105B1F7B394075F1F4FC0CF8B2D42
:1016100003C088E001C081E029960FB6F894DEBFD0
:101620000FBECDBFDF91CF911F910F91FF90EF9033
:10163000DF90CF90BF90089580EC9DE09F938F93B3
:101640000E94FF8B0F900F9008952F923F924F9220
:101650005F926F927F928F929F92AF92BF92CF9242
:10166000DF92EF92FF920F931F93CF93DF93EC01E2
:101670004B01009711F427E004C08130910549F433
:1016800026E04AE250E06BE270E089E290E00E94DE
:101690002D56CE010E94AA0A9E01255B364F5901A4
:1016A000D9018C93CD2B69F094E1C92E9BE1D92E01
:1016B000CCE0DBE1E12CF12C21E7222E2DE0322ED3
:1016C000A6C085E298E20E949B58BC01882777FD5E
:1016D0008095982F0E947A826B017C01892869F09D
:1016E00020E030E048EC52E40E94DB819F938F932E
:1016F0007F936F938EEA9DE0ACC0C5E2D8E209EA21
:101700001DE089911F928F931F930F930E94FF8B6F
:101710000F900F900F900F90B8E2CD32DB0789F752
:1017200020E030E048EC52E4C701B6010E94DB81C2
:101730009F938F937F936F9389E99DE09F938F93FE
:101740000E94FF8B0F900F900F900F900F900F90B3
:1017500080912D28882319F08CE793E002C080EF58
:1017600093E09F938F9385E99DE09F938F930E94D1
:10177000FF8B0F900F900F900F9075C000E010E05E
:10178000FE01E00FF11F80811F928F93ADE7BDE056
:10179000BF93AF930E94FF8B0F5F1F4F0F900F906F
:1017A0000F900F900830110559F720E030E048EC19
:1017B00052E4C301B2010E94DB819F938F937F9318
:1017C0006F93A5E7BDE0BF93AF930E94FF8B0F908F
:1017D0000F900F900F900F900F90D6018C9188234F
:1017E00009F455C08CE793E09F938F933F922F921B
:1017F0000E94FF8B0E941C0BBFEFEB1AFB0AE9E073
:10180000CE0ED11C29960F900F900F900F90D501FE
:101810008C9190E0E816F906ECF5CE010E949B58F9
:10182000BC01882777FD8095982F0E947A822B0132
:101830003C018114910409F4A1CF20E030E048EC90
:1018400052E40E94DB819F938F937F936F9382E892
:101850009DE09F938F930E94FF8B0F900F900F90AE
:101860000F900F900F90DF91CF911F910F91FF90EC
:10187000EF90DF90CF90BF90AF909F908F907F9030
:101880006F905F904F903F902F900C941C0B80EFC7
:1018900093E0AACFDF91CF911F910F91FF90EF902E
:1018A000DF90CF90BF90AF909F908F907F906F9080
:1018B0005F904F903F902F900895CF93DF9300D08B
:1018C000CDB7DEB780912628898380912C288A8322
:1018D000CE0101960E94A64B0F900F90DF91CF9101
:1018E0000895CF93DF93EC0120912528309126288D
:1018F00040912728509128286091292870912A2802
:1019000080912B2890912C28AFEF0E948887E1F4DA
:1019100027E04AE250E06BE270E089E290E00E944A
:101920002D5680E090E00E94AA0AC55BD64F8883BE
:1019300049E050E06AE070E085E298E20E94428D62
:10194000DF91CF910C945D0CDF91CF9108951F92A0
:101950000F920FB60F9211240BB60F92DF92EF92F7
:10196000FF920F931F932F933F934F935F936F9328
:101970007F938F939F93AF93BF93CF93DF93EF9317
:10198000FF938091302882608093302880914A02B2
:1019900086FD2B9A80914A0287FD2B9A80917002D6
:1019A000909171021816190614F4749A739A809122
:1019B00051099091520985FF02C0749873988091E3
:1019C0000202909103020197909303028093020216
:1019D000892B09F039C180915F09909160090196C6
:1019E0009093600980935F098091AF239091B02319
:1019F000A091B123B091B2230196A11DB11D809396
:101A0000AF239093B023A093B123B093B22380E18E
:101A100090E0909303028093020280914A0280FD3D
:101A200002C01D9B07C010924F0910924E0983B748
:101A3000817F09C081E090E090934F0980934E0927
:101A400083B7817F866083BF80915109909152094D
:101A500097FF08C080914E0990914F09892B61F042
:101A6000749A739803EB1AE1CCEBD3E234E0E32EE3
:101A7000F12CDD24D3941FC0739A7498F3CF809116
:101A80005F099091600901960E945985892BD1F0D8
:101A9000F801608571856115710509F5F8016085AA
:101AA00071856115710569F5065F1F4F2596FAE18D
:101AB0000B3D1F07D1F1F801608571856115710536
:101AC00039F3DDCF7798809151099091520992FFB7
:101AD000DFCF7498F0927102E0927002D9CF8091BA
:101AE0005F099091600901960E945985892BB1F692
:101AF0001C821B82AE0162E18CE092E00E94B24D3A
:101B0000CDCF80915F09909160090E945985892B02
:101B100059F6D8821A8309831C821B82AE0162E1C6
:101B20008AE292E00E94B24DBFCF60914E02709166
:101B30004F0261157105A1F180915F0990916009D3
:101B40000E945985892B61F5809110289091112868
:101B5000A0911228B09113284091A11B5091A21B73
:101B60006091A31B7091A41B841B950BA60BB70B54
:101B70008093DB1A9093DC1AA093DD1AB093DE1ADF
:101B80008091102890911128A0911228B0911328CB
:101B90008093A11B9093A21BA093A31BB093A41BA3
:101BA00060914C0270914D0261157105A1F1809117
:101BB0005F09909160090E945985892B61F5809198
:101BC000142890911528A0911628B09117284091BB
:101BD000A51B5091A61B6091A71B7091A81B841B8D
:101BE000950BA60BB70B8093DF1A9093E01AA09386
:101BF000E11AB093E21A8091142890911528A091CF
:101C00001628B09117288093A51B9093A61BA0932C
:101C1000A71BB093A81B80914A0286FD2B98809148
:101C20004A0290914B0291FF0FC00E943D628A319F
:101C300019F0C1E0C80F01C0CBE00E94F7608C2F03
:101C40000E9455620E943F6140E050E060E082E700
:101C500092E00E94B24DFF91EF91DF91CF91BF9141
:101C6000AF919F918F917F916F915F914F913F9134
:101C70002F911F910F91FF90EF90DF900F900BBE6F
:101C80000F900FBE0F901F9018958091031B90919D
:101C9000BB23891B08950E94450E882371F0E091B3
:101CA000BB23EF71F0E0E85AF44E808190E0209180
:101CB000BB232F5F2093BB2308958FEF9FEF0895E1
:101CC000CF93DF93EC0110927C0910927B098881FD
:101CD00099810097C1F08736934021F019821882CC
:101CE00083E0B6C0613109F0B2C0F89478940E94E4
:101CF0004B0E992790937709809376098D3009F4DC
:101D000041C08F3F49F40E94450E8111EECF87E616
:101D100093E0998388839BC08231910509F458C070
:101D20008F37910509F050C0809174099091750921
:101D3000181619060CF56091F0307091F13088E0BA
:101D400090E00E94BB8B6091F0307091F13080E2A6
:101D500090E00E94BB8B6091F0307091F13088E090
:101D600090E00E94BB8B8091740990917509019756
:101D70009093750980937409809174099091750905
:101D8000CF9709F61092BB231092031B8091740920
:101D900090917509FC01E053FC4D108290937C09F1
:101DA00080937B09109275091092740980912E28F6
:101DB00090912F28009709F4A6CF40E050E0609161
:101DC0008A110E94B24D9FCF8830910571F5ACCF3A
:101DD0006091F0307091F1308DE090E00E94BB8B0B
:101DE000109273091092720980917209909173098F
:101DF0002091740930917509821793070CF0BCCFBC
:101E0000FC01E053FC4D80816091F0307091F13025
:101E100090E00E94BB8B80917209909173090196AA
:101E20009093730980937209DFCF6091F0307091C5
:101E3000F1300E94BB8B80917409909175092091BB
:101E40007609FC01E053FC4D2083019691CF81E09F
:101E5000DF91CF91089580914E0990914F09892B80
:101E6000B1F080914A0290914B0293FD10C00E9404
:101E7000F76083B7817F866083BFF89483B7816002
:101E800083BF7894889583B78E7F83BF78940895B5
:101E9000CF93DF93EC0188819981009719F08D35FC
:101EA0009F4099F40E94B45F0E942B0F40E050E0E5
:101EB00065E880918E1190918F110E94B24D8DE551
:101EC0009FE09983888381E003C01982188283E0B0
:101ED000DF91CF910895CF93DF9300D0CDB7DEB7D8
:101EE000892B81F05F934F938EE69DE09F938F93B4
:101EF00069837A830E94FF8B0F900F900F900F9051
:101F00007A8169817F936F938BE69DE09F938F9396
:101F10000E94FF8B0F900F900F900F900F900F90DB
:101F2000DF91CF910895FF920F931F93CF93DF938B
:101F30000E94B45F80EB0E94195981111CC00E945D
:101F40007D598091A91F9091AA1F81609093AA1F2B
:101F50008093A91F85E893E09F938F938BE69DE084
:101F60009F938F930E94FF8B0F900F900F900F9075
:101F7000C1E0D0E002C0C0E0D0E0FEB08F2D8470A0
:101F8000F82E729A0E94B45F8EE40E941959811152
:101F900016C00E947D598091A91F9091AA1F82604E
:101FA0009093AA1F8093A91F8E010F5F1F4F40EBD4
:101FB00058E06DE873E0CE010E946B0FE801F1106C
:101FC00001C072980E94B45F8EEE0E94195981116F
:101FD00016C00E947D598091A91F9091AA1F84600C
:101FE0009093AA1F8093A91F8E010F5F1F4F40EB94
:101FF00058E065E973E0CE010E946B0FE8010E9492
:10200000B45F86EA0E941959811116C00E947D5959
:102010008091A91F9091AA1F88609093AA1F809316
:10202000A91F8E010F5F1F4F40EB58E06CE973E072
:10203000CE010E946B0FE8010E94B45F8CE30E9406
:10204000195981111EC00E947D598091A91F90913C
:10205000AA1F80619093AA1F8093A91F8E010F5F12
:102060001F4F40EB58E064EA73E0CE010E946B0F13
:1020700083E69DE09F938F930E94FF8B0F900F90BC
:10208000E8010E94B45F82ED0E941959811116C0C7
:102090000E947D598091A91F9091AA1F8062909300
:1020A000AA1F8093A91F8E010F5F1F4F40EB58E0BE
:1020B0006CEA73E0CE010E946B0FE8010E94B45FEE
:1020C00080E80E941959811116C00E947D598091A3
:1020D000A91F9091AA1F91609093AA1F8093A91F96
:1020E0008E010F5F1F4F40EB58E065EB73E0CE01B0
:1020F0000E946B0FE8010E94B45F80ED0E941959A5
:10210000811116C00E947D598091A91F9091AA1F2C
:1021100080689093AA1F8093A91F8E010F5F1F4FA5
:1021200040EB58E06BEB73E0CE010E946B0FE801CF
:102130000E94B45F8CEE0E941959811116C00E9452
:102140007D598091A91F9091AA1F92609093AA1F18
:102150008093A91F8E010F5F1F4F40EB58E063EC87
:1021600073E0CE010E946B0FE80107E010E00E94CF
:10217000B45F8CE70E941959811113C00E947D59E8
:102180008091A91F9091AA1F80649093AA1F8093A9
:10219000A91F40EB58E06AEC73E0CE010E946B0F80
:1021A00005C0015011090115110509F70E947D595B
:1021B000DF91CF911F910F91FF900C941C0BCF9347
:1021C000DF9300D0CDB7DEB74A8369830E945459AC
:1021D0006981862F0E9485594A81842F0E948559E2
:1021E0000F900F90DF91CF910C947D59AF92BF92D9
:1021F000DF92EF92FF920F931F93CF93DF9300D064
:102200001F92CDB7DEB7182FD22E4A835B83698326
:102210000E9454596981862F0E948559812F8160BF
:102220000E947B594A81A42E5B81B52E00E010E00C
:10223000ED2CF12C81E0E81AF1080D1580F40E1553
:102240001F0519F40E94A05902C00E949659F50179
:1022500080830F5F1F4FFFEFAF1ABF0AEECF0F90C3
:102260000F900F90DF91CF911F910F91FF90EF9002
:10227000DF90BF90AF900C947D59AF92BF92CF92F8
:10228000DF92EF92FF920F931F93CF93DF93CDB71F
:10229000DEB760970FB6F894DEBF0FBECDBFB82E85
:1022A000A42E6623E9F18E010F5F1F4F80E1F80134
:1022B00011928A95E9F728E0A80168E980EB0E946D
:1022C000F610BB2041F023ED33E03F932F930E94A3
:1022D000ED8B0F900F906E01F8E0CF0ED11C5AEDF0
:1022E000E52E53E0F52EF80181918F011F928F9317
:1022F000FF92EF920E94ED8B0F900F900F900F9036
:102300000C151D0581F788851F928F932FE234E00D
:102310003F932F930E94ED8B0F900F900F900F9093
:10232000AA20E9F18E010F5F1F4F80E1F8011192A1
:102330008A95E9F728E0A80160E880EB0E94F61092
:10234000BB2041F08FED93E09F938F930E94ED8B24
:102350000F900F906E01F0E1CF0ED11C4AEDE42EEC
:1023600043E0F42EF80181918F011F928F93FF9229
:10237000EF920E94ED8B0F900F900F900F900C1525
:102380001D0581F788851F928F938FE294E09F93BC
:102390008F930E94ED8B0F900F900F900F9060968F
:1023A0000FB6F894DEBF0FBECDBFDF91CF911F9166
:1023B0000F91FF90EF90DF90CF90BF90AF90089576
:1023C000CF93DF9300D0CDB7DEB71A82198222E017
:1023D000AE014F5F5F4F6AEA8EEE0E94F610898170
:1023E00090E0982F88272A81822B9093791B8093E5
:1023F000781B22E0AE014F5F5F4F6CEA8EEE0E94C9
:10240000F610898190E0982F88272A81822B90935B
:102410007B1B80937A1B22E0AE014F5F5F4F6EEA19
:102420008EEE0E94F610898190E0982F88272A81ED
:10243000822B90937D1B80937C1B22E0AE014F5F2B
:102440005F4F60EB8EEE0E94F610898190E0982F2E
:1024500088272A81822B90938B1B80938A1B22E0F2
:10246000AE014F5F5F4F62EB8EEE0E94F6108981E6
:1024700090E0982F88272A81822B90938D1B809340
:102480008C1B22E0AE014F5F5F4F64EB8EEE0E942B
:10249000F610898190E0982F88272A81822B9093CB
:1024A0008F1B80938E1B22E0AE014F5F5F4F66EB68
:1024B0008EEE0E94F610898190E0982F88272A815D
:1024C000822B90937F1B80937E1B22E0AE014F5F97
:1024D0005F4F68EB8EEE0E94F610898190E0982F96
:1024E00088272A81822B9093811B8093801B22E076
:1024F000AE014F5F5F4F6AEB8EEE0E94F61089814E
:1025000090E0982F88272A81822B9093851B8093B7
:10251000841B22E0AE014F5F5F4F6CEB8EEE0E949A
:10252000F610898190E0982F88272A81822B90933A
:10253000871B8093861B22E0AE014F5F5F4F6EEBDF
:102540008EEE0E94F610898190E0982F88272A81CC
:10255000822B9093891B8093881B0F900F90DF91A3
:10256000CF9108952F923F924F925F926F927F92F8
:102570008F929F92AF92BF92CF92DF92EF92FF9293
:102580000F931F93CF93DF93CDB7DEB76A970FB644
:10259000F894DEBF0FBECDBF182F488F298F198248
:1025A0001A821B8280919C1B811107C06A8F0E9436
:1025B000E01181E080939C1B6A8D662309F46CC056
:1025C0004EE264EF8EEE0E94DF1069E07AE180E077
:1025D00090E00E94065922E0AE014F5F5F4F66EF28
:1025E0008EEE0E94F6102981822F90E0A0E0B0E0EC
:1025F0002227382F492F5A2F8A81282B80918E1B12
:1026000090918F1B281B390B41095109A0918C1BFC
:10261000B0918D1B0E9436856B017C018FE0F59493
:10262000E794D794C7948A95D1F76091861B7091EF
:10263000871B882777FD8095982F2BE0660F771FE3
:10264000881F991F2A95D1F72091881B3091891BEB
:10265000442737FD4095542F2C0D3D1D4E1D5F1D09
:102660000E94A385C20ED31ED092831BC092821BF0
:1026700088E0C80ED11C34E0D594C7943A95E1F7B0
:10268000EE24D7FCE094FE2CC092901BD092911BBC
:10269000E092921BF092931B012F0295000F000F06
:1026A000007C0C5CA12FB0E0BD8BAC8BA3E0B0E054
:1026B000012E02C0AA0FBB1F0A94E2F725E335E002
:1026C0000E942F85DC01CB010296A11DB11D8C87D4
:1026D0009D87AE87BF8780E593ECA0E0B0E004C0A3
:1026E000B595A795979587951A95D2F7888B998B6D
:1026F000AA8BBB8B10E0188619861A861B86A8E069
:102700002A2E312CAC89BD892A1A3B0A988D1917BB
:1027100009F436C1402F64EF8EEE0E94DF106C8505
:102720007D858E859F850E94065923E0AE014F5F0F
:102730005F4F66EF8EEE0E94F610E091821BF091E3
:10274000831BE05AFF409F01DF010E9418856B0147
:102750007C0180917A1B90917B1B9F8B8E8BA0902C
:10276000781BB090791B20917C1B30917D1B0E94BF
:1027700018852B013C013DE075946794579447946C
:102780003A95D1F7A0917E1BB0917F1BA7019601CE
:102790006CE055954795379527956A95D1F70E9436
:1027A0004185BB2797FDB095AB2F480E591E6A1E79
:1027B0007B1E92E0490E511C611C711CB2E07594A5
:1027C000679457944794BA95D1F7A0E85A0E611CC4
:1027D000711CA0918A1BB0918B1BA30192010E94D6
:1027E0003685DC01CB012FE0B695A79597958795A7
:1027F0002A95D1F78C839D83AE83BF8329818A81FB
:1028000090E0A0E0B0E04424582E692E7A2E622A8F
:102810008B81482A022C04C075946794579447947E
:102820000A94D2F74501AA2497FCA094BA2C42E05E
:10283000880C991CAA1CBB1C4A95D1F7A091801B3F
:10284000B091811BA70196010E9441856B017C011B
:1028500057E1F594E794D794C7945A95D1F72E8908
:102860003F89DF010E941885EBE095958795779564
:102870006795EA95D1F7C60ED71EE81EF91E8C0C97
:102880009D1CAE1CBF1C0C8804C0880C991CAA1C83
:10289000BB1C0A94D2F792E0890E911CA11CB11CBA
:1028A000F2E0B594A79497948794FA95D1F74818D5
:1028B00059086A087B08A3019201688979898A8985
:1028C0009B890E94498597FD0DC0660F771F881F61
:1028D000991F2C813D814E815F810E948185490134
:1028E0005A010CC02C813D814E815F810E948185FF
:1028F00049015A01880C991CAA1CBB1C9927B7FCDA
:102900009A958B2D7A2D692D9B01AC010E944985EA
:102910009B01AC01AEEDBBE00E9436856C01FF244B
:10292000D7FCF094EF2CA3E4B3EEA50194010E9430
:102930004485BB2797FDB095AB2FC80ED91EEA1E64
:10294000FB1EAFECCA0EAEE0DA1EE11CF11CA4E0E7
:10295000F594E794D794C794AA95D1F7C80CD91CDD
:10296000EA1CFB1C88859985AA85BB858C0D9D1D5D
:10297000AE1DBF1D88879987AA87BB871F5FC6CEFC
:10298000112391F0212F30E040E050E068857985F7
:102990008A859B850E9481852093941B3093951B8B
:1029A0004093961B5093971BA98DAA2389F16091A0
:1029B000941B7091951B8091961B9091971B6115AC
:1029C00071058105910521F10E947A8220E836EE99
:1029D00045EC57E40E94DB8121E03EED42E45EE3FA
:1029E0000E94BB849B01AC0160E070E080E89FE343
:1029F0000E9410812BE43AE34DEB57E30E94DB8108
:102A00006093981B7093991B80939A1B90939B1BC8
:102A10006A960FB6F894DEBF0FBECDBFDF91CF919F
:102A20001F910F91FF90EF90DF90CF90BF90AF90EC
:102A30009F908F907F906F905F904F903F902F90DE
:102A400008950F931F93CF93DF9300D000D000D051
:102A5000CDB7DEB78E010F5F1F4F86E0F8011192F0
:102A60008A95E9F78091AA1A811113C040E061E3C9
:102A700086EA0E94DF104AE06CE286EA0E94DF10DC
:102A800081E08093AA1A6CE77EE380E090E00E94E8
:102A9000065948E06DE286EA0E94DF106CE77EE3AB
:102AA00080E090E00E94065926E0A80162E386EAF1
:102AB0000E94F61047E06DE286EA0E94DF108A81EC
:102AC00090E0982F88272981822B9093A51A8093D4
:102AD000A41A2C8130E0322F22274B81242B3093F3
:102AE000A71A2093A61A4E8150E0542F44276D81D7
:102AF000462B5093A91A4093A81A5F934F933F9384
:102B00002F939F938F9383EE93E09F938F930E94D5
:102B1000ED8B0FB6F894DEBF0FBECDBF26960FB675
:102B2000F894DEBF0FBECDBFDF91CF911F910F9103
:102B30000895CF92DF92EF92FF920F931F93CF935E
:102B4000DF93CDB7DEB72A970FB6F894DEBF0FBE7E
:102B5000CDBF8E010F5F1F4F86E0F80111928A955D
:102B6000E9F741E062E08CE30E94DF1048E560E0B5
:102B70008CE30E94DF1062E174E380E090E00E9449
:102B8000065926E0A80163E08CE30E94F61043E0BA
:102B900062E08CE30E94DF10098110E0102F002713
:102BA0008A81082B1093851A0093841AEB80F12CEC
:102BB000FE2CEE248C81E82AF092871AE092861A85
:102BC000CD80D12CDC2CCC248E81C82AD092891ABD
:102BD000C092881AB801882777FD8095982F0E94A7
:102BE0007A829B01AC01B701882777FD8095982FE9
:102BF0002F83388749875A870E947A822F813885A8
:102C000049855A850E94848120EE3EE245E652E4E1
:102C10000E94588420E030E044E353E40E94118194
:102C20009F938F937F936F93DF92CF92FF92EF9258
:102C30001F930F9381EF93E09F938F930E94ED8BEF
:102C40000FB6F894DEBF0FBECDBF2A960FB6F8942C
:102C5000DEBF0FBECDBFDF91CF911F910F91FF90CF
:102C6000EF90DF90CF900895CF93DF93EC018881B0
:102C700099810097F9F086349F4021F019821882DB
:102C800083E063C081E699E00E945850892BE1F00F
:102C9000809151099091520993FD18C0809151097A
:102CA0009091520994FD43C080915109909152092D
:102CB00095FD44C060E870E081E699E00E943150E3
:102CC00086E49FE09983888381E03FC08091A91FBB
:102CD00082FFE4CF21E048E061E083E00E94B2128D
:102CE00080919B1B8F9380919A1B8F938091991B4E
:102CF0008F938091981B8F938091971B8F938091D6
:102D0000961B8F938091951B8F938091941B8F932B
:102D100082EC9DE09F938F930E94FF8B8DB79EB7AF
:102D20000A960FB6F8949EBF0FBE8DBFB7CF8091A5
:102D3000A91F83FFB9CF0E942115B6CF8091A91F8B
:102D400084FFB8CF0E949915B5CFDF91CF91089538
:102D5000CF93C82F8CEE0E947B598C2F0E948559EF
:102D600065E375E080E090E00E9406598DEE0E94D8
:102D70007B590E949659C82F0E94A0592C2F30E0F1
:102D8000322F2227A901482BCA01CF910895CF9352
:102D9000DF93C82F8CEE0E947B598C2F0E9485599F
:102DA00062E174E380E090E00E9406598CEE0E949C
:102DB0007B5980E00E94855965E375E080E090E0F2
:102DC0000E9406598DEE0E947B590E949659C82F89
:102DD0000E949659D82F0E94A0594D2F50E060E0D4
:102DE00070E0762F652F542F44276C2B482BCB0196
:102DF000BA01DF91CF9108952F923F924F925F9247
:102E00006F927F928F929F92AF92BF92CF92DF92FA
:102E1000EF92FF920F931F93CF93DF93CDB7DEB75F
:102E2000CD54D1090FB6F894DEBF0FBECDBF80914F
:102E3000000290910102892BD1F1109201021092AF
:102E400000028CEE0E947B598EE10E9485596BE155
:102E50007EE480E090E00E94065982EA0E94A81673
:102E600090935E0980935D0984EA0E94A81690936E
:102E70005C0980935B0986EA0E94A81690935A0920
:102E80008093590988EA0E94A81690935809809364
:102E900057098AEA0E94A81690935609809355090B
:102EA0008CEA0E94A816909354098093530988E4F1
:102EB0000E94C7166FAB78AF89AF9AAF88E50E94C2
:102EC000C7164B015C01809155099091560920E08D
:102ED00030E040E050E0BA0126962FAF26972796C3
:102EE0003FAF279728964FAF289729965FAF29972E
:102EF0002A966FAF2A972B967FAF2B979C0140E0C5
:102F000050E060E070E080E090E008E00E942A87F6
:102F10000E94D6863901B42FA52FF62FE72F8C01FA
:102F20009401A50160E070E080E090E05301CB2EB9
:102F3000DA2EEF2EFE2E0E94618729833A832A0122
:102F40001B014C01B101C401315041095F4F6F4F6A
:102F50007F4F8F4F9F4FA1E0B0E02596BFAFAEAF40
:102F6000259721153F4F4F4F514061057105810550
:102F7000910509F020F425961FAE1EAE25972596E3
:102F80006EAC7FAC259780915309909154095C01F8
:102F9000C12CD12CE12CF12C00E010E029813A81E8
:102FA000A201B101C4010E94F985D22EE32EF42EB4
:102FB000052F162FB72FF82FE92FA0E00E94888742
:102FC00084F42150310940485F4F6F4F7F4F8F4F3E
:102FD0009F4FD22EE32EF42E052F162FB72FF82F4A
:102FE000E92F2D2D3E2D4F2D502F612F7B2F8F2F11
:102FF0009E2F07E10E9443872B8F3C8F4D8F5E8F62
:103000006F8F78A389A39AA32053384F4F4F5F4FF8
:103010006F4F7F4F8F4F9F4F2B8B3C8B4D8B5E8B1A
:103020006F8B788F898F9A8F2056304F4F4F5F4F1D
:103030006F4F7F4F8F4F9F4F243D304341055105C8
:10304000610571058105910541F038F025966EAC5A
:103050007FAC2597FFEF6F1A7F0A80915B099091F3
:103060005C099C0140E050E060E070E080E090E0AE
:1030700000E10E942A872B833C834D835E836A870D
:1030800079878F8398874091570950915809A98073
:10309000BA806201710184019A0140E050E060E071
:1030A00070E080E090E00E94F985D22EE32EF42EAD
:1030B000052F162FB72FF82FE92FA0E00E94888741
:1030C0005CF4AFE70E946A87D22EE32EF42E052F20
:1030D000162FB72FF82FE92F2D2D3E2D4F2D502FC6
:1030E000612F7B2F8F2F9E2F07E00E94438759016E
:1030F0006A017B018C012B813C814D815E816A8557
:1031000079858F8198850E9461872B833C834D83CD
:103110005E836F8378878F87988B2E5F3F4F434006
:1031200051096E4F7F4F8F4F9F4F22303105494FCE
:103130005F4F644071058105910521F018F01FEF84
:10314000611A710A80915D0990915E09BC0180E06D
:1031500090E020E030E840E050E00E94528629876D
:103160003A874B875C876A8B798B8D879E874091E6
:10317000590950915A09A980BA80620171018401EC
:103180009A0140E050E060E070E080E090E00E9452
:10319000F985D22EE32EF42E052F162FB72FF82FF8
:1031A000E92FA0E00E94888784F421503F4F4F4FC1
:1031B0005F4F6F4F7F4F8F4F9F4FD22EE32EF42ED6
:1031C000052F162FB72FF82FE92F2D2D3E2D4F2D20
:1031D000502F612F7B2F8F2F9E2F08E00E94438757
:1031E00059016A017B018C0129853A854B855C85F3
:1031F0006A8979898D859E850E94618729873A87AA
:103200004B875C876D877E87898B9A8B2F5F3F4FBB
:103210004140510961097109810991092130304802
:103220004C4F5F47614071058105910521F018F011
:10323000BFEF6B1A7B0A2B893C894D895E896F89A8
:10324000788D898D9A8D2F3C374041055105610558
:1032500071058105910511F00CF0A5C1A980BA8016
:103260006201710184019501A201B101C4010E94B2
:10327000F985A12CB12CC12C10E8D12EE12CF12C18
:1032800000E010E00E94BC852BAF3CAF4DAF5EAFBD
:103290006FAF21967FAF219722968FAF229723960B
:1032A0009FAF2397AB8CBC8CCD8CDE8CEF8CF8A0C1
:1032B00009A11AA19501A601B701C8010E94F985CB
:1032C00059016A017B01E82F192F02E00E942A8729
:1032D0000E2F0E94618769017A01162F272EF82F81
:1032E000E92F322E8D2C942EAF2CB62E072F582E70
:1032F000B92FA0E00E9488875CF4A1E00E946A8751
:10330000322E832E942EA52EB62E072F582EB92F8F
:10331000232D382D492D5A2D6B2D702F852D9B2F48
:1033200001E00E9443872E962FAF2E972D963FAF38
:103330002D9749A75AA76BA77CA78DA79EA7522EAA
:10334000432E4BA35CA36DA37EA38FA398A7B22D9E
:103350009601A701612F722D8F2F9E2FA0E00E9452
:1033600088874CF4A3E00E946A8769017A01162FCE
:10337000B72FF82FE92F9601A701612F7B2F8F2FF1
:103380009E2F02E00E9443872FA738AB49AB5AAB70
:103390006BAB7CAB8DAB9EAB19014A01B62FA72F4F
:1033A00024968FAF2497F92F2B893C894D895E890C
:1033B0006F89788D898D9A8D24323A4F4F4F5F4FA8
:1033C0006F4F7F4F8F4F9F4F0CF08CC02B8D3C8DDC
:1033D0004D8D5E8D6F8D78A189A19AA12455324FB4
:1033E0004F4F5F4F6F4F7F4F8F4F9F4F59016A0174
:1033F0007B018C010E94F98519014A01B62FA72F84
:10340000FC0103E00E942A8751016401EB2EFA2E91
:103410008F010E94768759016A017B018C012E96EB
:103420002FAD2E972D963FAD2D9749A55AA56BA58B
:103430007CA58DA59EA50E946187522E432E4BA38D
:103440005CA36DA37EA38FA398A79101A4016B2F0A
:103450007A2FCF0102E00E942A8751016401EB2EEE
:10346000FA2E8F010E94768702E00E942A870E2F93
:103470000E947687F22E032F142FD52EE62EB72F1B
:10348000F82FE92FA0E00E9488875CF4A1E00E9459
:103490006A87F22E032F142FD52EE62EB72FF82F82
:1034A000E92F2F2D302F412F5D2D6E2D7B2F8F2F4C
:1034B0009E2F01E00E94438759016A017B018C0124
:1034C0002FA538A949A95AA96BA97CA98DA99EA99C
:1034D0000E94618719014A01B62FA72F24968FAF4A
:1034E0002497F92F2B813C814D815E816F817885F6
:1034F0008F859889A52CB42CCBA0DCA0EDA0FEA0D4
:103500000FA118A50E9476872B833C834D835E8391
:103510006F8378878F87988B29853A854B855C8563
:103520006D857E8589899A8951016401EB2EFA2E79
:1035300024960FAD24971F2F0E94768729873A87FC
:103540004B875C876D877E87898B9A8B2B893C891B
:103550004D895E896F89788D898D9A8DABACBCACB5
:10356000CDACDEACEFAC2196FFAC219722960FAD2F
:10357000229723961FAD23970E9476872056304FBF
:103580004F4F5F4F6F4F7F4F8F4F9F4F243D3043C3
:1035900041055105610571058105910521F018F07E
:1035A0002FEF621A720A6FA978AD89AD9AADAB019F
:1035B000BC0180E090E0DC0124964FAF2497259673
:1035C0005FAF259726966FAF269727967FAF2797F1
:1035D00028968FAF289729969FAF29972A96AFAF45
:1035E0002A972B96BFAF2B97A984BA84CB84DC840F
:1035F000ED84FE8409891A899A01AB0160E070E0CC
:1036000080E090E00E94F985F22E032F142FD52E32
:10361000E62EB72FF82FE92FA0E00E94888784F4C8
:1036200021503109404E5F4F6F4F7F4F8F4F9F4F5B
:10363000F22E032F142FD52EE62EB72FF82FE92FB9
:103640002F2D302F412F5D2D6E2D7B2F8F2F9E2FF5
:1036500005E10E944387AB80BC80CD80DE80EF8097
:10366000F8840F8518890E947687F22E032F142F75
:10367000D52EE62EB72FF82FE92FA0E00E948887DD
:1036800084F4215030484F4F5F4F6F4F7F4F8F4F23
:103690009F4FF22E032F142FD52EE62EB72FF82F83
:1036A000E92F2F2D302F412F5D2D6E2D7B2F8F2F4A
:1036B0009E2F0FE00E94438769017A018B018A8364
:1036C000998329011A014B015C01285E33404109AD
:1036D00051096109710981099109283D304D414025
:1036E0005105610571058105910521F018F0BFEFC5
:1036F0006B1A7B0A0E947D59672859F09601A70131
:10370000B8018A8199810E94D68629011A014B014C
:103710005C019201A101B401C5010E94748220E004
:1037200030E048EC52E40E94DB81C35BDF4F0FB610
:10373000F894DEBF0FBECDBFDF91CF911F910F91E7
:10374000FF90EF90DF90CF90BF90AF909F908F90C1
:103750007F906F905F904F903F902F9008954F9281
:103760005F926F927F928F929F92AF92BF92CF9211
:10377000DF92EF92FF922B013C0169017A0123EC69
:1037800035EF4CE851E4C701B6010E9458844B0163
:103790005C0128EB3EE143E753E4C701B6010E9418
:1037A00011819B01AC01C501B4010E94DB810E9423
:1037B00048824B015C0120E030E048EC52E4C30158
:1037C000B2010E94DB8121E835E943EC50E40E941C
:1037D0005884A50194010E9458844B015C0123E3A5
:1037E00033E948E853E4C701B6010E9411819B0107
:1037F000AC01C501B4010E94DB8123E333EB48E552
:1038000053E40E945884FF90EF90DF90CF90BF90D8
:10381000AF909F908F907F906F905F904F900895A2
:103820004F925F926F927F928F929F92AF92BF92D0
:10383000CF92DF92EF92FF9269017A010E94DA83C0
:1038400020E030E040E050E40E94108122E93CE5B5
:103850004EED5EE30E94DB814B015C0123EC35EF12
:103860004CE851E4C701B6010E9458842B013C0189
:1038700028EB3EE143E753E4C701B6010E94118102
:103880009B01AC01C301B2010E94DB819B01AC0131
:10389000C501B4010E9411816B017C0128EB3EE15E
:1038A00043E753E40E9458844B015C01A701960151
:1038B00063EC75EF8CE891E40E9410819B01AC01F0
:1038C000C501B4010E94DB81FF90EF90DF90CF90A3
:1038D000BF90AF909F908F907F906F905F904F9030
:1038E00008954F925F926F927F928F929F92AF92C4
:1038F000BF92CF92DF92EF92FF922B013C016901C0
:103900007A0123EC35EF4CE851E4C701B6010E947F
:1039100058844B015C0128EB3EE143E753E4C701C7
:10392000B6010E9411819B01AC01C501B4010E9446
:10393000DB810E9448824B015C0120E030E048ECD2
:1039400052E4C301B2010E94DB81A50194010E94EF
:10395000588420E030E040E251E40E94108124EEDF
:1039600038E34EE05FE30E9458849B01AC01C7013D
:10397000B6010E941181FF90EF90DF90CF90BF9031
:10398000AF909F908F907F906F905F904F90089531
:10399000CF92DF92EF92FF920F931F93CF93DF931B
:1039A00080E80E947B598AEF0E9485598FE00E942F
:1039B000855965E375E080E090E00E94065981E852
:1039C0000E947B590E949659C82F0E9496590E94C6
:1039D0009659D82F0E9496590E949659182F0E94E6
:1039E00096590E94A059082F0E94A05980E80E9471
:1039F0007B598CEF0E94855989EC0E94855965E3BB
:103A000075E080E090E00E94065981E80E947B59B1
:103A10000E949659D82E0E949659C82E0E949659F7
:103A20000E949659F82E0E949659E82E0E94A0599D
:103A30001F92CF921F92DF921F920F931F921F939C
:103A40001F92DF931F92CF931F92EF921F92FF92CC
:103A500086E094E09F938F930E94ED8B0E947D59A6
:103A60008DB79EB742960FB6F8949EBF0FBE8DBF1E
:103A700020E030E040E050E060E070E080E090E086
:103A8000DF91CF911F910F91FF90EF90DF90CF903A
:103A900008950F931F93CF93DF93EC0180E80E946A
:103AA0007B59209741F085EE0E94855961E077E9C6
:103AB00080E090E007C083EE0E94855969E97AEBC7
:103AC00081E090E00E94065981E80E947B590E94A3
:103AD0009659182F0E949659082F0E94A0590E94AB
:103AE0007D59602F70E0712B6C7F80E090E0CD2BD2
:103AF00069F00E94788220E030E04AEF5AE30E94A9
:103B0000588420E030E040EC50E40CC00E94788201
:103B100022E538EB4FE25BE30E94588426E636E666
:103B20004BE352E40E941081DF91CF911F910F91DE
:103B300008950F931F93CF93DF93729A80914A0257
:103B400083FF08C08EE40E941959811163C0C0E54B
:103B5000D0E008C0C0E5D0E00E9429092197209755
:103B6000D9F7F0CF0E94290921972097D9F78FE440
:103B70000E9419590E949659082F0F730E94965956
:103B8000182F0E949659D82F0E94A059C82F0E9422
:103B90007D5980914A0283FF7298602F70E0762FE2
:103BA0006627610F711D80E090E00E94788220E11D
:103BB00034E048EC5BE30E94588460939D1B709353
:103BC0009E1B80939F1B9093A01B6D2F70E0762F00
:103BD00066276C0F711D769567957695679580E0E1
:103BE00090E00E94788224EA3CEF44E25CE30E9489
:103BF000588420E030E040E252E40E94108160935B
:103C0000312870933228809333289093342880E0B1
:103C100090E002C081E090E0DF91CF911F910F9181
:103C200008957298729A8EE40E94195980EA0E944F
:103C3000855980E00E94855980E00E9485598FE473
:103C40000E9419590E9496598EE40E94195980E8E1
:103C50000E94855980E00E94855980E00E94855924
:103C60000E947D5980E090E0089586E59DE09F9355
:103C70008F930E94FF8B809163020F900F90882397
:103C800061F01F928F9383E59DE09F938F930E9435
:103C9000FF8B0F900F900F900F9008958EE29DE094
:103CA0009F938F930E94FF8B86E09DE09F938F935D
:103CB0000E94FF8B8FED9CE09F938F930E94FF8B60
:103CC00084EA9CE09F938F930E94FF8B82E79CE0A5
:103CD0009F938F930E94FF8B86E39CE09F938F932B
:103CE0000E94FF8B80E19CE09F938F930E94FF8B4B
:103CF0008AED9BE09F938F930E94FF8B8091A91F79
:103D00009091AA1F827091702DB73EB7205F3F4FF0
:103D10000FB6F8943EBF0FBE2DBF892B41F08AEA43
:103D20009BE09F938F930E94FF8B0F900F908EE7E5
:103D30009BE09F938F930E94FF8B85E59BE09F9371
:103D40008F930E94FF8B89E29BE09F938F930E9449
:103D5000FF8B8AEF9AE09F938F930E94FF8B88ECF2
:103D60009AE09F938F930E94FF8B87E99AE09F933D
:103D70008F930E94FF8B8DE59AE09F938F930E9413
:103D8000FF8B8DE29AE09F938F930E94FF8B81E0DF
:103D90009AE09F938F930E94FF8B82ED99E09F930F
:103DA0008F930E94FF8B89E999E09F938F930E94E4
:103DB000FF8B80E699E09F938F930E94FF8B89E2AF
:103DC00099E09F938F930E94FF8B88EF98E09F93D9
:103DD0008F930E94FF8B89EC98E09F938F930E94B2
:103DE000FF8B8AE998E09F938F930E94FF8B8DB79A
:103DF0009EB780960FB6F8949EBF0FBE8DBF83E727
:103E000098E09F938F930E94FF8B8DE398E09F93A0
:103E10008F930E94FF8B87E098E09F938F930E947F
:103E2000FF8B8EED97E09F938F930E94FF8B83EA29
:103E300097E09F938F930E94FF8B88E797E09F9373
:103E40008F930E94FF8B2DB73EB7245F3F4F0FB675
:103E5000F8943EBF0FBE2DBF089585E394E00C9407
:103E6000238C4F925F926F927F928F929F92AF922C
:103E7000BF92CF92DF92EF92FF92CF93DF93CDB7B5
:103E8000DEB728970FB6F894DEBF0FBECDBF809186
:103E9000AF239091B023A091B123B091B223898335
:103EA0009A83AB83BC834090AF235090B023609043
:103EB000B1237090B2238091AF239091B023A09151
:103EC000B123B091B2238D839E83AF83B887609175
:103ED000AF237091B0238091B1239091B2232CE352
:103EE000822E912CA12CB12CA50194010E948185D8
:103EF0007F936F9330E1C32E3EE0D32EE12CF12C63
:103F00006D817E818F819885A70196010E948185B0
:103F1000A50194010E9481853F932F9340E8842E50
:103F200041E5942EAA24A394B12CC301B201A501AA
:103F300094010E948185A70196010E9481853F938B
:103F40002F9369817A818B819C81A50194010E94C4
:103F500081853F932F9382E597E09F938F930E94F3
:103F6000FF8B0FB6F894DEBF0FBECDBF28960FB6FD
:103F7000F894DEBF0FBECDBFDF91CF91FF90EF90E1
:103F8000DF90CF90BF90AF909F908F907F906F9079
:103F90005F904F900895E6EFF0E380819181823445
:103FA000924479F0E65FF043FF93EF9384E397E068
:103FB0009F938F930E94FF8B0F900F900F900F9005
:103FC00008953A96E53F81E4F80738F30895CF93D2
:103FD000DF93EC018C9A0E940C0A9F938F937F933E
:103FE0006F9388E297E09F938F930E94FF8B0F90CF
:103FF0000F900F900F900F900F90209719F00E9444
:104000001C0B08C086E297E09F938F930E94FF8B62
:104010000F900F9081E00E94BD09209168023091BD
:10402000690240916A0250916B020E9458849F93EA
:104030008F937F936F938AE197E09F938F930E9472
:10404000FF8B0F900F900F900F900F900F90209775
:1040500019F00E941C0B08C088E197E09F938F9392
:104060000E94FF8B0F900F9082E00E94BD0920916B
:1040700064023091650240916602509167020E948D
:1040800058849F938F937F936F938CE097E09F93D7
:104090008F930E94FF8B0F900F900F900F900F90B7
:1040A0000F90209719F00E941C0B08C08AE097E03F
:1040B0009F938F930E94FF8B0F900F9083E00E943D
:1040C000BD099F938F937F936F938BEF96E09F93A0
:1040D0008F930E94FF8B8C980F900F900F900F90F2
:1040E0000F900F90209719F00E941C0B08C089EFC9
:1040F00096E09F938F930E94FF8B0F900F9080917B
:10410000A91F87FF83C021E042E161E080ED0E94AA
:10411000DD5A9F938F937F936F938CEE96E09F93DE
:104120008F930E94FF8B0F900F900F900F900F9026
:104130000F90209719F00E941C0B08C08AEE96E0A1
:104140009F938F930E94FF8B0F900F9021E042E18D
:1041500062E080ED0E94DD5A9F938F937F936F936F
:104160008DED96E09F938F930E94FF8B0F900F90A1
:104170000F900F900F900F90209719F00E941C0B3A
:1041800008C08BED96E09F938F930E94FF8B0F905A
:104190000F9021E042E163E080ED0E94DD5A9F93A1
:1041A0008F937F936F938EEC96E09F938F930E94F3
:1041B000FF8B0F900F900F900F900F900F90CD2BC3
:1041C00019F00E941C0B08C08CEC96E09F938F9313
:1041D0000E94FF8B0F900F9021E042E164E080EDA0
:1041E0000E94DD5A9F938F937F936F938FEB96E09E
:1041F0009F938F930E94FF8B0F900F900F900F90C3
:104200000F900F90DF91CF910C941C0BCD2BD1F31D
:10421000DF91CF9108950F931F93CF93DF9388235E
:1042200089F049E050E06FEF70E085E298E20E948B
:104230005B8B49E050E06AE070E085E298E20E9422
:10424000428D13C0C5E2D8E20AEB16E089911F92B5
:104250008F931F930F930E94FF8B0F900F900F90DF
:104260000F9088E2CD32D80789F7DF91CF911F9167
:104270000F910C941C0BCF92DF92EF92FF92CF9391
:10428000DF936B017C0160FF11C082E794E09F9394
:104290008F938BE69DE09F938F930E94FF8B0F90EF
:1042A0000F900F900F9081E090E002C080E090E0CE
:1042B000C1FE09C0EC01219640EB58E067E774E0CD
:1042C0000E946B0FCE01C2FE09C0EC01219640EBAB
:1042D00058E06FE774E00E946B0FCE01C3FE09C087
:1042E000EC01219640EB58E067E874E00E946B0F08
:1042F000CE01C4FE09C0EC01219640EB58E06BE80A
:1043000074E00E946B0FCE01C5FE09C0EC0121963E
:1043100040EB58E06EE874E00E946B0FCE01C6FEE1
:1043200009C0EC01219640EB58E062E974E00E947C
:104330006B0FCE01C7FE09C0EC01219640EB58E09F
:1043400068E974E00E946B0FCE01D0FE09C0EC0159
:10435000219640EB58E060EA74E00E946B0FCE01BA
:10436000D1FE09C0EC01219640EB58E068EA74E008
:104370000E946B0FCE01D2FE09C0EC01219640EBEA
:1043800058E06CEA74E00E946B0FCE012091A91FE7
:104390003091AA1F24703270232B59F0D3FE09C02C
:1043A000EC01219640EB58E062EB74E00E946B0F49
:1043B000CE012091A91F23FF0BC0D4FE09C0EC0140
:1043C000219640EB58E067EB74E00E946B0FCE0142
:1043D0002091A91F24FF0BC0D5FE09C0EC01219636
:1043E00040EB58E06DEB74E00E946B0FCE01D6FEFF
:1043F00009C0EC01219640EB58E065EC74E00E94A6
:104400006B0FCE01B701A60144275078452B462BF0
:10441000472B61F040EB58E060ED74E0DF91CF9105
:10442000FF90EF90DF90CF900C946B0FCD28CE28AB
:10443000CF2841F485EB96E09F938F930E94FF8BEA
:104440000F900F90DF91CF91FF90EF90DF90CF9082
:1044500008950F931F93CF93DF938C01C0E0D0E0BA
:104460000115110509F48AC060EB76E0C8010E94CD
:104470003A8B892B09F4C16068EA76E0C8010E9492
:104480003A8B892B09F4C26060EA76E0C8010E9489
:104490003A8B892B09F4C4606CE976E0C8010E946C
:1044A0003A8B892B09F4C86069E976E0C8010E945B
:1044B0003A8B892B09F4C06165E976E0C8010E9456
:1044C0003A8B892B09F4C0626FE876E0C8010E943C
:1044D0003A8B892B09F4C06467E876E0C8010E9432
:1044E0003A8B892B09F4C0686FE776E0C8010E9417
:1044F0003A8B892B09F4D1606BE776E0C8010E9402
:104500003A8B892B09F4D26065E776E0C8010E94F6
:104510003A8B892B09F4D46060E776E0C8010E94E9
:104520003A8B892B09F4D8606AE676E0C8010E94CC
:104530003A8B892B09F4D06162E676E0C8010E94CB
:104540003A8B892B09F4D06267E576E0C8010E94B6
:104550003A8B892B09F4D06466E476E0C8010E94A6
:104560003A8B892B09F4D0686091610270916202E4
:1045700080E090E00E944E8B8C0172CFCE01DF91E3
:10458000CF911F910F910895AF92BF92CF92DF927A
:10459000EF92FF920F931F93CF93DF93F22E032F8F
:1045A000142FE52E5B016C01217030E040E050E0FB
:1045B00060E070E080E090E0A0E00E94888789F0F1
:1045C000E1EEF4E0FF93EF93EBE6FDE0FF93EF9372
:1045D0000E94FF8B0F900F900F900F90E1E0F0E0A2
:1045E00002C0E0E0F0E08091A91F80FF17C02F2DEE
:1045F000247030E040E050E060E070E080E090E067
:10460000A0E00E94888751F0EF01219640EB58E02E
:1046100065EE74E0CF010E946B0FFE012F2D22701A
:1046200030E040E050E060E070E080E090E0A0E04A
:104630000E94888751F0EF01219640EB58E069EE27
:1046400074E0CF010E946B0FFE012F2D287030E027
:1046500040E050E060E070E080E090E0A0E00E9488
:10466000888751F0EF01219640EB58E061E075E05A
:10467000CF010E946B0FFE012F2D207130E040E032
:1046800050E060E070E080E090E0A0E00E94888769
:1046900051F0EF01219640EB58E06CEE74E0CF0151
:1046A0000E946B0FFE012F2D207230E040E050E0A1
:1046B00060E070E080E090E0A0E00E94888751F028
:1046C000EF01219640EB58E06FEE74E0CF010E94BD
:1046D0006B0FFE012F2D207430E040E050E060E0D1
:1046E00070E080E090E0A0E00E94888751F0EF0148
:1046F000219640EB58E065EF74E0CF010E946B0F0C
:10470000FE012F2D207830E040E050E060E070E0C6
:1047100080E090E0A0E00E94888751F0EF012196B0
:1047200040EB58E06BEF74E0CF010E946B0FFE018D
:1047300020E0302F317040E050E060E070E080E039
:1047400090E0A0E00E94888751F0EF01219640EBB5
:1047500058E06EEF74E0CF010E946B0FFE0120E085
:10476000302F327040E050E060E070E080E090E098
:10477000A0E00E94888751F0EF01219640EB58E0BD
:1047800063E075E0CF010E946B0FFE0120E0302F47
:10479000347040E050E060E070E080E090E0A0E045
:1047A0000E94888751F0EF01219640EB58E06AE0C3
:1047B00075E0CF010E946B0FFE0120E0302F3870B2
:1047C00040E050E060E070E080E090E0A0E00E9417
:1047D000888751F0EF01219640EB58E06DE075E0DD
:1047E000CF010E946B0FFE0120E0302F307140E0BE
:1047F00050E060E070E080E090E0A0E00E948887F8
:1048000051F0EF01219640EB58E062E175E0CF01F5
:104810000E946B0FFE0120E0302F307240E050E02C
:1048200060E070E080E090E0A0E00E94888751F0B6
:10483000EF01219640EB58E069E175E0CF010E945D
:104840006B0FFE018091A91F81FF17C020E0302F60
:10485000307440E050E060E070E080E090E0A0E084
:104860000E94888751F0EF01219640EB58E060E20A
:1048700075E0CF010E946B0FFE018091A91F9091FE
:10488000AA1F90FF17C020E030E040E05E2D50717D
:1048900060E070E080E090E0A0E00E94888751F046
:1048A000EF01219640EB58E063E275E0CF010E94F2
:1048B0006B0FFE018091A91F9091AA1F90FF17C056
:1048C00020E030E040E05E2D507260E070E080E07B
:1048D00090E0A0E00E94888751F0EF01219640EB24
:1048E00058E066E275E0CF010E946B0FFE018091F7
:1048F000A91F9091AA1F90FF17C020E030E040E070
:104900005E2D507460E070E080E090E0A0E00E94D6
:10491000888751F0EF01219640EB58E06CE275E09A
:10492000CF010E946B0FFE0120E0302F307840E075
:1049300050E060E070E080E090E0A0E00E948887B6
:1049400051F0EF01219640EB58E067E375E0CF01AD
:104950000E946B0FFE0120E030E0412F417050E0DB
:1049600060E070E080E090E0A0E00E94888751F075
:10497000EF01219640EB58E06CE375E0CF010E9417
:104980006B0FFE0120E030E0412F427050E060E00C
:1049900070E080E090E0A0E00E94888751F0EF0195
:1049A000219640EB58E06FE375E0CF010E946B0F5A
:1049B000FE0120E030E0412F447050E060E070E004
:1049C00080E090E0A0E00E94888751F0EF012196FE
:1049D00040EB58E062E475E0CF010E946B0FFE01EE
:1049E0008091A91F87FF17C020E030E0412F487059
:1049F00050E060E070E080E090E0A0E00E948887F6
:104A000051F0EF01219640EB58E065E475E0CF01ED
:104A10000E946B0FFE018091A91F87FF17C020E045
:104A200030E0412F407150E060E070E080E090E0C5
:104A3000A0E00E94888751F0EF01219640EB58E0FA
:104A400069E475E0CF010E946B0FFE018091A91F00
:104A500087FF17C020E030E0412F407250E060E057
:104A600070E080E090E0A0E00E94888751F0EF01C4
:104A7000219640EB58E06DE475E0CF010E946B0F8A
:104A8000FE018091A91F87FF17C020E030E0412F71
:104A9000407450E060E070E080E090E0A0E00E94B0
:104AA000888751F0EF01219640EB58E061E575E011
:104AB000CF010E946B0FFE018091A91F82FF17C0DA
:104AC00020E030E0412F407850E060E070E080E08E
:104AD00090E0A0E00E94888751F0EF01219640EB22
:104AE00058E060E176E0CF010E946B0FFE018091FB
:104AF000A91F82FF17C020E030E040E05E2D51701A
:104B000060E070E080E090E0A0E00E94888751F0D3
:104B1000EF01219640EB58E065E575E0CF010E947A
:104B20006B0FFE018091A91F9091AA1F90FF17C0E3
:104B300020E030E040E05E2D527060E070E080E008
:104B400090E0A0E00E94888751F0EF01219640EBB1
:104B500058E068E575E0CF010E946B0FFE0180917F
:104B6000A91F9091AA1F90FF17C020E030E040E0FD
:104B70005E2D547060E070E080E090E0A0E00E9464
:104B8000888751F0EF01219640EB58E060E675E030
:104B9000CF010E946B0FFE018091A91F9091AA1F67
:104BA00091FF1EC020E030E040E05E2D587060E0D4
:104BB00070E080E090E0A0E00E94888789F040EB00
:104BC00058E069E675E0CF01DF91CF911F910F9119
:104BD000FF90EF90DF90CF90BF90AF900C946B0F51
:104BE0002F2D302F412F5E2DB501C601A0E00E9470
:104BF000888741F481E496E09F938F930E94FF8B16
:104C00000F900F90DF91CF911F910F91FF90EF9038
:104C1000DF90CF90BF90AF900895AF92BF92DF9298
:104C2000EF920F931F93CF93DF93EC015B01FB0196
:104C300010826CE376E00E943A8B892B59F58091C3
:104C4000A91F7DE4D72EE0E8EE2E82FD02C004E02D
:104C500001C004E810E081FF02C060ECE62E26E00F
:104C60004AE250E06BE270E089E290E00E942D564B
:104C700081E090E00E94AA0A882311F05DE5D52E1C
:104C80008091A91F9091AA1F90FD16E091FF06C088
:104C9000186004C0D12CE12C00E010E06AE376E05B
:104CA000CE010E943A8B892B61F481E0F50180836B
:104CB000609161027091620280E090E00E944E8BF0
:104CC000EC0168E376E0CE010E943A8B892B61F417
:104CD0008FEFF5018083609161027091620280E044
:104CE00090E00E944E8BEC01209709F41AC164E316
:104CF00076E0CE010E943A8B892B19F4FD2DF160EC
:104D0000DF2E60E376E0CE010E943A8B892B19F406
:104D10008D2D8460D82E6DE276E0CE010E943A8B14
:104D2000892B19F4ED2DE260DE2E6BE276E0CE01E8
:104D30000E943A8B892B19F4FD2DF860DF2E68E272
:104D400076E0CE010E943A8B892B19F48D2D80617B
:104D5000D82E62E276E0CE010E943A8B892B19F4BC
:104D6000ED2DE062DE2E6CE176E0CE010E943A8B02
:104D7000892B19F4FD2DF064DF2E69E176E0CE0178
:104D80000E943A8B892B19F48D2D8068D82E64E10E
:104D900076E0CE010E943A8B892B19F4EE2DE1606A
:104DA000EE2E6DE076E0CE010E943A8B892B19F44D
:104DB000FE2DF260EF2E6AE076E0CE010E943A8B83
:104DC000892B19F48E2D8460E82E65E076E0CE0103
:104DD0000E943A8B892B19F4EE2DE860EE2E6EEFCF
:104DE00075E0CE010E943A8B892B19F4FE2DF061FB
:104DF000EF2E67EF75E0CE010E943A8B892B19F4F4
:104E00008E2D8062E82E64EF75E0CE010E943A8B11
:104E1000892B19F4EE2DE064EE2E6FEE75E0CE01D5
:104E20000E943A8B892B19F4FE2DF068EF2E6CEE60
:104E300075E0CE010E943A8B892B09F4016069EE7E
:104E400075E0CE010E943A8B892B09F4026066EE70
:104E500075E0CE010E943A8B892B09F4046062EE62
:104E600075E0CE010E943A8B892B09F408606EED43
:104E700075E0CE010E943A8B892B09F400616AED3E
:104E800075E0CE010E943A8B892B09F4006266ED31
:104E900075E0CE010E943A8B892B09F4006464ED21
:104EA00075E0CE010E943A8B892B09F4006861ED10
:104EB00075E0CE010E943A8B892B09F4116069ECF0
:104EC00075E0CE010E943A8B892B09F4126060ECE8
:104ED00075E0CE010E943A8B892B09F4146067EBD0
:104EE00075E0CE010E943A8B892B09F4186064EBBF
:104EF00075E0CE010E943A8B892B09F410616EEAAD
:104F000075E0CE010E943A8B892B09F4106263EAA6
:104F100075E0CE010E943A8B892B09F0DCCE10643B
:104F2000DACE2D2D3E2DA80160E070E080E090E00B
:104F3000DF91CF911F910F91EF90DF90BF90AF90D5
:104F400008955F926F927F928F929F92AF92BF92DD
:104F5000CF92DF92EF92FF920F931F93CF93DF9345
:104F6000782EC3EBDAE100E010E0FDE9EF2EF5E08A
:104F7000FF2E8170582E872D8270682EA8E8CA2EC9
:104F8000A5E0DA2EB0E9AB2EB5E0BB2E8EE8882E78
:104F900085E0982E772051F01F930F93FF92EF92A8
:104FA0000E94FF8B0F900F900F900F905520A1F053
:104FB00089858F9388858F93BF92AF920E94FF8BD4
:104FC0000F900F900F900F906620C1F09F928F92DC
:104FD0000E94FF8B0F900F90662081F0DF92CF929E
:104FE0000E94FF8B288139814A815B816C817D81A0
:104FF0008E819F810E94C4220F900F900E941C0BF3
:105000000F5F1F4F2A960430110521F6DF91CF91D3
:105010001F910F91FF90EF90DF90CF90BF90AF90D6
:105020009F908F907F906F905F900895CF9388E7C7
:1050300095E09F938F930E94FF8B0E942D1F8AE91A
:105040009AE19F938F9380E795E09F938F930E94BF
:10505000FF8B8CE695E09F938F930E94FF8B80E0FF
:105060000E940B2187E695E09F938F930E94FF8B10
:105070000E94930F8091A91F2DB73EB7265F3F4F27
:105080000FB6F8943EBF0FBE2DBF80FF05C041E0B4
:1050900061E081E00E943D110E94311F8091490230
:1050A0001F928F938EE595E09F938F930E94FF8BC5
:1050B00080914D091F928F9385E595E09F938F9383
:1050C0000E94FF8BC0E4CF9383E18F9383E38F93A0
:1050D0008F9381E495E09F938F930E94FF8B1F92A3
:1050E000CF9389E295E09F938F930E94FF8B8091ED
:1050F00036281F928F93809135281F928F9386E1D7
:1051000095E09F938F930E94FF8B809148021F929E
:105110008F938DE095E09F938F930E94FF8B8091FA
:105120004A0290914B022DB73EB7245E3F4F0FB617
:10513000F8943EBF0FBE2DBF96FF03C082E795E0F7
:1051400002C085E795E09F938F9383E095E09F935E
:105150008F930E94FF8B83E00E94A1270F900F90F6
:105160000F900F901D9B03C082E795E002C085E77A
:1051700095E09F938F9387EF94E09F938F930E9486
:10518000FF8B8DEE94E09F938F930E94FF8B809115
:105190004A020F900F900F900F900F900F9081FF89
:1051A00009C087EE94E09F938F930E94FF8B0F902E
:1051B0000F9013C080FF03C082E795E002C085E72F
:1051C00095E09F938F9383EE94E09F938F930E943B
:1051D000FF8B0F900F900F900F908CED94E09F93AA
:1051E0008F930E94FF8B609151097091520980E06A
:1051F00090E00E943B210E941C0B0F900F9077992A
:1052000003C082E795E002C085E795E09F938F9306
:1052100083ED94E09F938F930E94FF8B0E94C308BD
:105220000E94660A9F938F937F936F9385EC94E01F
:105230009F938F930E94FF8B0E94200A9F938F93CE
:105240007F936F9387EB94E09F938F930E94FF8BE4
:1052500081E090E00E94E71F809110289091112832
:10526000A0911228B0911328BF93AF939F938F936F
:1052700089EA94E09F938F930E94FF8B809120286E
:105280008F9380911F288F9380911E288F938091F8
:105290001D288F9385E994E09F938F930E94FF8B45
:1052A0008091142890911528A0911628B091172864
:1052B000BF93AF939F938F9387E894E09F938F93CF
:1052C0000E94FF8B8DB79EB782960FB6F8949EBF53
:1052D0000FBE8DBF809124288F93809123288F93B8
:1052E000809122288F93809121288F9383E794E0E7
:1052F0009F938F930E94FF8B61E070E080E090E0CD
:105300000E94250B0F900F900F900F900F900F9011
:1053100061E070E081E090E0CF910C94250BF8946F
:10532000E0E0F0E081E2809357008491E2E0F0E079
:1053300041E2409357004491E4E0F0E091E2909321
:105340005700E49190E0A0E0B0E0DC0199278827C5
:1053500050E060E070E0762F652F542F4427840FD3
:10536000951FA61FB71F8E0F911DA11DB11D809304
:10537000541B9093551BA093561BB093571B7894C6
:105380000895CF93DF93CDB7DEB761970FB6F8944A
:10539000DEBF0FBECDBF48E250E068E170E083EBB6
:1053A0009AE10E94248D2091B31A3091B41A409151
:1053B000B51A5091B61A6091B71A7091B81A8091C7
:1053C000B91A9091BA1AAFEF0E94888709F05DC0B0
:1053D0008DE48093B31A80E88093B41A84E08093BC
:1053E000B51A1092B61A1092B71A1092B81A1092F3
:1053F000B91A1092BA1A8CE390E09093BC1A809379
:10540000BB1A1092BD1A1092BE1A1092BF1A1092B7
:10541000C01A1092C11A1092C21A1092C31A109296
:10542000C41A1092C61A1092C51A1092C71A109276
:10543000C81A1092C91A1092CA1A1092CB1A109256
:10544000CC1A1092CD1A1092CE1A1092D01A109235
:10545000CF1A1092D11A1092D21A1092D31A109217
:10546000D41A1092D51A1092D61A1092D71A1092F6
:10547000D81A1092DA1A1092D91A48E250E068E16C
:1054800070E083EB9AE10E94428D42E050E066E1D9
:1054900070E0CE010F960E94248D8F8598898F3FF2
:1054A0002FEF920779F48AE090E490934B02809377
:1054B0004A0242E050E066E170E08AE492E00E9435
:1054C000428D04C090934B0280934A0242E050E028
:1054D0006CE470E0CE010F960E94248D8F85988930
:1054E0008F3F2FEF920769F41092520910925109E1
:1054F00042E050E06CE470E081E599E00E94428D6A
:1055000004C0909352098093510949E050E06AE049
:1055100070E085E298E20E94248D0E945D0C44E0D8
:1055200050E064E470E0CE010B960E94248D8B85E0
:105530009C85AD85BE8544E050E064E470E08F3F1B
:105540009F4FAF4FBF4F29F488E692E00E94428DF3
:1055500004C088E692E00E94248D44E050E060E4BC
:1055600070E0CE010B960E94248D8B859C85AD85C5
:10557000BE8544E050E060E470E08F3F9F4FAF4F46
:10558000BF4F29F484E692E00E94428D04C084E675
:1055900092E00E94248D44E050E068E470E0CE0187
:1055A0000B960E94248D8B859C85AD85BE8544E03D
:1055B00050E068E470E08F3F9F4FAF4FBF4F29F43A
:1055C0008CE692E00E94428D04C08CE692E00E943C
:1055D000248D41E050E065E170E0CE0141960E94EB
:1055E000248D898941E050E065E170E08F3F29F426
:1055F0008DE499E00E94428D04C08DE499E00E9400
:10560000248D41E050E064E170E0CE0141960E94BB
:10561000248D898941E050E064E170E08F3F29F4F6
:1056200089E492E00E94428D04C089E492E00E94E5
:10563000248D41E050E063E170E0CE0141960E948C
:10564000248D898941E050E063E170E08F3F29F4C7
:1056500088E492E00E94428D04C088E492E00E94B7
:10566000248D4AE050E060E070E0CE0101960E9497
:10567000248D89814AE050E060E070E08F3F29F49A
:105680008AE99AE10E94428D04C08AE99AE10E9467
:10569000248D61960FB6F894DEBF0FBECDBFDF91AB
:1056A000CF910895CF92DF92EF92FF9260916102C5
:1056B0007091620280E090E00E944E8B69E775E095
:1056C0000E94628B892B09F0F1C08DE48093B31A9C
:1056D00080E88093B41A84E08093B51A1092B61AC9
:1056E0001092B71A1092B81A1092B91A1092BA1AE8
:1056F0008CE390E09093BC1A8093BB1A1092BD1A71
:105700001092BE1A1092BF1A1092C01A1092C11AAB
:105710001092C21A1092C31A1092C41A1092C61A8A
:105720001092C51A1092C71A1092C81A1092C91A6C
:105730001092CA1A1092CB1A1092CC1A1092CD1A4B
:105740001092CE1A1092D01A1092CF1A1092D11A2B
:105750001092D21A1092D31A1092D41A1092D51A0B
:105760001092D61A1092D71A1092D81A1092DA1AEA
:105770001092D91A48E250E068E170E083EB9AE1B8
:105780000E94428D8AE090E490934B0280934A02FB
:1057900042E050E066E170E08AE492E00E94428DCF
:1057A000109252091092510942E050E06CE470E00E
:1057B00081E599E00E94428D42E2C42EDD24DA9414
:1057C0004CECE42E4BE3F42EC0926802D0926902B6
:1057D000E0926A02F0926B0244E050E064E470E010
:1057E00088E692E00E94428DC0926402D0926502E7
:1057F000E0926602F092670244E050E060E470E0FC
:1058000084E692E00E94428D87ED94E3AFEEBCE324
:1058100080936C0290936D02A0936E02B0936F021E
:1058200044E050E068E470E08CE692E00E94428D33
:1058300010924D0980E00E94996341E050E065E1DB
:1058400070E08DE499E00E94428D8AE180934902E4
:105850000E94406241E050E064E170E089E492E03F
:105860000E94428D8FE08093480241E050E063E166
:1058700070E088E492E00E94428D8AE0EAE9FAE171
:10588000DF011D928A95E9F74AE050E060E070E0A0
:10589000CF010E94428D81E00E940B2180E090E0C8
:1058A000FF90EF90DF90CF900C94710CFF90EF90F1
:1058B000DF90CF9008952F923F924F925F926F9218
:1058C0007F928F929F92AF92BF92CF92DF92EF9290
:1058D000FF920F931F93CF93DF93CDB7DEB72B9734
:1058E0000FB6F894DEBF0FBECDBF9B878A87FC0141
:1058F00080819181892B11F00C94643C609161024C
:105900007091620280ED93E20E944E8B60E470E041
:1059100080ED93E20E94818B009759F46091F03002
:105920007091F1308AE090E00E94BB8B81E00C9492
:10593000693C8130910549F42090D023312C412CD1
:10594000512C612C712C4301BDC082309105A1F412
:105950008091D0232091D12390E0982F8827820F27
:10596000911D1C01892F880F880B482E582E682EF8
:10597000782E882E982EA6C083309105D1F52091DF
:10598000D0231091D123E091D22330E040E050E0C9
:1059900060E070E080E090E000E10E942A87522EF3
:1059A000632E742E852E962EB72FA82FF92F212F18
:1059B00030E040E050E060E070E080E090E008E03F
:1059C0000E942A8759016A017B018C01252D362D01
:1059D000472D582D692D7B2F8A2F9F2F0E9461877D
:1059E000AE2EB12CC12CD12CE12CF12C00E010E01A
:1059F00059C004970CF45DC02091D0231091D1239D
:105A0000E091D223F091D32330E040E050E060E019
:105A100070E080E090E008E10E942A8729013A01C5
:105A20004B01B82FA92F212F30E040E050E060E07B
:105A300070E080E090E000E10E942A8759016A014D
:105A40007B018C019201A301B4018B2F9A2F0E943C
:105A50006187AF2EB12CC12CD12CE12CF12C00E0B0
:105A600010E00E946187522E632E742E852E962E92
:105A7000B72FA82FF92F2E2F30E040E050E060E044
:105A800070E080E090E008E00E942A8759016A01F6
:105A90007B018C01252D362D472D582D692D7B2F0F
:105AA0008A2F9F2F0E94618719012A013B014C0117
:105AB00009C07AE0272E312C412C512C612C712CFD
:105AC000812C912C0E941C0B9101A201B301C401F5
:105AD0002736FFE63F07FCE64F07510561057105D4
:105AE0008105910511F40C94B9362736EFE63E078F
:105AF000ECE64E075105610571058105910511F030
:105B000008F075C12936F2E73F07410551056105E7
:105B100071058105910511F40C94A2392936E2E74B
:105B20003E0741055105610571058105910511F09B
:105B300008F097C02536F4E63F0741055105610599
:105B400071058105910509F41FC52536E4E63E0778
:105B500041055105610571058105910509F088F53B
:105B6000A6E70E94888709F4C6C60E94888709F0C4
:105B700060F4A8E60E94888709F44CC5A5E70E9456
:105B8000888709F4A2C60C94623C9101A201B3017A
:105B9000C4012A33F6E23F0741055105610571054D
:105BA0008105910509F4C9C22436314641055105E4
:105BB000610571058105910511F40C941B3A0C9453
:105BC000623C9101A201B301C4012737FFE63F0700
:105BD00041055105610571058105910511F40C948C
:105BE000D6372737EFE63E074105510561057105B8
:105BF0008105910509F0C0F42436F9E63F07410517
:105C00005105610571058105910509F437C62536F1
:105C10003E4641055105610571058105910511F467
:105C20000C940A380C94623C9101A201B301C401A6
:105C30002333F1E73F0741055105610571058105F2
:105C4000910511F40C941B3A253632474105510554
:105C5000610571058105910511F40C94C4380C940B
:105C6000623C9101A201B301C4012236F5E63F076F
:105C7000F4E64F075105610571058105910509F4A9
:105C800083C42236E5E63E07E4E64E07510561058A
:105C900071058105910511F008F051C02133F4E63A
:105CA0003F07F1E64F075105610571058105910533
:105CB00009F453C22133E4E63E07E1E64E075105FD
:105CC000610571058105910509F0C8F42337F2E7F4
:105CD0003F0741055105610571058105910511F4E5
:105CE0000C94F3392337334741055105610571059C
:105CF0008105910511F40C94073A0C94623C9101D2
:105D0000A201B301C4012336F4E63F07F1E64F07D1
:105D10005105610571058105910511F40C941B3A3B
:105D200028373446414651056105710581059105C5
:105D300011F00C94623C0E9421150C94643C91017A
:105D4000A201B301C4012D36F5E73F07F8E64F077E
:105D50005105610571058105910511F40C94313AE5
:105D60002D36E5E73E07E8E64E075105610571056A
:105D70008105910509F0E0F42237F2E73F07F5E6E7
:105D80004F075105610571058105910511F40C94CA
:105D90003B3723363D46484651056105710581056F
:105DA000910511F00C94623C0E9499150C94643C8E
:105DB0009101A201B301C4012336F2E33F07F9E6E2
:105DC0004F075105610571058105910509F4E5C18C
:105DD000243633464C465105610571058105910510
:105DE00011F00C94623C0E948E5A0C94643C910118
:105DF000A201B301C4012037FCE63F07F5E64F07D7
:105E0000F8E65F07610571058105910509F402C493
:105E10002037ECE63E07E5E64E07E8E65E0761055B
:105E200071058105910511F008F0C0C02437F8E72D
:105E30003F07F4E74F07510561057105810591059D
:105E400009F4C0C52437E8E73E07E4E74E075105EB
:105E5000610571058105910511F008F050C02133ED
:105E6000F1E33F07F1E74F07510561057105810532
:105E7000910511F40C9470372133E1E33E07E1E71B
:105E80004E075105610571058105910509F0C8F4BA
:105E90002537F3E63F07FDE64F075105610571051C
:105EA0008105910511F40C9470372033314341473B
:105EB0005105610571058105910509F4DCC70C9454
:105EC000623C9101A201B301C4012037F5E63F070E
:105ED000F2E74F075105610571058105910511F440
:105EE0000C94C4382C36344744475105610571057C
:105EF0008105910511F40C949F3B0C94623C910137
:105F0000A201B301C4012936FCE63F07F1E64F07C1
:105F1000F3E65F07610571058105910509F472C11A
:105F20002936ECE63E07E1E64E07E3E65E0761054B
:105F300071058105910509F0E0F42437F4E63F0787
:105F4000F7E74F075105610571058105910511F4CA
:105F50000C94ED3B24373F464F4652466105710590
:105F60008105910511F00C94623C0C9400000C9496
:105F7000643C9101A201B301C4012E36F1E63F0752
:105F8000F8E64F07F3E65F076105710581059105A6
:105F900009F4EEC426333946454755466105710577
:105FA0008105910509F43AC30C94623C9101A20168
:105FB000B301C4012437F3E73F07F5E64F07F2E7E3
:105FC0005F07610571058105910511F40C94843812
:105FD0002437E3E73E07E5E64E07E2E75E076105A3
:105FE00071058105910511F008F052C02337F5E6DF
:105FF0003F07F2E74F07F0E75F076105710581058D
:10600000910511F40C94E13A2337E5E63E07E2E707
:106010004E07E0E75E07610571058105910509F00E
:10602000C8F42136FDE63F07F5E74F07F8E65F07BE
:10603000610571058105910509F4D6C722373747F7
:1060400040475047610571058105910509F4A9C0D4
:106050000C94623C9101A201B301C4012337F2E721
:106060003F07F7E74F07F0E75F0761057105810517
:10607000910511F40C94873821363C464546524729
:10608000610571058105910509F4E5C20C94623C36
:106090009101A201B301C4012437F2E73F07F1E601
:1060A0004F07F5E75F07610571058105910509F463
:1060B0005BC32437E2E73E07E1E64E07E5E75E070C
:1060C000610571058105910509F0C8F42437F3E7EE
:1060D0003F07F5E64F07F4E75F07610571058105A6
:1060E000910509F498C4273730474847544761055C
:1060F00071058105910509F413C40C94623C91016A
:10610000A201B301C4012237F7E63F07F0E74F07CA
:10611000F5E75F07610571058105910509F406C67C
:106120002C36314644475847610571058105910574
:1061300011F40C94693B0C94623C84E08093BC2382
:106140001092BE231092BD234CEB53E262E18AE22F
:1061500092E00E94B24D0C94643C21E042E161E087
:1061600080ED0E94DD5A21E042E161E080ED0E9475
:10617000DD5A21E042E161E080ED0E94DD5A21E03C
:1061800042E161E080ED0E94DD5A21E042E161E000
:1061900080ED0E94DD5A0C94643C0E94930F0C9495
:1061A000643C609161027091620280E090E00E9424
:1061B0004E8B8C0162E775E00E94628B892B19F48B
:1061C00077980C94643C65E775E0C8010E94628B87
:1061D000892B19F4779A0C94643C779903C082E771
:1061E00095E002C085E795E09F938F938DE594E05D
:1061F0009F938F930E94FF8B0F900F900F900F90A3
:106200000C94643C609161027091620280E090E0C5
:106210000E944E8B8C016CE375E00E94628B892B8F
:1062200009F077C0609161027091620280E090E0B5
:106230000E944E8B8C01009711F40C94643C60E832
:1062400075E00E94628B892BB1F482E29FEFACEC87
:10625000BBE38093680290936902A0936A02B093B3
:106260006B0244E050E064E470E088E692E00E9453
:10627000428D0C94643C66E875E0C8010E94628B14
:10628000892BB1F482E29FEFACECBAE38093680211
:1062900090936902A0936A02B0936B0244E050E0CD
:1062A00064E470E088E692E00E94428D0C94643CC5
:1062B000C8010E94388A2B013C0120E030E0A9018E
:1062C0000E94D7818823D9F081E00E94BD099B01FB
:1062D000AC01C301B2010E94DB816093680270933C
:1062E000690280936A0290936B0244E050E064E498
:1062F00070E088E692E00E94428D0C94643C84ED4C
:1063000092E09F938F930E94FF8B0F900F900C94BD
:10631000643C6FE375E0C8010E94628B892B09F031
:1063200077C0609161027091620280E090E00E940B
:106330004E8B8C01009711F40C94643C60E875E07E
:106340000E94628B892BB1F482E29FEFACECBBE33D
:106350008093640290936502A0936602B0936702F3
:1063600044E050E060E470E084E692E00E94428DF8
:106370000C94643C66E875E0C8010E94628B892B2E
:10638000B1F482E29FEFACECBAE3809364029093A5
:106390006502A0936602B093670244E050E060E4B7
:1063A00070E084E692E00E94428D0C94643CC80147
:1063B0000E94388A2B013C0120E030E0A9010E94B4
:1063C000D7818823D9F082E00E94BD099B01AC01EE
:1063D000C301B2010E94DB81609364027093650285
:1063E000809366029093670244E050E060E470E0BE
:1063F00084E692E00E94428D0C94643C87EC92E02B
:106400009F938F930E94FF8B0F900F900C94643C8E
:1064100067E375E0C8010E94628B892B09F073C0A5
:10642000609161027091620280E090E00E944E8B68
:106430008C01009711F40C94643C60E875E00E94B4
:10644000628B892BB1F487ED94E3AFEEBCE38093CC
:106450006C0290936D02A0936E02B0936F0244E0C1
:1064600050E068E470E08CE692E00E94428D0C946B
:10647000643C66E875E0C8010E94628B892B51F488
:1064800088EB92E09F938F930E94FF8B0F900F9069
:106490000C94643CC8010E94388A2B013C0120E026
:1064A00030E0A9010E94D781882319F180E00E9481
:1064B000BD094B015C0121EE3AE744E95EE3C3010B
:1064C000B2010E941081A50194010E94DB816093BA
:1064D0006C0270936D0280936E0290936F0244E0A1
:1064E00050E068E470E08CE692E00E94428D0C94EB
:1064F000643C8BEA92E09F938F930E94FF8B0F90F6
:106500000F900C94643C0E940C0A9F938F937F938E
:106510006F9384EA92E09F938F930E94FF8B82E0B7
:106520000E94BD092091640230916502409166028B
:10653000509167020E945884162F072FF82EE92EDB
:1065400081E00E94BD09EF92FF920F931F9320916B
:1065500068023091690240916A0250916B020E9478
:1065600058849F938F937F936F9388E992E09F93D2
:106570008F930E94FF8B0E941C0B0FB6F894DEBF16
:106580000FBECDBF0C94643C6091610270916202B9
:1065900080E090E00E944E8B0097C1F00E9429227B
:1065A00020915109309152098217930709F1909374
:1065B00052098093510942E050E06CE470E081E5BB
:1065C00099E00E94428D86E594E002C08FE494E059
:1065D0009F938F930E94FF8B609151097091520994
:1065E00080E090E00E943B210E941C0B0F900F90D6
:1065F00084E494E09F938F930E94FF8B6FEF7FEF73
:1066000080E090E00E943B210E941C0B0F900F90B5
:106610000C94643C0E944E1E0C94643C8091D423E4
:10662000843329F440E061E080E00E943D118091D4
:106630006302882311F40C94643C1F928F9381E4CD
:1066400094E09F938F930E94FF8B0F900F900F9079
:106650000F900C94643C8091D423893709F070C06A
:10666000609161027091620280E090E00E944E8B26
:106670008C0162E775E00E94628B892B31F4809176
:106680004A0290914B0290640CC065E775E0C80126
:106690000E94628B892B91F480914A0290914B0267
:1066A0009F7B90934B0280934A0242E050E066E168
:1066B00070E08AE492E00E94428D42C06BE875E08F
:1066C000C8010E94628B892B21F58091B21A8F93A9
:1066D0008091B11A8F938091B01A8F938091AF1AE5
:1066E0008F938091AE1A8F938091AD1A8F93809182
:1066F000AC1A8F938091AB1A8F938DE692E09F93A3
:106700008F930E94FF8B0FB6F894DEBF0FBECDBFF4
:1067100017C080914A0290914B0296FF03C082E716
:1067200095E002C085E795E09F938F9389E692E01C
:106730009F938F930E94FF8B0F900F900F900F905D
:1067400080916302882311F40C94643C1F928F9310
:106750008EE394E09F938F930E94FF8B0F900F9096
:106760000F900F900C94643C6091610270916202F2
:1067700080E090E00E944E8B5C0161E975E00E9430
:10678000628B892B11F489E108C065E975E0C501C8
:106790000E94628B892B49F480E18093C40010929F
:1067A000C50082E08093C00055C069E975E0C5016D
:1067B0000E94628B892B11F488E0EFCF6EE975E0BF
:1067C000C5010E94628B892B39F063EA75E0C5012F
:1067D0000E94628B892B11F483E0DFCF8091C4008B
:1067E000893141F484E692E09F938F930E94FF8B5E
:1067F0000F900F908091C400803141F48FE592E0BA
:106800009F938F930E94FF8B0F900F908091C400F5
:10681000883041F489E592E09F938F930E94FF8B2B
:106820000F900F908091C400833041F483E592E093
:106830009F938F930E94FF8B0F900F908091C400C5
:10684000883041F48DE492E09F938F930E94FF8BF8
:106850000F900F9080916302882311F40C94643C94
:106860001F928F938BE394E09F938F930E94FF8BF3
:106870000F900F900F900F900C94643C6091610208
:106880007091620280E090E00E944E8B60E875E0BB
:106890000E94628B892B11F481E001C080E00E948C
:1068A0000B2180916302882311F40C94643C1F92A5
:1068B0008F9388E394E09F938F930E94FF8B0F90B8
:1068C0000F900F900F900C94643C0E94311F8091A8
:1068D0006302882311F40C94643C1F928F9385E328
:1068E00094E09F938F930E94FF8B0F900F900F90D7
:1068F0000F900C94643C0E942D1F809163028823AA
:1069000011F40C94643C1F928F9382E394E09F9364
:106910008F930E94FF8B0F900F900F900F90D4C712
:10692000609161027091620280E090E00E944E8B63
:106930000E943C8A803168F480934D090E949963DB
:1069400041E050E065E170E08DE499E00E94428D05
:10695000BBC780914D091F928F9383E492E09F9370
:106960008F930E94FF8B0F900F900F900F90ACC7EA
:10697000609161027091620280E090E00E944E8B13
:106980000E943C8A95EF980F903168F480934902F9
:106990000E94406241E050E064E170E089E492E0EE
:1069A0000E94428D91C7809149021F928F938AE382
:1069B00092E09F938F930E94FF8B0F900F900F9008
:1069C0000F9082C7609161027091620280E090E056
:1069D0000E944E8B009781F04AE050E0BC018AE9AA
:1069E0009AE10E94728B4AE050E060E070E08AE930
:1069F0009AE10E94428D68C78AE99AE19F938F933A
:106A000088EA95E09F938F930E94ED8B0F900F90F3
:106A10000F900F9059C7609161027091620280E0FF
:106A200090E00E944E8B5C0168EC73E00E94628BE8
:106A3000892B99F4219A80914A0290914B028061AE
:106A400090934B0280934A0242E050E066E170E08E
:106A50008AE492E00E94428D37C760E475E0C50188
:106A60000E94628B892B99F4229A80914A0290911C
:106A70004B02806290934B0280934A0242E050E0C6
:106A800066E170E08AE492E00E94428D1DC76AEAE6
:106A900073E0C5010E94628B892B99F4239A80913F
:106AA0004A0290914B02806490934B0280934A0279
:106AB00042E050E066E170E08AE492E00E94428D9C
:106AC00003C767EE74E0C5010E94628B892B99F4BD
:106AD000239A80914A0290914B02806890934B02D6
:106AE00080934A0242E050E066E170E08AE492E07E
:106AF0000E94428DE9C669EF78E0C5010E94628B71
:106B0000892B31F581E08093BC2383EB9AE190934C
:106B1000BE238093BD231092C0231092BF23809187
:106B20004A0290914B02916090934B0280934A02EB
:106B300042E050E066E170E08AE492E00E94428D1B
:106B40004CEB53E262E18AE292E00E94B24DBCC695
:106B500061ED73E0C5010E94628B892BD1F4E3EEF5
:106B6000FAE1119211929BE1E330F907D1F780919C
:106B70004A0290914B02926090934B0280934A029A
:106B800042E050E066E170E08AE492E00E94428DCB
:106B90009BC665E775E0C5010E94628B20914A02A1
:106BA00030914B02892BA1F42F703C7F30934B0224
:106BB00020934A022B9A42E050E066E170E08AE4BA
:106BC00092E00E94428D80911C280E9455627CC6F2
:106BD00024FF03C082E795E002C085E795E09F931C
:106BE0008F938FE292E09F938F930E94FF8B80910F
:106BF0004A020F900F900F900F9085FF03C082E71D
:106C000095E002C085E795E09F938F9384E292E040
:106C10009F938F930E94FF8B80914A020F900F9059
:106C20000F900F9086FF03C082E795E002C085E7D2
:106C300095E09F938F9389E192E09F938F930E94B9
:106C4000FF8B80914A020F900F900F900F9087FF5B
:106C500003C082E795E002C085E795E09F938F939C
:106C60008EE092E09F938F930E94FF8B80914A0267
:106C700090914B020F900F900F900F9090FF03C0D8
:106C800082E795E002C085E795E09F938F9383E0CC
:106C900092E09F938F930E94FF8B80914A02909184
:106CA0004B020F900F900F900F9091FF03C082E75F
:106CB00095E002C085E795E09F938F9388EF91E080
:106CC0009F938F930E94FF8B80914A0290914B0279
:106CD0000F900F900F900F9091FFF6C580EB95E00D
:106CE0000E94238C53EEA52E5AE1B52E0BE010E046
:106CF00068EB862E65E0962EF50180819181F2E0A9
:106D0000AF0EB11C9F938F931F930F939F928F92FF
:106D10000E94ED8B0F5F1F4F0F900F900F900F9001
:106D20000F900F900B31110539F7CEC58EE294E02C
:106D30009F938F930E94FF8B809163020F900F901F
:106D4000882361F01F928F938BE294E09F938F933F
:106D50000E94FF8B0F900F900F900F9088E10FB65D
:106D6000F89480936000109260000FBE0C94007C39
:106D7000ABC5609161027091620280E090E00E9478
:106D80004E8B8C0162E775E00E94628B892BA9F41F
:106D90000E943F6180914A0290914B028D7F8160F9
:106DA00090934B0280934A0242E050E066E170E02B
:106DB0008AE492E00E94428D87C565E775E0C801CC
:106DC0000E94628B892BA1F40E94F76080914A0295
:106DD00090914B028C7F90934B0280934A0242E049
:106DE00050E066E170E08AE492E00E94428D6CC55A
:106DF00063EC75E0C8010E94628B892BA9F40E94A4
:106E0000F76080914A0290914B028E7F826090934E
:106E10004B0280934A0242E050E066E170E08AE46F
:106E200092E00E94428D50C580914A0281FF0FC0BE
:106E300083EC95E09F938F9384EF91E09F938F93E2
:106E40000E94FF8B0F900F900F900F903DC580FF19
:106E500003C082E795E002C085E795E09F938F939A
:106E600080EF91E09F938F930E94FF8B0F900F9084
:106E70000F900F9029C58091B6238F938091B523F1
:106E80008F938091B4238F938091B3238F938091BC
:106E9000BA238F938091B9238F938091B8238F93D6
:106EA0008091B7238F938DE094E09F938F930E94FE
:106EB000FF8B809163020FB6F894DEBF0FBECDBF8B
:106EC000882309F401C51F928F938AE094E09F9371
:106ED0008F930E94FF8B0F900F900F900F90F4C430
:106EE000F89481E090E029E0FC0120935700C895D8
:106EF000E02C80E090E0FC0120935700C895F02C36
:106F00007894F89483E090E0FC0120935700C895B2
:106F1000002D82E090E0FC0120935700C895102DD1
:106F200078948091571B8F938091561B8F938091FB
:106F3000551B8F938091541B8F9320E034E03F9337
:106F40002F930E94FF8B1F92EF921F92FF921F922E
:106F50000F931F921F9389ED93E09F938F930E944D
:106F6000FF8B0E94CB1F809166001F928F938DEC48
:106F700093E09F938F930E94FF8B0E941C0B809144
:106F800063020FB6F894DEBF0FBECDBF882309F4AD
:106F90009BC41F928F938AEC93E09F938F930E94E0
:106FA000FF8B0F900F900F900F908EC460E070E0F9
:106FB00080E090E00E94250B60E070E081E090E0CE
:106FC0000E94250B80916302882309F47DC41F92DF
:106FD0008F9387EC93E09F938F930E94FF8B0F908A
:106FE0000F900F900F9070C40E94111E0E941C0BF6
:106FF00080916302882309F467C41F928F9384EC05
:1070000093E09F938F930E94FF8B0F900F900F90B0
:107010000F905AC4609161027091620280E090E02A
:107020000E944E8B68EC75E00E94628B892B31F5D3
:10703000F89488E899E00E949F4E5C01009769F0FF
:10704000C5010F960E94A351B50184E092E00E9411
:10705000594EC5010E94474FF0CF88E899E00E9441
:107060002C4F892B29F088E899E00E94D84EF5CF63
:1070700088E899E00E949B4E789434C088E899E0B3
:107080000E949F4E5C010EEC15E0A114B10451F179
:10709000F50186811F928F9380851F928F93858142
:1070A0001F928F9381851F928F9387811F928F9359
:1070B00084811F928F9383811F928F9382811F926D
:1070C0008F9382851F928F931F930F930E94ED8B56
:1070D000C5010E94474F5C010FB6F894DEBF0FBE9A
:1070E000CDBFD3CF80916302882309F4EDC31F92F3
:1070F0008F9381EC93E09F938F930E94FF8B0F906F
:107100000F900F900F90E0C30E94522BDDC360914F
:1071100061027091620280E090E00E944E8B8C01CF
:107120006DE076E00E94628B892B91F480914A0297
:1071300090914B02977F90934B0280934A0242E0DA
:1071400050E066E170E08AE492E00E94428DBCC3A8
:1071500066E875E0C8010E94628B892B91F48091EA
:107160004A0290914B02986090934B0280934A029E
:1071700042E050E066E170E08AE492E00E94428DD5
:10718000A3C30E94C308A0C3609161027091620210
:1071900080E090E00E944E8BFC0120812332B1F40C
:1071A0004AE050E060E070E001960E94F0871B0129
:1071B000609161027091620280E090E00E944E8BCB
:1071C000F4E02F1631040CF094C002C0212C312CB5
:1071D000009709F48EC01982BE016F5F7F4F0E9435
:1071E0000D2629013A014B01B82FA92F8AE0829D73
:1071F000F001839DF00D1124ED54F54E20812A837A
:1072000031813B8382818C8393819D8324812E8372
:1072100035813F8386818887978199879201A30171
:10722000B4018B2F9A2FAA80BB80CC80DD80EE80AA
:10723000FF80088519850E947F8709F45DC08981D8
:10724000882351F18CF02A81422A3B81532A8C8178
:10725000682A9D81792A2E81822A3F81932A8885F6
:10726000B82B9985A92B18C04094509460947094C1
:1072700080949094B095A0952A8142223B8153221C
:107280008C8168229D8179222E8182223F819322E6
:107290008885B8239985A9234082518262827382AE
:1072A00084829582B683A78348E250E068E170E06B
:1072B00083EB9AE10E94428D89EB93E09F938F9339
:1072C0000E94FF8B8AE0829DF001839DF00D1124C6
:1072D000ED54F54E20813181428153816481758165
:1072E000868197810E94C4220E941C0B0F900F90F0
:1072F00003C082E00E94A1278DEA93E09F938F93C1
:107300000E94FF8B2FEF3FEF4FEF5FEF60E070E0E9
:1073100080E090E00E94C4220E941C0B80916302D6
:107320000F900F90882309F4CFC21F928F938AEA9F
:1073300093E09F938F930E94FF8B0F900F900F907D
:107340000F90C2C2609161027091620280E090E091
:107350000E944E8BFC0120812332A1F44AE050E0D0
:1073600060E070E001960E94F0878B0160916102FD
:107370007091620280E090E00E944E8B0430110513
:10738000ECF402C000E010E00097C1F04AE050E0E9
:1073900060E070E00E9424892AE0209FF001219F94
:1073A000F00D1124ED54F54E7187608748E250E0EE
:1073B00068E170E083EB9AE10E94428D81E00E94D7
:1073C000A12780916302882309F47EC21F928F93C4
:1073D00087EA93E09F938F930E94FF8B0F900F900B
:1073E0000F900F9071C20E94DC518091630288233C
:1073F00009F46AC21F928F9384EA93E09F938F935C
:107400000E94FF8B0F900F900F900F905DC20E9413
:10741000162880916302882309F456C21F928F9325
:1074200081EA93E09F938F930E94FF8B0F900F90C0
:107430000F900F9049C280E090E00E94E71F80917A
:107440006302882309F440C21F928F938EE993E070
:107450009F938F930E94FF8B0F900F900F900F9030
:1074600033C28091A91F81FF2DC00E94991D892BD5
:1074700049F58091A01B8F9380919F1B8F938091E2
:107480009E1B8F9380919D1B8F9383E993E09F9325
:107490008F930E94FF8B809134288F9380913328A3
:1074A0008F93809132288F93809131288F9386E833
:1074B00093E09F938F930E94FF8B0FB6F894DEBFEB
:1074C0000FBECDBF0E941C0B8091A91F9091AA1FD7
:1074D00090FF63C081E090E00E94491D3B014C0198
:1074E00080E090E00E94491D1B012C010E94C81CF5
:1074F0009F928F927F926F9285E793E09F938F93F5
:107500000E94FF8B5F924F923F922F9285E693E00D
:107510009F938F930E94FF8B222D332D442D552D49
:10752000662D772D882D992D0E94AF1B9F938F93E9
:107530007F936F938AE593E09F938F930E94FF8BD5
:10754000222D332D442D552D662D772D882D992DE7
:107550000E94101C9F938F937F936F938CE493E012
:107560009F938F930E94FF8B222D332D442D552DF9
:10757000662D772D882D992D0E94711C9F938F93D6
:107580007F936F9389E393E09F938F930E94FF8B88
:107590000FB6F894DEBF0FBECDBF0E941C0B8091CA
:1075A0006302882309F490C11F928F9386E393E0CE
:1075B0009F938F930E94FF8B0F900F900F900F90CF
:1075C00083C18091A91F82FF2BC021E048E061E0C8
:1075D00083E00E94B21280919B1B8F9380919A1B33
:1075E0008F938091991B8F938091981B8F9380919B
:1075F000971B8F938091961B8F938091951B8F93F0
:107600008091941B8F938FE193E09F938F930E94BF
:10761000FF8B0E941C0B0FB6F894DEBF0FBECDBFD0
:107620008091A91F9091AA1F91FF41C00E94FC1652
:10763000B62EA72E982E892E20E030E048EC52E49A
:10764000D501F4016B2F7A2F8F2F9E2F0E94588423
:1076500020E836EE45EC57E40E94DB8121E03EED68
:1076600042E45EE30E94BB849B01AC0160E070E0F9
:1076700080E89FE30E9410812BE43AE34DEB57E34F
:107680000E94DB819F938F937F936F938F929F9242
:10769000AF92BF9286E093E09F938F930E94FF8BFF
:1076A0000E941C0B0FB6F894DEBF0FBECDBF8091B9
:1076B0006302882309F408C11F928F9383E093E04B
:1076C0009F938F930E94FF8B0F900F900F900F90BE
:1076D000FBC0609161027091620280E090E00E94C4
:1076E0004E8B62E176E00E94628B892BB1F460914F
:1076F00061027091620280E090E00E944E8B0097E0
:1077000009F4E2C00E943C8A803108F0DDC090910B
:107710005201982B90935201D7C0809152018F70E3
:107720001F928F9383EE91E09F938F930E94FF8B24
:107730000E941C0B0F900F900F900F90C5C060918E
:1077400061027091620280E090E00E944E8B00978F
:1077500011F14AE050E060E070E00E94F087603193
:1077600098F4609348021F926F9386EF92E09F9384
:107770008F930E94FF8B41E050E063E170E088E46A
:1077800092E00E94428D11C0809148021F928F9317
:107790008DEE92E006C0809148021F928F9384EE96
:1077A00092E09F938F930E94FF8B0F900F900F900A
:1077B0000F900E941C0B80916302882309F484C0FF
:1077C0001F928F9381EE92E09F938F930E94FF8B85
:1077D0000F900F900F900F9077C0609161027091A1
:1077E000620280E090E00E944E8B8C0162E775E0BF
:1077F0000E94628B892BA1F40E94A85F80914A02AB
:1078000090914B02906190934B0280934A0242E028
:1078100050E066E170E08AE492E00E94428D54C03C
:1078200065E775E0C8010E94628B892B41F5F894E9
:107830000E94B65F88E10FB6F894809360001092C2
:1078400060000FBE84B7877F84BF8091600088612D
:107850008093600010926000789480914A02909129
:107860004B029F7E90934B0280934A0242E050E08D
:1078700066E170E08AE492E00E94428D25C067E1F3
:1078800076E0C8010E94628B20914A0230914B023F
:10789000892B21F434FF18C0F894FFCF34FF03C0C4
:1078A00082E795E002C085E795E09F938F938FED87
:1078B00091E09F938F930E94FF8B0F900F900F90FA
:1078C0000F9002C00E94351EEA85FB85118210824E
:1078D00083E02B960FB6F894DEBF0FBECDBFDF91CD
:1078E000CF911F910F91FF90EF90DF90CF90BF90BD
:1078F000AF909F908F907F906F905F904F903F9050
:107900002F9008950E949C5F6C9A6B9A6A9A6F9A66
:10791000729A749A739A779A809880B3897F80BBA1
:107920008398849887E080937E00549A0E948F29E0
:107930000E94C12981E00E94310980E090E00E940C
:10794000710C0E94135980914A0286FD239A089572
:10795000CF93DF93EC0188819981009741F08D32BC
:107960009F4009F47BC01982188283E080C00E9486
:10797000823C80914A0280FD05C081FF01C01D9BB1
:107980000E94F760809170008C7F809370008091DE
:10799000B60080628093B6001092B20082E08093BD
:1079A000B1008091B6008770E1F78091700081602E
:1079B000809370006DED78E080E090E00E94865F3B
:1079C0000E942D1F80E00E940B218DED9DE09F9372
:1079D0008F930E94FF8B0E94930F8091A91F0F909D
:1079E0000F9086FD0E943A5A80914D090E9499633A
:1079F000809149020E9440620E943D628093780912
:107A0000809149020E94406280914D091F928F939C
:107A1000809178091F928F938CE196E09F938F93CA
:107A20000E94ED8B10927A09109279090F900F90B5
:107A30000F900F900F900F908EE392E090932F286D
:107A400080932E2883E290E090938B1180938A118B
:107A50008DE29FE09983888381E009C06332E1F77A
:107A600060E070E089E799E00E945B2CE5CFDF9150
:107A7000CF9108958436910514F19F938F938EE2F0
:107A800096E09F938F930E94ED8B8091B32390910A
:107A9000B423A091B523B091B6230196A11DB11DC9
:107AA0008093B3239093B423A093B523B093B623CC
:107AB0000F900F900F900F9081E090E0089580E07C
:107AC00090E008952F923F924F925F926F927F9233
:107AD0008F929F92AF92BF92CF92DF92EF92FF92DE
:107AE0000F931F93CF93DF93CDB7DEB7C759D1095B
:107AF0000FB6F894DEBF0FBECDBFC157DF4F9983DD
:107B00008883CF58D0408A01633871F48DE799E0BB
:107B1000C956DF4F6883C759D0400E94F54BC956FC
:107B2000DF4F6881C759D040C157DF4FA881B98165
:107B3000CF58D0402D913C91213EBEE03B0709F447
:107B4000B4C340F42115310581F027343D4009F4D8
:107B5000F0C3E5C3223F4EE0340709F4C2C3293F16
:107B60003E4011F40C944849DAC346ED52E061E816
:107B700070E08DE799E00E94DB4B87E49DE08CC3C9
:107B8000E3E0F0E0EC0FFD1FE00FF11F1082C5579E
:107B9000DF4F2881CB58D040287030E040E050E0E3
:107BA00060E070E080E090E0A0E00E948887A1F1B2
:107BB00027E04AE250E06BE270E089E290E00E9448
:107BC0002D5685E298E20E949B58BC01882777FDDC
:107BD0008095982F0E947A8220E030E048EC52E4B1
:107BE0000E94DB819F938F937F936F938AE596E04A
:107BF0009F938F931F9287E78F93CE01800F911FE2
:107C000003969F938F930E94508C080F191F0FB6F5
:107C1000F894DEBF0FBECDBFC557DF4F2881CB58CC
:107C2000D040207130E040E050E060E070E080E063
:107C300090E0A0E00E948887F1F126E04AE250E05F
:107C40006BE270E089E290E00E942D5681E090E0C6
:107C50000E94AA0A80934C098CE09BE10E949B58E9
:107C6000BC01882777FD8095982F0E947A8220E0BA
:107C700030E048EC52E40E94DB819F938F937F9326
:107C80006F9384E696E09F938F931F9287E78F937D
:107C9000C8010296E1E0F0E0EC0FFD1F8E0F9F1F80
:107CA0009F938F930E94508C080F191F0FB6F89462
:107CB000DEBF0FBECDBF232D30E040E050E060E0DE
:107CC00070E080E090E0A0E00E94888701F10E94CF
:107CD000660A9F938F937F936F938FE696E09F93AF
:107CE0008F931F9287E78F93C801029641E050E07F
:107CF0004C0F5D1F840F951F9F938F930E94508C94
:107D0000080F191F0FB6F894DEBF0FBECDBFC557C1
:107D1000DF4F2881CB58D040207430E040E050E065
:107D200060E070E080E090E0A0E00E94888731F1A0
:107D30008091AE238F938091AD238F938091AC235C
:107D40008F938091AB238F938DE796E09F938F93D2
:107D50001F9287E78F93C8010296A1E0B0E0AC0FB5
:107D6000BD1F8A0F9B1F9F938F930E94508C080FFB
:107D7000191F0FB6F894DEBF0FBECDBFC557DF4F3A
:107D80002881CB58D040207830E040E050E060E0DF
:107D900070E080E090E0A0E00E94888741F1F894D4
:107DA0008091102890911128A0911228B091132849
:107DB0007894BF93AF939F938F938BE896E09F93B4
:107DC0008F931F9287E78F93C801029621E030E0DE
:107DD0002C0F3D1F820F931F9F938F930E94508CF7
:107DE000080F191F0FB6F894DEBF0FBECDBF20E0FD
:107DF000392D317040E050E060E070E080E090E0CC
:107E0000A0E00E94888709F0CEC420E0392D3270AE
:107E100040E050E060E070E080E090E0A0E00E9490
:107E2000888709F032C520E0392D347040E050E0F9
:107E300060E070E080E090E0A0E00E94888709F0B8
:107E400055C520E0392D387040E050E060E070E02A
:107E500080E090E0A0E00E94888709F076C520E0ED
:107E6000392D307140E050E060E070E080E090E05B
:107E7000A0E00E94888709F0DAC520E0392D307231
:107E800040E050E060E070E080E090E0A0E00E9420
:107E9000888709F0FCC520E0C257DF4F3881CE58F3
:107EA000D04040E050E060E070E080E090E0A0E092
:107EB0000E94888709F018C620E0CC56DF4F388131
:107EC000C459D04040E050E060E070E080E090E0D5
:107ED000A0E00E94888709F034C620E030E0C45753
:107EE000DF4F4881CC58D040417050E060E070E0F6
:107EF00080E090E0A0E00E94888709F050C620E072
:107F000030E0C457DF4F4881CC58D040427050E039
:107F100060E070E080E090E0A0E00E94888709F0D7
:107F200071C620E030E0C657DF4F4881CA58D040C4
:107F300050E060E070E080E090E0A0E00E94888780
:107F400009F093C620E030E0C457DF4F4881CC5899
:107F5000D040487050E060E070E080E090E0A0E049
:107F60000E94888709F0ABC620E030E0C457DF4F9D
:107F70004881CC58D040407150E060E070E080E033
:107F800090E0A0E00E94888709F0C9C620E030E0B8
:107F9000C457DF4F4881CC58D040407250E060E079
:107FA00070E080E090E0A0E00E94888709F0E7C6DA
:107FB00020E030E0C457DF4F4881CC58D0404074B7
:107FC00050E060E070E080E090E0A0E00E948887F0
:107FD00009F005C7C457DF4FF881CC58D040F0787E
:107FE000EF2E20E030E04F2F50E060E070E080E0C6
:107FF00090E0A0E00E94888709F021C7C357DF4FB7
:108000002881CD58D0402170F22E20E030E040E0B1
:108010005F2D60E070E080E090E0A0E00E94888743
:1080200009F017C720E030E04E2D50E060E070E02E
:1080300080E090E0A0E00E94888709F015C720E06A
:1080400030E040E05F2D60E070E080E090E0A0E094
:108050000E94888709F03AC720E030E040E0C3572B
:10806000DF4F5881CD58D040527060E070E080E022
:1080700090E0A0E00E94888709F05AC720E030E035
:1080800040E0C357DF4F5881CD58D040547060E076
:1080900070E080E090E0A0E00E94888709F078C757
:1080A00020E030E040E0C357DF4F5881CD58D0404A
:1080B000507160E070E080E090E0A0E00E9488876E
:1080C00009F096C720E030E040E0C357DF4F588109
:1080D000CD58D040507260E070E080E090E0A0E0C9
:1080E0000E94888709F0C0C720E030E040E0C35715
:1080F000DF4F5881CD58D040507460E070E080E090
:1081000090E0A0E00E94888709F0EBC720E030E013
:1081100040E0C357DF4F5881CD58D040587060E0E1
:1081200070E080E090E0A0E00E94888711F00C945D
:10813000AE4820E030E040E0CB56DF4F5881C559D3
:10814000D04060E070E080E090E0A0E00E9488878E
:1081500011F00C94DF48779A80915109909152095F
:1081600092FD749AC557DF4F2881CB58D040392DE6
:10817000C457DF4F4881CC58D040C357DF4F588198
:10818000CD58D040CF56DF4F6881C159D040CE5630
:10819000DF4F7881C259D040CD56DF4F8881C35917
:1081A000D040982DA0E0FE0133967F010E94888781
:1081B00011F00C9416498091480280618983809166
:1081C00071098A83F701E00FF11F10828091510934
:1081D0009091520998012D5F3F4F790180FF0CC0AB
:1081E000FF922F938CEE97E09F938F930E94ED8BDD
:1081F0000F900F900F900F90B701CE0101960E9443
:10820000245580914A0282FF0AC020E134E2A7018E
:10821000BE016F5F7F4F81E592E00E94AA59809175
:1082200051099091520982FD73980E943F618DE738
:1082300099E00E94F74B80914A0290914B0290FF87
:108240003BC00F5F1F4F0E943D62F82E89E10E94E4
:10825000556220914A0230914B0230FF29C0739839
:10826000809171098F5F809371098A83B8016F5F74
:108270007F4FCE0101960E9424558DE799E00E9420
:10828000F74B40E050E065E880918E1190918F119E
:108290000E94B24D81EE9EE0C157DF4FA881B981A7
:1082A000CF58D0408D939C9338C000E010E0D1CFE0
:1082B0008F2D0E945562739A80914E0990914F09BB
:1082C000892B11F00E94F760809171098F5F809374
:1082D0007109809151099091520982FF4ECC739A95
:1082E0004CCC89E699E00E945850892BB1F00E944D
:1082F0003F6180914A0287FD2B9860E470E089E637
:1083000099E00E94315089EF9EE0C157DF4FE8812C
:10831000F981CF58D0409183808381E0CBC7C1578A
:10832000DF4FA881B981CF58D0401D921C9283E0C5
:10833000C1C7623191F780914A0290914B0291FD41
:108340001CCC23E333E343E150E46091AB23709111
:10835000AC238091AD239091AE230E94D78187FFFB
:1083600014C08091B7239091B823A091B923B09104
:10837000BA230196A11DB11D8093B7239093B82312
:10838000A093B923B093BA23F8CBF8018081813050
:1083900071F50180F281E02D2081C557DF4F2883E0
:1083A000CB58D04091803281C457DF4F3883CC58AE
:1083B000D0404381C357DF4F4883CD58D0405481CC
:1083C000CF56DF4F5883C159D0408581CE56DF4FFD
:1083D0008883C259D0409681CD56DF4F9883C359C8
:1083E000D0408780A084B184612C712C47C082303A
:1083F000E1F463807480A12CB12CB1E0C557DF4F4C
:10840000B883CB58D040912CC457DF4F1882CC583A
:10841000D040E0E8C357DF4FE883CD58D040CF5677
:10842000DF4F1882C159D0401EC0843009F0A5CB5F
:10843000A12CB12C612C712CF5E0C557DF4FF883CE
:10844000CB58D040912CC457DF4F1882CC58D04025
:10845000C357DF4F1882CD58D04021E0CF56DF4FB1
:108460002883C159D040CE56DF4F1882C259D04020
:10847000CD56DF4F1882C359D040812CC457DF4FEF
:108480003881CC58D0403470C657DF4F3883CA5833
:10849000D04020E030E0C657DF4F4881CA58D04076
:1084A00050E060E070E080E090E0A0E00E9488870B
:1084B00009F08C9AC557DF4F4881CB58D0404072A5
:1084C000342E242F30E040E050E060E070E080E0A7
:1084D00090E0A0E00E94888711F00E94660A592D62
:1084E0005074C257DF4F5883CE58D04020E0352F0C
:1084F00040E050E060E070E080E090E0A0E00E94AA
:10850000888711F00E94991D892D8078CC56DF4F05
:108510008883C459D04020E0382F40E050E060E02C
:1085200070E080E090E0A0E00E94888751F00E9417
:108530000C0A609318287093192880931A28909336
:108540001B28C557DF4F2881CB58D040217030E021
:1085500040E050E060E070E080E090E0A0E00E9449
:108560008887F1F08AE99AE19F938F9382E496E0FD
:108570009F938F931F9287E78F93CE0103969F93CC
:108580008F930E94508C7C010E943A3D0FB6F89464
:10859000DEBF0FBECDBF892B09F0EFCA870102C035
:1085A00000E010E0C557DF4F2881CB58D040227043
:1085B00030E040E050E060E070E080E090E0A0E07B
:1085C0000E948887C9F1C80102966AE476E0E1E07A
:1085D000F0E0EC0FFD1F8E0F9F1F0E946B8B0D5F55
:1085E0001F4FB5E2CB2EB8E2DB2E8AEDE82E83E0FA
:1085F000F82E97E7592ED6018D916D011F928F931A
:10860000FF92EF921F925F92C8010296E1E0F0E0C4
:10861000EC0FFD1F8E0F9F1F9F938F930E94508C16
:10862000080F191F0FB6F894DEBF0FBECDBF3DE295
:10863000C31638E2D306F9F6C557DF4F2881CB5869
:10864000D040247030E040E050E060E070E080E036
:1086500090E0A0E00E94888709F446C0C801029615
:108660006EE476E041E050E04C0F5D1F840F951FF3
:108670000E946B8B0C5F1F4F2E015AE7450E511C59
:1086800080E1D2011D928A95E9F728E0A20168E90C
:1086900080EB0E94F6106201B8E0CB0ED11CFAED1F
:1086A000EF2EF3E0FF2EA7E72A2EF20181912F0192
:1086B0001F928F93FF92EF921F922F92C801029602
:1086C00021E030E02C0F3D1F820F931F9F938F936B
:1086D0000E94508C080F191F0FB6F894DEBF0FBE12
:1086E000CDBF4C145D0409F7C357DF4F5881CD58F7
:1086F000D0405078CB56DF4F5883C559D04020E04A
:1087000030E040E060E070E080E090E0A0E00E94B7
:108710008887E1F480914E0990914F099F938F9340
:1087200083E596E09F938F931F9287E78F93CE0107
:10873000800F911F03969F938F930E94508C080F78
:10874000191F0FB6F894DEBF0FBECDBF20E030E09A
:1087500040E050E0CF56DF4F6881C159D040617092
:1087600070E080E090E0A0E00E94888709F40FCAE2
:10877000E3E0F0E0EC0FFD1FE00FF11F80E28083EB
:10878000E3EDF3E280810F5F1F4F882309F4F8C9FE
:108790008081A1E0B0E0AC0FBD1FA00FB11F129609
:1087A0008C933196EFCFA114B10409F42ECBF89439
:1087B000C0901028D0901128E0901228F090132833
:1087C00078948091041B9091051BA091061BB09199
:1087D000071BA7019601281B390B4A0B5B0BCA012B
:1087E000B9010E9478821B012C01B50180E090E064
:1087F0000E9478829B01AC01C201B1010E94DB8121
:108800002C015F928F937F936F9386E996E09F93FD
:108810008F931F9287E78F939E01200F311F2D5F4B
:108820003F4F3F932F93C956DF4F6883C759D040BE
:10883000CA56DF4F7883C659D0400E94508C080F2B
:10884000191FC956DF4F6881C759D040CA56DF4F3C
:108850007881C659D040862F972FA42DB52D8093AF
:108860001D2890931E28A0931F28B0932028C09203
:10887000041BD092051BE092061BF092071B0FB65B
:10888000F894DEBF0FBECDBFC0CAA114B10409F475
:10889000CACAF8948091DB1A9091DC1AA091DD1A73
:1088A000B091DE1A78949F938F9380914F028F93AB
:1088B00080914E028F9383EA96E09F938F931F924D
:1088C00087E78F93C8010296A1E0B0E0AC0FBD1F0F
:1088D0008A0F9B1F9F938F930E94508C080F191F24
:1088E0000FB6F894DEBF0FBECDBF9DCAF89480913D
:1088F000142890911528A0911628B09117287894E3
:10890000BF93AF939F938F9383EB96E09F938F9347
:108910001F9287E78F93C801029621E030E02C0F69
:108920003D1F820F931F9F938F930E94508C080FBF
:10893000191FC8010E943A3D0FB6F894DEBF0FBE62
:10894000CDBF892B09F019C97CCAA114B10409F45F
:1089500086CAF894C0901428D0901528E090162864
:10896000F090172878948091081B9091091BA09192
:108970000A1BB0910B1BA7019601281B390B4A0B50
:108980005B0BCA01B9010E9478821B012C01B50161
:1089900080E090E00E9478829B01AC01C201B101AD
:1089A0000E94DB812C015F928F937F936F938EEBFC
:1089B00096E09F938F931F9287E78F939E01200FDE
:1089C000311F2D5F3F4F3F932F93C956DF4F688371
:1089D000C759D040CA56DF4F7883C659D0400E944D
:1089E000508C080F191FC956DF4F6881C759D040F6
:1089F000CA56DF4F7881C659D040862F972FA42DB5
:108A0000B52D8093212890932228A0932328B093FA
:108A10002428C092081BD092091BE0920A1BF092F6
:108A20000B1B0FB6F894DEBF0FBECDBF18CAAB2824
:108A300009F423CAF8948091DF1A9091E01AA0916A
:108A4000E11AB091E21A78949F938F9380914D022E
:108A50008F9380914C028F938BEC96E09F938F9332
:108A60001F9287E78F93C8010296A1E0B0E0AC0F98
:108A7000BD1F8A0F9B1F9F938F930E94508C080FDE
:108A8000191F0FB6F894DEBF0FBECDBFF6C9809197
:108A9000AF239091B023A091B123B091B223BF93A3
:108AA000AF939F938F938BED96E09F938F931F923D
:108AB00087E78F93C801029621E030E02C0F3D1F1D
:108AC000820F931F9F938F930E94508C080F191F42
:108AD000C8010E943A3D0FB6F894DEBF0FBECDBF6D
:108AE000892B09F04AC8D7C98091A01B8F93809128
:108AF0009F1B8F9380919E1B8F9380919D1B8F93C3
:108B000086EE96E09F938F931F9287E78F93C8011D
:108B10000296A1E0B0E0AC0FBD1F8A0F9B1F9F9390
:108B20008F930E94508C080F191FC8010E943A3D74
:108B30000FB6F894DEBF0FBECDBF892B09F01DC85C
:108B4000BBC980911B288F9380911A288F938091A5
:108B500019288F93809118288F9381EF96E09F9327
:108B60008F931F9287E78F93C801029621E030E030
:108B70002C0F3D1F820F931F9F938F930E94508C49
:108B8000080F191FC8010E943A3D0FB6F894DEBFC6
:108B90000FBECDBF892B11F00C94BD3D9EC981E065
:108BA0000E94BD09209168023091690240916A02D9
:108BB00050916B020E9458849F938F937F936F9381
:108BC0008EEF96E09F938F931F9287E78F93C80154
:108BD0000296A1E0B0E0AC0FBD1F8A0F9B1F9F93D0
:108BE0008F930E94508C080F191FC8010E943A3DB4
:108BF0000FB6F894DEBF0FBECDBF892B11F00C94D9
:108C0000BD3D7DC982E00E94BD0920916402309182
:108C1000650240916602509167020E9458849F93BA
:108C20008F937F936F938BE097E09F938F931F9227
:108C300087E78F93C801029621E030E02C0F3D1F9B
:108C4000820F931F9F938F930E94508C080F191FC0
:108C5000C8010E943A3D0FB6F894DEBF0FBECDBFEB
:108C6000892B11F00C94BD3D5CC983E00E94BD09C5
:108C70009F938F937F936F9388E197E09F938F9358
:108C80001F9287E78F93C8010296A1E0B0E0AC0F76
:108C9000BD1F8A0F9B1F9F938F930E94508C080FBC
:108CA000191F8C98C8010E943A3D0FB6F894DEBF98
:108CB0000FBECDBF892B11F00C94BD3D43C98091EF
:108CC000A91F87FF51C921E042E161E080ED0E94C8
:108CD000DD5A9F938F937F936F9385E297E09F93E5
:108CE0008F931F9287E78F93C801029621E030E0AF
:108CF0002C0F3D1F820F931F9F938F930E94508CC8
:108D0000080F191FC8010E943A3D0FB6F894DEBF44
:108D10000FBECDBF892B11F00C94BD3D25C98091AC
:108D2000A91F87FF33C921E042E162E080ED0E9484
:108D3000DD5A9F938F937F936F9383E397E09F9385
:108D40008F931F9287E78F93C8010296A1E0B0E04E
:108D5000AC0FBD1F8A0F9B1F9F938F930E94508C57
:108D6000080F191FC8010E943A3D0FB6F894DEBFE4
:108D70000FBECDBF892B11F00C94BD3D07C980916A
:108D8000A91F87FF15C921E042E163E080ED0E9441
:108D9000DD5A9F938F937F936F9381E497E09F9326
:108DA0008F931F9287E78F93C801029621E030E0EE
:108DB0002C0F3D1F820F931F9F938F930E94508C07
:108DC000080F191FC8010E943A3D0FB6F894DEBF84
:108DD0000FBECDBF892B11F00C94BD3DE9C8809129
:108DE000A91F87FFF7C821E042E164E080ED0E94FF
:108DF000DD5A9F938F937F936F938FE497E09F93B8
:108E00008F931F9287E78F93C8010296A1E0B0E08D
:108E1000AC0FBD1F8A0F9B1F9F938F930E94508C96
:108E2000080F191FC8010E943A3D0FB6F894DEBF23
:108E30000FBECDBF892B11F00C94BD3DCBC88091E6
:108E4000A91F82FFDBC846E061E083E00E94B21206
:108E5000D5C88091A91F82FFE5C821E046E061E006
:108E600083E00E94B212DEC88091A91F82FFE7C88A
:108E70008091971B8F938091961B8F938091951B68
:108E80008F938091941B8F938DE597E09F938F93A1
:108E90001F9287E78F93C801029641E050E04C0F84
:108EA0005D1F840F951F9F938F930E94508C080F16
:108EB000191FC8010E943A3D0FB6F894DEBF0FBEDD
:108EC000CDBF892B11F00C94BD3DB9C88091A91F6D
:108ED00082FFC2C880919B1B8F9380919A1B8F93B6
:108EE0008091991B8F938091981B8F9385E697E0D3
:108EF0009F938F931F9287E78F93C8010296E1E0BB
:108F0000F0E0EC0FFD1F8E0F9F1F9F938F930E9429
:108F1000508C080F191FC8010E943A3D0FB6F894F3
:108F2000DEBF0FBECDBF892B11F00C94BD3D94C8A0
:108F30008091A91F9091AA1F90FFA0C880E090E0A7
:108F40000E94491D9F938F937F936F9380E797E0D3
:108F50009F938F931F9287E78F93C801029641E0FA
:108F600050E04C0F5D1F840F951F9F938F930E94BD
:108F7000508C080F191FC8010E943A3D0FB6F89493
:108F8000DEBF0FBECDBF892B11F00C94BD3D76C85E
:108F90008091A91F9091AA1F90FF82C881E090E064
:108FA0000E94491D9F938F937F936F9380E897E072
:108FB0009F938F931F9287E78F93C8010296E1E0FA
:108FC000F0E0EC0FFD1F8E0F9F1F9F938F930E9469
:108FD000508C080F191FC8010E943A3D0FB6F89433
:108FE000DEBF0FBECDBF892B11F00C94BD3D58C81C
:108FF0008091A91F9091AA1F90FF64C881E090E022
:109000000E94491D6B017C0180E090E00E94491D97
:109010009B01AC01C701B6010E94AF1B9F938F93C8
:109020007F936F9381E997E09F938F931F9287E7D8
:109030008F93C801029641E050E04C0F5D1F840FF2
:10904000951F9F938F930E94508C080F191FC80182
:109050000E943A3D0FB6F894DEBF0FBECDBF892BFC
:1090600011F00C94BD3D2EC88091A91F9091AA1FAC
:1090700090FF3AC881E090E00E94491D6B017C019D
:1090800080E090E00E94491D9B01AC01C701B60140
:109090000E94101C9F938F937F936F938CE997E0AE
:1090A0009F938F931F9287E78F93C8010296E1E009
:1090B000F0E0EC0FFD1F8E0F9F1F9F938F930E9478
:1090C000508C080F191FC8010E943A3D0FB6F89442
:1090D000DEBF0FBECDBF892B11F00C94BD3D0C94AB
:1090E00074408091A91F9091AA1F90FF0FC881E042
:1090F00090E00E94491D6B017C0180E090E00E949D
:10910000491D9B01AC01C701B6010E94711C9F93D0
:109110008F937F936F938AEA97E09F938F931F9229
:1091200087E78F93C801029641E050E04C0F5D1F26
:10913000840F951F9F938F930E94508C080F191FC7
:10914000C8010E943A3D0FB6F894DEBF0FBECDBFF6
:10915000892B11F00C94BD3D0C9486408091A91F81
:109160009091AA1F91FD02C00C9499400E94FC1698
:109170009F938F937F936F938DEB97E09F938F9344
:109180001F9287E78F93C8010296E1E0F0E0EC0FB1
:10919000FD1F8E0F9F1F9F938F930E94508C080F6F
:1091A000191FC8010E943A3D0FB6F894DEBF0FBEEA
:1091B000CDBF892B11F00C94BD3D0C949940D30187
:1091C00016968C9116971F928F9315968C911597E2
:1091D0001F928F9313968C9113971F928F931296D1
:1091E0008C911F928F938EEC97E09F938F931F9299
:1091F00087E78F93C8010296E1E0F0E0EC0FFD1FD6
:109200008E0F9F1F9F938F930E94508C080F191FE2
:10921000C8010E943A3D0FB6F894DEBF0FBECDBF25
:10922000892B11F00C94BD3D0C94AB4080915109F9
:109230009091520982FD0CC080914A0280FD08C0C5
:1092400081FD02C00C94DB401D9902C00C94DB40F0
:10925000FF92EF9285EE97E09F938F930E94ED8BA4
:10926000809163020F900F900F900F90882311F45C
:109270000C94DB401F928F938AED9DE09F938F9318
:109280000E94FF8B0F900F900F900F900C94DB407B
:1092900089E699E00E945850892B09F43EC80E9443
:1092A000F76080914A0287FD02C00C94BD3D2B9A65
:1092B0000C94BD3DC956DF4F0FB6F894DEBF0FBE0C
:1092C000CDBFDF91CF911F910F91FF90EF90DF9075
:1092D000CF90BF90AF909F908F907F906F905F9056
:1092E0004F903F902F9008950C941E4C4F925F9298
:1092F0006F927F928F929F92AF92BF92CF92DF92A6
:10930000EF92FF920F931F93CF93DF93CDB7DEB70A
:1093100060970FB6F894DEBF0FBECDBF6B010E9401
:109320003D62E82FF0E0EE0FFF1FE353F54E808122
:109330009181019691838083809151099091520986
:1093400081FD749880904A0290904B020E9478545C
:109350007C01FC018081982F92959F70913099F447
:109360008F7051F48091B11A9091B21A0196909336
:10937000B21A8093B11AFAC0B60185E398E20E944E
:10938000944B892B51F08091AF1A9091B01A0196AD
:109390009093B01A8093AF1AE9C0C40184E0989FFB
:1093A000812D99271124F82FF1708F2E88E899E0EC
:1093B0000E949F4E8C01009709F448C0B601C80175
:1093C00002960E94944B892BE9F1980147EF58E0EF
:1093D00060E074E6C8010F960E941F51F701918169
:1093E000F8018481981321C082858F5F82878091E4
:1093F000AD1A9091AE1A01969093AE1A8093AD1A61
:1094000084E00E949555F801208530E0281739073F
:1094100008F066C184E00E949555F8018087F70145
:1094200080818F70F8018187A1C0F801128684E0E5
:109430000E949555F8018087F70180818F70F801AF
:1094400081874FC1C8010E94474FB4CF84E092E0AA
:109450000E94344E8C01009709F488C0B601C801FF
:1094600002960E948B4BF70181818150F801848321
:1094700080E091E0A0E0B0E083879487A587B6877D
:10948000128684E00E949555F8018087F70180815B
:109490008F70F8018187B80188E899E00E94FF4E3B
:1094A000980147EF58E060E074E6C8010F960E940B
:1094B0001F5199249394F7018181F8018483F70166
:1094C00080818F70F801878384E00E949555F801B0
:1094D000858383E00E9495555C01F801868387812E
:1094E0008F3009F0912CF7014180F8018481481AEE
:1094F000512C612C712C46E0440C551C661C771CC9
:109500004A95D1F72385348545855685A0ECB0E092
:109510000E943685BB27A92F982F872F480E591EEA
:109520006A1E7B1E43865486658676868091510925
:109530009091520981FD24C080914A0280FD20C093
:1095400081FD1CC0992091F082E08093BC23109291
:10955000BE231092BD231093C0230093BF234CEB76
:1095600053E262E18AE292E00E94B24D8091510999
:109570009091520981FFB7C0749AB5C01D9BE2CF8C
:10958000A4E6B0E0A30192010E943685672F782FF0
:10959000892F992724E630E040E050E00E94818541
:1095A0007F936F93452C562C672C77245F924F92B4
:1095B000BB24BF92AF92F80185811F928F93F70170
:1095C00080818F701F928F9381811F928F93F601FC
:1095D00081811F928F9380811F928F93C701029682
:1095E0009F938F938DEF97E09F938F930E94ED8BC6
:1095F000809163020FB6F894DEBF0FBECDBF882303
:1096000061F01F928F9387ED9DE09F938F930E944F
:10961000FF8B0F900F900F900F9080914A029091C6
:109620004B0296FF2DC0882059F1F7012081322F7F
:109630003F70832F90E00297D4F08FEF830F207F4D
:10964000822B80838DE799E00E9474498091AB1A48
:109650009091AC1A01969093AC1A8093AB1A8091BA
:1096600051099091520996FF0BC0739809C08091DF
:10967000B11A9091B21A01969093B21A8093B11ACE
:109680008091A91F86FF5ECF0E942C5AC7010596C4
:109690000E94F859F70181811F928F93F80186810A
:1096A0001F928F9385811F928F9381E498E09F93FF
:1096B0008F931F9280E18F939E012F5F3F4F79011F
:1096C000FF922F930E94508C82E00E94125AC70191
:1096D0000E94F8590FB6F894DEBF0FBECDBF32CF4F
:1096E000812C912CE8CE60960FB6F894DEBF0FBEA9
:1096F000CDBFDF91CF911F910F91FF90EF90DF9041
:10970000CF90BF90AF909F908F907F906F905F9021
:109710004F9008950895FB012081FC012083FB01F7
:109720002181FC0121830895FC019081DB018C9152
:10973000981309C081E090E0318111962C91321785
:1097400021F080E0089580E090E00895BC0185E379
:1097500098E20C948B4BDC011996ED91FC911A97D1
:109760000280F381E02D309709F0099408950F935A
:109770001F93CF93DF9300D0CDB7DEB78C0188E184
:109780000E94A855BC01CE0101960E948B4BD801C6
:109790001996ED91FC911A970190F081E02DBE0190
:1097A0006F5F7F4FC80109950F900F90DF91CF91A8
:1097B0001F910F910895EF92FF920F931F93CF93F4
:1097C000DF93EC018B017A014AEE52E00E94044CD7
:1097D000FA86E9866EEE72E0C801DF91CF911F91A3
:1097E0000F91FF90EF900C945D4C0C941C4CCF9318
:1097F000DF93EC0165E378E288E10E949E55CE019B
:10980000DF91CF910C941E4CEF92FF920F931F9318
:10981000CF93DF93EC018B017A010E94394CF886DB
:10982000EF8262EF72E0C801DF91CF911F910F913B
:10983000FF90EF900C945D4C0C94414C0C94B966E5
:10984000DC011796ED91FC9118970190F081E02DC5
:109850000994DC011796ED91FC9118970280F38131
:10986000E02D309709F0099408958CE891E10C946B
:109870009B4EFC0173836283BC018CE891E10C94E4
:10988000FF4EBC018CE891E10C94E44ECF93DF9342
:10989000EC018CE891E10E949F4E009749F0FC0199
:1098A000228133812C173D0729F00E94474FF5CFC5
:1098B00080E090E0DF91CF9108950F931F93CF93B5
:1098C000DF938B010E94464CEC01009731F01D8321
:1098D0000C83C8010E94EA688E83DF91CF911F91AB
:1098E0000F9108951F93CF93DF93EC01162FEC8116
:1098F000FD813097D1F090938F1180938E1182E08B
:109900008887CE0106960995992787FD909502973D
:10991000029710F0133839F4BE01CE01DF91CF91D8
:109920001F910C949F4C81E08887DF91CF911F910C
:109930000895FC01208520FD0C94724C0895CF926F
:10994000DF92EF92FF920F931F93CF93DF93EC017F
:109950006B01E0908E11F0908F1100919011109199
:109960009111F801EC17FD0739F0309709F44AC05E
:109970000190F081E02DF6CF209709F443C088854F
:10998000882309F118860115110561F0C017D10768
:1099900029F0AE0167E8C8010E94994CF8010081E6
:1099A0001181F1CFEC81FD81309769F0CC15DD0597
:1099B00051F0D0938F11C0938E1140E050E063E8D6
:1099C000CE0106960995E0919011F0919111CE1774
:1099D000DF0769F4888199819093911180939011A8
:1099E0000DC0808191818C179D0721F0FC0130977B
:1099F000C1F704C08881998191838083F0928F118F
:109A0000E0928E11DF91CF911F910F91FF90EF9017
:109A1000DF90CF9008951F93CF93DF9310929A1108
:109A2000C0919011D091911111E0209779F0898522
:109A3000882341F01887198640E050E062E8CE01A3
:109A40000E94724C0990D881C02DEFCFDF91CF9149
:109A50001F91089580913D1291E0980F90933D12CF
:109A6000089560918E1170918F110C949F4C8AE82B
:109A700080933D1210923B1210923C121092911161
:109A80001092901110928F1110928E110895809162
:109A90009A1181110E940B4D70913C12772309F4A9
:109AA00051C0E0913B122E2F30E085E0E89FF0019D
:109AB0001124E556FE4E60816093991141815281D7
:109AC00050939811409397118381948190939611AC
:109AD000809395112F5F3F4F2F71332720933B12B7
:109AE000715070933C12009731F5809190119091D4
:109AF000911190939411809393118091931190916F
:109B00009411892BF9F080919A1181110E940B4DCB
:109B100040919711509198116091991180919311F2
:109B2000909194110E94994CE0919311F0919411AD
:109B300080819181DECF613819F421E0FC0120871A
:109B40000E94994C80919A1120913C1290E0820FD2
:109B5000911D089580919A1120913C1290E0820FFE
:109B6000911D089520913C122032B9F0E0913B12F2
:109B7000E20FEF71E093921135E0E39FF0011124C1
:109B8000E556FE4E608352834183948383832F5F27
:109B900020933C1280E090E0089581E090E00895E9
:109BA000CF93DF93C0918E11D0918F110E94994C69
:109BB000D0938F11C0938E11DF91CF910895AB0197
:109BC0003091901120919111E32FF22FE817F907AE
:109BD000B1F0309721F00190F081E02DF7CF0097A0
:109BE00071F0FC0130832183909391118093901147
:109BF00021E020871782168261E80C94D04D0895E9
:109C0000009749F0FC0120852150223020F421E00A
:109C1000218720939A11089521E030E0FC0180858E
:109C2000811102C020E030E0C9010895CF93DF9395
:109C3000EC014A815B8160E070E08C819D810E9433
:109C40005B8B2A813B8188819981289FA001299F74
:109C5000500D389F500D112460E070E08E819F817F
:109C6000DF91CF910C945B8BFC018281938120E08A
:109C700030E028173907D1F0A481B581A20FB31FB6
:109C80004C91411110C081E08C9380819181289F7B
:109C9000A001299F500D389F500D11248681978176
:109CA000840F951F08952F5F3F4FE3CF80E090E032
:109CB0000895FC01268137814281538180E090E044
:109CC00084179507C9F02617370781F4A481B58159
:109CD000A80FB91F2C91121614F421502C93048054
:109CE000F581E02DE80FF91F80810895A081B181F1
:109CF0002A0F3B1F0196E4CF8FEF0895FC01868168
:109D0000978168177907A0F0A081B18142815381C2
:109D1000A49F9001A59F300DB49F300D1124280FF2
:109D2000391F81E090E06217730720F080E008950A
:109D300080E090E00895FC01118210820895FC01FA
:109D4000808191810895FB0120813181FC01318363
:109D500020830895DC01ED91FC91309731F08081F2
:109D60009181009729F0FC01FACF80E090E00895FE
:109D7000CF010895DC01ED91FC9111973097A9F086
:109D800020813181232B21F41D921C92CF01089553
:109D9000A081B1818D919C911197892B11F0FD01CA
:109DA000F7CF11821082CD01089580E090E00895F0
:109DB000DC01ED91FC911197309721F020813181E8
:109DC0002D933C93CF010895DC01ED91FC913097E8
:109DD000A9F0A0E0B0E020813181E617F70741F457
:109DE000109709F4DC012D933C93118210820895A1
:109DF0002115310519F0DF01F901EDCF08950F9319
:109E00001F93CF93DF938C01EB010E94E44E1982E4
:109E10001882C8010E94AA4E009711F4F80101C0EF
:109E2000FC01D183C083DF91CF911F910F910895E1
:109E30000F931F93CF93DF93EC018B010E94E44EAD
:109E400088819981F8019183808319830883DF9148
:109E5000CF911F910F910895DC01ED91FC9180E06D
:109E600090E0309729F001960190F081E02DF9CF34
:109E70000895FB01309719F4BA010C94184F8081B2
:109E80009181DA018D939C935183408308950097CB
:109E900021F0FC0180819181089580E090E0089597
:109EA0008091401290914112892B29F410923F1217
:109EB00010923E1208950E94445EE0914012F0918B
:109EC00041122281338140815181240F351F281B8B
:109ED000390B0480F581E02D309769F04281538180
:109EE00060817181460F571F481B590B421753075A
:109EF00080F79A01EECF280F391F30933F1220933D
:109F00003E12089582E792E00C94004EEF92FF9289
:109F10000F931F93CF93DF938C01FC01808191817C
:109F2000009799F08A359105D9F0F80111821082D5
:109F300083E068C0868197818417950709F049C03E
:109F40000480F581E02D3097A9F71092411210920C
:109F500040128AE590E0F8019183808381E052C04D
:109F6000673891F16238A9F7C0914012D09141123F
:109F7000E12CF12C209769F3CE010E94BB6C892B58
:109F8000F1F0AE0168E88E819F810E94B24D892B6D
:109F9000A1F41F821E828C819D81E114F10421F0C5
:109FA000F7019583848304C09093411280934012FB
:109FB0001D821C820E94504FD7CF0E94824F7E018B
:109FC0000C80DD81C02DD6CFE0914012F09141127E
:109FD000BACFF0934112E0934012A481B58110975B
:109FE00009F4B7CF16968D919C9117978417950712
:109FF00011F0FD01F2CF14968D919C9115979583E8
:10A000008483EBCFDF91CF911F910F91FF90EF9061
:10A010000895CF93DF93EC010E94824F8E819F8140
:10A020003091401220914112892B59F0E32FF22FE9
:10A03000309739F0EC17FD0781F00480F581E02DB1
:10A04000F7CF80918E1190918F119F838E833C83E7
:10A050002D83D0934112C0934012DF91CF910C9485
:10A06000504FCF93DF93EC010E949B6CCE01DF91A8
:10A07000CF910C940950CF93DF93EC010E94A76C11
:10A08000CE01DF91CF910C940950CF93DF93EC0177
:10A090000E94B16CCE01DF91CF910C940950FC016C
:10A0A00020813181260F371F318320830C94504F3C
:10A0B00021E030E0FC0186819781892B11F020E0BE
:10A0C00030E0C9010895FC012281338180819181B2
:10A0D000820F931F0895FC0180819181089581E092
:10A0E00090E02091401230914112232B11F480E036
:10A0F00090E008958091401290914112892B29F0AF
:10A1000080913E1290913F12089580E090E0089572
:10A11000CF93DF93EC01E0914012F09141128E1742
:10A120009F0769F48C819D81909341128093401226
:10A130000DC0848195818C179D0721F0FC0130971B
:10A14000C1F706C08C819D81958384830E94504F06
:10A150001D821C821F821E82DF91CF910895EF9293
:10A16000FF920F931F93CF93DF938C017A01FC0131
:10A1700080819181009741F08B34910501F1F801C4
:10A180001182108283E048C083E492E10E949F4ED6
:10A19000EC01209751F06C817D81CE0102960E94E6
:10A1A00031500990D881C02DF4CF81E080934212C4
:10A1B0008BE490E0F8019183808381E02DC06838C2
:10A1C000E1F783E492E10E949F4EEC01209781F336
:10A1D000CE010296E816F906D9F4BE0183E492E1B5
:10A1E0000E94E44EE0908E11F0908F118A859B853D
:10A1F00090938F1180938E11EC85FD85309719F027
:10A200008E859F850995F0928F11E0928E11D0CFA7
:10A210000990D881C02DDACFDF91CF911F910F9196
:10A22000FF90EF9008951092421283E492E10E9411
:10A230009B4E60E070E08CE792E00C94DF4D0F9352
:10A240001F93CF93DF93EC0100918E1110918F112A
:10A250001B870A875D874C873F872E878091421234
:10A26000882379F08CE792E090938F1180938E1180
:10A27000CE0102960E94315010938F1100938E11DF
:10A2800002C07D836C83BE0183E492E10E94E44EB0
:10A29000BE0183E492E1DF91CF911F910F910C9465
:10A2A000FF4E0F931F93CF93DF93EC0180914212E7
:10A2B000882391F000918E1110918F118CE792E01C
:10A2C00090938F1180938E11CE0102960E943B5085
:10A2D00010938F1100938E11BE0183E492E10E94CE
:10A2E000E44EBE0183E492E1DF91CF911F910F9183
:10A2F0000C94FF4E0F931F93CF93DF93EC0180914B
:10A300004212882391F000918E1110918F118CE7E9
:10A3100092E090938F1180938E11CE0102960E944D
:10A32000455010938F1100938E11BE0183E492E18A
:10A330000E94E44EBE0183E492E1DF91CF911F9130
:10A340000F910C94FF4ECF93DF93EC01809142125A
:10A35000882329F0CE0102960E94885004C01F82F3
:10A360001E8219861886BE0183E492E1DF91CF91A7
:10A370000C94E44ECF93DF93EC018091421288233A
:10A3800031F0CE010296DF91CF910C94585083E4C6
:10A3900092E10E949F4E009739F08C179D0739F08B
:10A3A000FC0180819181F7CF81E090E002C080E0E4
:10A3B00090E0DF91CF9108952F923F924F925F925C
:10A3C0006F927F928F929F92AF92BF92CF92DF92C5
:10A3D000EF92FF920F931F93CF93DF93CDB7DEB72A
:10A3E000E8970FB6F894DEBF0FBECDBFECE6FAE2F9
:10A3F0002081318142815381E8E6FAE25080418038
:10A4000032802380E4E6FAE28081898391819A8315
:10A41000A281AB836380E0E6FAE2B081BC838181F4
:10A420008D8392819E83A381AF83ECE5FAE2B081B4
:10A43000B8878181898792819A87A381AB87E8E574
:10A44000FAE2B081BC8781818D8792819E87A3814A
:10A45000AF87E4E5FAE2B081B88B8181898B928184
:10A460009A8BA381AB8BE0E5FAE2B081BC8B818152
:10A470008D8B92819E8BA381AF8BECE4FAE2B0814D
:10A48000B88F8181898F92819A8FA381AB8FE8E405
:10A49000FAE2B081BC8F81818D8F92819E8FA381E2
:10A4A000AF8FE4E4FAE2B081B8A3818189A39281FD
:10A4B0009AA3A381ABA3E0E4FAE2B081BCA38181BB
:10A4C0008DA392819EA3A381AFA3ECE3FAE2B081B6
:10A4D000B8A7818189A792819AA7A381ABA7E8E356
:10A4E000FAE2B081BCA781818DA792819EA7A3814A
:10A4F000AFA7E4E3FAE2B081B8AB818189AB928186
:10A500009AAB7380E0E3FAE2B080A180928083800E
:10A51000ECE2FAE2F080E180D280C380E8E2FAE285
:10A52000A081AFABB181B8AF128103812BAB3CAB43
:10A530004DAB5EAB0E94725E5EA95F934DA94F93D7
:10A540003CA93F932BA92F932F923F924F925F925A
:10A550006F922B812F932A812F9329812F932F8103
:10A560002F932E812F932D812F932C812F932B8529
:10A570002F932A852F9329852F9328852F932F8515
:10A580002F932E852F932D852F932C852F932B89F9
:10A590002F932A892F9329892F9328892F932F89E5
:10A5A0002F932E892F932D892F932C892F932B8DC9
:10A5B0002F932A8D2F93298D2F93288D2F932F8DB5
:10A5C0002F932E8D2F932D8D2F932C8D2F932BA189
:10A5D0002F932AA12F9329A12F9328A12F932FA145
:10A5E0002F932EA12F932DA12F932CA12F932BA529
:10A5F0002F932AA52F9329A52F9328A52F932FA515
:10A600002F932EA52F932DA52F932CA52F937F92BB
:10A610002AA92F9329A92F9328A92F938F929F922C
:10A62000AF92BF92CF92DF92EF92FF920F931F9360
:10A6300028AD2F932FA92F939F938F937F936F9381
:10A64000A6E3B8E28C911F928F93E5E3F8E2808154
:10A650001F928F9382E59EE09F938F930E94FF8BC2
:10A66000ECE9FAE22081318142815381E8E9FAE2A2
:10A670005080418032802380ECE8FAE29080818033
:10A6800072806380E8E8FAE28081898391819A830D
:10A69000A281AB83B381BC83E4E8FAE280818D833D
:10A6A00091819E83A281AF83B381B887E0E8FAE20B
:10A6B0008081898791819A87A281AB87B381BC878A
:10A6C000ECE7FAE280818D8791819E87A281AF8736
:10A6D000B381B88BE8E7FAE28081898B91819A8B0C
:10A6E000B280A380E4E7FAE2F080E180D280C38008
:10A6F000E0E7FAE2A081AB8BB181BC8B12810381D0
:10A700000FB6F894DEBF0FBECDBF2BAB3CAB4DAB4D
:10A710005EAB0E94725E5EA95F934DA94F933CA908
:10A720003F932BA92F932F923F924F925F926F925C
:10A730007F928F929F922C812F932B812F932A812E
:10A740002F9329812F9328852F932F812F932E814B
:10A750002F932D812F932C852F932B852F932A8533
:10A760002F9329852F9328892F932F852F932E851B
:10A770002F932D852F93AF92BF922A892F932989EA
:10A780002F93CF92DF92EF92FF920F931F932C891A
:10A790002F932B892F939F938F937F936F93A6E390
:10A7A000B8E28C911F928F93E5E3F8E280811F92CB
:10A7B0008F9383EE9DE09F938F930E94FF8B0FB644
:10A7C000F894DEBF0FBECDBFE8960FB6F894DEBF9B
:10A7D0000FBECDBFDF91CF911F910F91FF90EF90F2
:10A7E000DF90CF90BF90AF909F908F907F906F90B1
:10A7F0005F904F903F902F90089580E38093F912DF
:10A800000895CF93DF936091F91270E0C0E3D0E038
:10A81000C61BD70B695B7D4EAE010E94528BCE01E9
:10A82000DF91CF910895CF92DF92EF92FF920F9335
:10A830001F93CF93DF937C01C090FC12D090FD1248
:10A840006091F91270E0E601E096C61BD70BC138A3
:10A85000D105D8F400E310E0061B170B695B7D4EB1
:10A86000A8010E94528B609145127091461280910E
:10A87000FA129091FB12680F791FA601C701800F91
:10A88000911F0E94528BCE0102C080E090E0DF91C8
:10A89000CF911F910F91FF90EF90DF90CF9008958F
:10A8A0009091F912980F9093F91208954091FC122B
:10A8B0005091FD124817590798F02091FA123091E3
:10A8C000FB12280F391F3093FB122093FA12481BFA
:10A8D000590B5093FD124093FC1281E090E00895D3
:10A8E00080E090E008959093FD128093FC1208950B
:10A8F0008091FA129091FB1289589D4E0895809193
:10A90000F91290E0895B9D4E089581E090E02091DE
:10A910004512309146122757324111F480E090E001
:10A9200008950E948554892B61F0609145127091C1
:10A9300046124091FC125091FD1287E792E10C946F
:10A94000528B2091FA123091FB1221153105B9F08A
:10A950008091FC129091FD12C096E7E7F2E1AF0101
:10A96000475452414817590734F4DF01A20FB31F6F
:10A970004C914193F4CF1092FB121092FA12089569
:10A98000809145129091461208958091FC12909109
:10A99000FD1208959091F91280E3891B089520E338
:10A9A0008091F912281B8091FC129091FD12820F68
:10A9B000911D08951F93CF93DF93EC011091F9122D
:10A9C000812F90E08C179D076CF00E94CF548C0F64
:10A9D0009D1F8138910530F41C1B1093F91281E002
:10A9E00090E002C080E090E0DF91CF911F91089548
:10A9F000CF93DF93EFE3F8E21192119288E2EF3602
:10AA0000F807D1F7C7E3D8E268EE72E0CE010E9402
:10AA10008B4B229688E2CF33D807B1F7DF91CF91E5
:10AA200008951092FB121092FA121092FD121092D9
:10AA3000FC1280E38093F91287E792E1909346122B
:10AA4000809345120C94F854EF92FF920F931F934A
:10AA5000CF93DF9300D0CDB7DEB78C0169837A83C3
:10AA60000E9411556981E62E7A81F72E81E8E81659
:10AA7000F10418F080E8E82EF12CA701B8018091CC
:10AA80004512909146120E94528BF092FD12E09274
:10AA9000FC12C7010F900F90DF91CF911F910F9182
:10AAA000FF90EF9008950F931F93CF93DF938C0146
:10AAB000EB010E9411551093461200934512D0935A
:10AAC000FD12C093FC12DF91CF911F910F91089559
:10AAD00020E3EFE3F8E2DC0101900D922A95E1F723
:10AAE00088E0E7E3F8E2DB0101900D928A95E1F757
:10AAF000089520E3FC01AFE3B8E201900D922A959E
:10AB0000E1F788E0FB01A7E3B8E201900D928A9596
:10AB1000E1F70895E82FF0E0EE0FFF1FE15CF74D3D
:10AB20007183608381E090E00895E82FF0E0EE0FFC
:10AB3000FF1FE15CF74D80819181089590E0880FBF
:10AB4000991F895F974D0E948B4B81E090E008959B
:10AB500090E0880F991F895F974D089581159105A1
:10AB600011F00197F1F70895E0917228F0917328A0
:10AB700090818091712889230895E0916F28F09148
:10AB80007028808190917128892B8083E0917428AE
:10AB9000F0917528808190917128892B8083089588
:10ABA000E0916F28F09170289081809171288095B4
:10ABB00089238083E0917428F09175289081809199
:10ABC000712880958923808308951F93CF93DF9305
:10ABD000E0916F28F0917028908180917128809584
:10ABE00089238083E0917428F09175288081909169
:10ABF0007128892B80838FEB93E00E94AE551FB79D
:10AC0000F894E0917428F0917528908180917128D2
:10AC100080958923808383E890E00E94AE55E0917F
:10AC20007228F0917328D081C09171281FBF789449
:10AC30008BE393E00E94AE55E0917228F091732867
:10AC4000908180917128982319F08D2F8C2301C059
:10AC500081E0DF91CF911F91089550937528409323
:10AC600074287093702860936F2890937328809352
:10AC7000722881E001C0880F2A95EAF78093712835
:10AC80000C94E555CF93DF93C82FDFB7F894E0918C
:10AC90007428F0917528808190917128892B808388
:10ACA00083E090E00E94AE55CC2351F0E0917428EF
:10ACB000F0917528808190917128909598239083C8
:10ACC00087E190E00E94AE55E0917228F0917328E0
:10ACD000808190917128892309F4C0E089E590E092
:10ACE0000E94AE55E0917428F09175288081909172
:10ACF0007128909598239083DFBF8BE390E00E94AA
:10AD0000AE558C2FDF91CF910895CF93DF93C82F4D
:10AD1000D8E08C2F81700E944256C6958111C06880
:10AD2000D150B9F78C2FDF91CF9108958FEF0C940C
:10AD30008556DF92EF92FF920F931F93CF93DF938D
:10AD4000E82EEB010E94E55581112FC080EF0E9493
:10AD50008556F12C10E488EFD82ED10E81E00E94A8
:10AD60004256082F81E00E944256882319F00023A2
:10AD700061F01DC0011109C01E1528F0888180FFF7
:10AD800004C0E11611F0F12E01E0802F0E9442561E
:10AD90009881969501119068988311501D11DECF0E
:10ADA00021961111D8CF8F2D03C08FEF01C08EEFE8
:10ADB000DF91CF911F910F91FF90EF90DF90089559
:10ADC000FF920F931F93CF93DF93F82EEB010E9416
:10ADD000E555209769F085E50E9485568E01085F4C
:10ADE0001F4F89910E948556C017D107D1F703C024
:10ADF0008CEC0E9485568F2DDF91CF911F910F9182
:10AE0000FF900C9485560F931F93CF93DF93DB0134
:10AE1000EC9111969C911197F0E0F92B803181F41F
:10AE2000BF016E7FE3E0660F771FEA95E1F71696A4
:10AE30009C911697ECE0F0E0E91BF109E60FF71F93
:10AE4000F7FF07C091E0EA019883F195E195F109D8
:10AE500002C0EA011882883279F414968C91982FF6
:10AE60009076903649F086FF02C0EE7F05C085FFE0
:10AE700002C0EC7F01C0E87FCF0144E09695879542
:10AE80004A95E1F7D9018C93EF70E801E88380E0FF
:10AE9000DF91CF911F910F9108950F931F93CF933F
:10AEA000DF93EC018B01B80188810E949956888359
:10AEB00081508D3F30F4F8018081883211F080316B
:10AEC00091F7DF91CF911F910F910895CF93DF9369
:10AED000EC010E94E555BE0184EB0E94E05681E042
:10AEE0000E944256C82F0E94E55581E0C11101C061
:10AEF00080E0DF91CF9108951F93CF93DF9300D02F
:10AF0000CDB7DEB7182F69837A830E94E5550E947A
:10AF1000B45569817A81882341F084E40E94E05627
:10AF2000113029F00E94BD5502C082E001C080E0CE
:10AF30000F900F90DF91CF911F9108954F925F92E4
:10AF40006F927F928F929F92AF92BF92CF92DF9239
:10AF5000EF92FF920F931F93CF93DF93CDB7DEB79E
:10AF600029970FB6F894DEBF0FBECDBF6C015B0111
:10AF70004A0189010E94E555B6018EEB0E94E05618
:10AF8000CE0101967C013E019AE0690E711C2701F9
:10AF90000E949656F70181937F01E615F705C1F7E8
:10AFA00069E070E0C2010E942C71811109C0940116
:10AFB000A501B201F60180810E94035780E001C023
:10AFC00083E029960FB6F894DEBF0FBECDBFDF91A8
:10AFD000CF911F910F91FF90EF90DF90CF90BF9096
:10AFE000AF909F908F907F906F905F904F9008955B
:10AFF0005F926F927F928F929F92AF92BF92CF9209
:10B00000DF92EF92FF920F931F93CF93DF93CDB711
:10B01000DEB729970FB6F894DEBF0FBECDBF582E0E
:10B020006B015A01890160E070E08EEB0E94E056EE
:10B03000CE0101967C014E019AE0890E911C3701E8
:10B040000E949656F70181937F01E815F905C1F733
:10B0500069E070E0C3010E942C71811108C0950164
:10B06000A601B301852D0E94035780E001C083E053
:10B0700029960FB6F894DEBF0FBECDBFDF91CF91FA
:10B080001F910F91FF90EF90DF90CF90BF90AF9006
:10B090009F908F907F906F905F9008950F931F9374
:10B0A000CF93DF93CDB7DEB728970FB6F894DEBF06
:10B0B0000FBECDBF182F062F98E0E4EFF2E0DE01BF
:10B0C000119601900D929A95E1F7242F332727FDD1
:10B0D000309541E752E0249FC001259F900D349F99
:10B0E000900D112464E670E00E946D85CB0144E66A
:10B0F000049F800D911D1124FE013196AE01475F22
:10B100005F4F619170E02617370711F4019603C075
:10B11000E417F507B1F7112319F09195819591097D
:10B1200028960FB6F894DEBF0FBECDBFDF91CF914A
:10B130001F910F910895EF92FF920F931F93CF935A
:10B14000DF93CDB7DEB72B970FB6F894DEBF0FBEF7
:10B15000CDBFF82EE92E682F792F88E08F0D0E9441
:10B160007C57882319F084E391E243C066E471E4DC
:10B170008FE090E00E9406598E01075F1F4F9801F3
:10B18000AE01465F5F4FBE01655F7F4F8F2D9E2DE5
:10B190000E949E578111E7CF88E0E4EFF2E0DE01E4
:10B1A000119601900D928A95E1F7498521E732E0E9
:10B1B000429FC001439F900D112464E670E00E94FD
:10B1C0006D858A8594E6899F600D711D1124FE01AD
:10B1D00031968191481303C06F5F7F4F03C0E01722
:10B1E000F107B9F78B85882319F07195619571097D
:10B1F000CB012B960FB6F894DEBF0FBECDBFDF910B
:10B20000CF911F910F91FF90EF900895DC01CB013A
:10B2100081159105A105B10529F081509040A0400C
:10B22000B040D9F708951092B90080E28093B80039
:10B23000089594EA9093BC0040EA56E861E070E01B
:10B240009091BC0097FD0BC04150510961097109F3
:10B25000411551056105710599F781E008959091B7
:10B26000B900987F983011F09031B9F78093BB0006
:10B2700084E88093BC0080EA96E8A1E0B0E02091E9
:10B28000BC0027FD08C00197A109B1090097A105DD
:10B29000B105A9F7E2CF8091B900887F883111F01C
:10B2A0008034D9F680E0089524EA34E844E9209314
:10B2B000BC009091BC0097FFFCCF9091B900987FA3
:10B2C000983011F0903199F78093BB003093BC0017
:10B2D0009091BC0097FFFCCF9091B900987F90327D
:10B2E00011F0983539F44093BC009091BC0094FD66
:10B2F000FCCFDDCF08950C94195984E98093BC00EC
:10B300008091BC0084FDFCCF08958093BB0084E84D
:10B310008093BC008091BC0087FFFCCF9091B90066
:10B32000987F81E0983209F480E0089584EC80935E
:10B33000BC008091BC0087FFFCCF8091BB000895CA
:10B3400084E88093BC008091BC0087FFFCCF809193
:10B35000BB000895E0E1DC01FD91CD01F0933F01D8
:10B36000E150C9F780913C018F7D80933C01809131
:10B370003C01877F80933C01FB0180E19191909398
:10B380003E018150D9F780913C01806880933C0157
:10B3900080913D0180FFFCCF4051510980913C01DB
:10B3A000806280933C0180913C01877F80933C01C7
:10B3B000141615069CF4FB0180E1919190933E01D7
:10B3C0008150D9F780913C01806880933C01809145
:10B3D0003D0180FFFCCF40515109EACFF90180E1E6
:10B3E00090913E0191938150D9F781E090E00895CA
:10B3F0000F931F93CF93DF93EC018CE70E94545976
:10B400008CE70E9485598E01005F1F4F89910E9431
:10B410008559C017D107D1F7DF91CF911F910F91B7
:10B420000C947D59813019F440E050E002C040ECAA
:10B4300050E060E070E08CE790E00C94DF10813029
:10B4400019F44EE050E002C048E050E060E070E0E7
:10B450008CE790E00C94DF1041E050E060E070E099
:10B460008CE790E00E94DF106AE67AE080E090E0EE
:10B470000C94065948E350E060E070E08CE790E0FF
:10B480000E94DF1049E350E060E070E08CE790E05C
:10B490000E94DF1044E150E060E070E08CE790E053
:10B4A0000E94DF1048E750E060E070E08CE790E039
:10B4B0000E94DF104EE550E060E070E08CE790E025
:10B4C0000E94DF104DE650E060E070E08CE790E015
:10B4D0000E94DF106CE17AE186E090E00E9406595C
:10B4E0004CE050E060E070E08CE790E00E94DF10FC
:10B4F00041E050E060E070E08CE790E00E94DF10F7
:10B5000046E050E060E070E08CE790E00E94DF10E1
:10B510006AE67AE080E090E00C940659CF93DF93DE
:10B52000CDB7DEB7A2970FB6F894DEBF0FBECDBF82
:10B5300081E1EDECF8E0DE01529601900D928A95E2
:10B54000E1F781E1EEEDF8E0DE01119601900D9258
:10B550008A95E1F70E943A5ACE0142960E94F85924
:10B5600082E00E94125A6AE67AE080E090E00E944F
:10B570000659CE0101960E94F85960E17EEA88E200
:10B5800090E00E94065980E00E941F5A60E17EEA26
:10B5900088E290E00E9406594EE050E060E070E0E2
:10B5A0008CE790E00E94DF10A2960FB6F894DEBF01
:10B5B0000FBECDBFDF91CF910895CF92DF92EF9272
:10B5C000FF920F931F93CF93DF9300D01F92CDB7BD
:10B5D000DEB7F82E042F122F213031F0223031F057
:10B5E000243031F0283031F090E005C091E003C004
:10B5F00092E001C093E00C3059F00E3011F49460E9
:10B6000007C0003111F4986003C0023109F49C6056
:10B61000613059F0623011F4906207C0633011F468
:10B62000906403C0643009F490669068692F70E0FC
:10B6300023E030E0AE014F5F5F4F8F2D90E00E941E
:10B64000F61069E07AE180E090E00E9406598F2DC3
:10B650008160F82E0E9419590E94965989830E9490
:10B6600096598A83023119F40E9496598B830E945D
:10B67000965987FDF1CF0E94A0590E947D5969E03B
:10B680007AE180E090E00E9406598F2D0E941959BE
:10B690000E94965989830E9496598A83023119F42F
:10B6A0000E94A0598B830E94A0590E947D59398124
:10B6B0002A81023149F5832F90E0A0E0B0E04B8170
:10B6C0007727662731FF0EC030E0322F2227620F26
:10B6D000731F811D911D640F711D811D911D8C6F44
:10B6E0009F6F0BC030E0322F2227620F731F811D26
:10B6F000911D640F711D811D911D0E947A8220E8A9
:10B700003FEF4FEF57E420C0632F70E0762F66279E
:10B71000620F711D882777FD8095982F0E947A828D
:10B720000C3029F420E030EE4FEF54E40DC00E3021
:10B7300029F420E038EF4FEF55E406C0003131F432
:10B7400020E03EEF4FEF56E40E94DB812FE632E12E
:10B7500043E050E40E9458846B017C01612F70E04B
:10B7600080E090E00E947A829B01AC01C701B601A3
:10B770000E94DB810F900F900F90DF91CF911F916E
:10B780000F91FF90EF90DF90CF900895E6E4F1E005
:10B790008081208190813081829586958695837005
:10B7A00022952F70822B832B92959F70892B089561
:10B7B0000F931F93CF93DF9300D0CDB7DEB746E052
:10B7C0006CE080E00E94085F89E18093C4001092E1
:10B7D000C50082E08093C00080E00E94935F0E94D9
:10B7E000345E84B784B784B784B784B7E6EFF0E3F8
:10B7F00022E432E4318320833A968DB79EB70A97CC
:10B80000E817F907B8F38FEE98E09F938F938FE9CD
:10B810009FE09F938F930E94FF8B0E946F6D0E9409
:10B82000374D60E070E082E792E00E94DF4D0E94B9
:10B830001351E091FC02F091FD0209950E94C65B54
:10B8400090E00E94AB6DCE0101960E94695D0F9061
:10B850000F900F900F90882341F08FE79FE09F9308
:10B860008F930E94FF8B0F900F90CE0101960E9444
:10B87000A64B0E94775D8C010E94735DAE014F5F05
:10B880005F4FB8010E945F620E94E35C0E944062C9
:10B890000E947B5D0E94996382E79FE09F938F9354
:10B8A0000E94FF8B8A811F928F930EE61FE01F93E9
:10B8B0000F930E94FF8B89811F928F931F930F9389
:10B8C0000E94FF8B8CE69FE09F938F930E94FF8BDB
:10B8D0000E94AF6DE0913903F0913A030995E09130
:10B8E0002B03F0912C030995E0911203F0911303BF
:10B8F00009950E94A063182F0E943D621F921F931A
:10B900001F928F93809138038F93809137038F9389
:10B9100080912A038F93809129038F9381E59FE083
:10B920009F938F930E94FF8BE0914303F091440318
:10B930000FB6F894DEBF0FBECDBF309791F00995DA
:10B94000BC0180E890E00E9459857F936F938EE35D
:10B950009FE09F938F930E94FF8B0F900F900F900B
:10B960000F908CE39FE09F938F930E94FF8B60E08A
:10B9700070E088EC92E00E94DF4D8AED92E00E9438
:10B980007F6C84E39FE09F938F930E94FF8B0F90C7
:10B990000F900F900F900F900F90DF91CF911F910C
:10B9A0000F9108957F936F939F938F938EE29FE003
:10B9B0009F938F930E94FF8B0F900F900F900F908B
:10B9C0000F900F9008951F93CF93DF93CDB7DEB7FD
:10B9D000A0970FB6F894DEBF0FBECDBF83E590E011
:10B9E0000E943C8D182F282F35EF380F303108F08A
:10B9F000982F9095291709F461C08AEB9FE09F93D7
:10BA00008F930E94FF8BEFEFFFE00F900F90DE010E
:10BA1000119684918D93319680E1E730F807C9F74C
:10BA2000F89448E050E06FE670E0CE0101960E9485
:10BA3000428DE1EFFFE0DE01119684918D93319606
:10BA40008FE0EF3FF807C9F74EE050E061E670E0A5
:10BA5000CE0101960E94428DE7EEFFE0DE011196D5
:10BA600084918D9331968FE0E13FF807C9F74AE062
:10BA700050E067E570E0CE0101960E94428D6DECCA
:10BA80007BEA81E590E00E945A8D60E070E08FE4EF
:10BA900090E00E945A8D60E08EE490E00E944C8D10
:10BAA00060E070E085E590E00E945A8D1AE16AE15D
:10BAB00075EE83E590E00E945A8D7894812FA096D0
:10BAC0000FB6F894DEBF0FBECDBFDF91CF911F91AF
:10BAD0000895F89442E050E06FE670E00E94248DF3
:10BAE000789480E0089581E590E00C943C8D8FE49B
:10BAF00090E00C943C8D8EE490E00C94348D409159
:10BB0000842850918528609186287091872890E03C
:10BB1000A0E0B0E0480F591F6A1F7B1F40938428A4
:10BB200050938528609386287093872840918028B9
:10BB3000509181286091822870918328480F591F65
:10BB40006A1F7B1F4093802850938128609382282E
:10BB5000709383282091242A2223A1F040917C28ED
:10BB600050917D2860917E2870917F28480F591F41
:10BB70006A1F7B1F40937C2850937D2860937E280A
:10BB800070937F2808951F920F920FB60F92112481
:10BB90000BB60F922F933F934F935F936F937F93C7
:10BBA0008F939F93AF93BF93EF93FF938091001375
:10BBB000909101130196909301138093001380914B
:10BBC000FF128F5F8093FF128038A9F41092FF124A
:10BBD0008091842890918528A0918628B09187280B
:10BBE0000196A11DB11D8093842890938528A09370
:10BBF0008628B09387288091242A8823E1F08091B9
:10BC0000FE128F5F8093FE128038A9F41092FE120C
:10BC100080917C2890917D28A0917E28B0917F28EA
:10BC20000196A11DB11D80937C2890937D28A0933F
:10BC30007E28B0937F280E946F50892B11F00E94BC
:10BC4000824FFF91EF91BF91AF919F918F917F9123
:10BC50006F915F914F913F912F910F900BBE0F907D
:10BC60000FBE0F901F901895F8941092B60016BC56
:10BC700083EF87BD82E084BD94E095BD95B395BB0D
:10BC800080936E0078940895809100139091011331
:10BC9000209100133091011382179307A9F708959B
:10BCA000009751F022E330E00000215031092115C6
:10BCB0003105D1F70197F4CF08950F931F93CF93D8
:10BCC000DF93EC010E94445E8C010E94445E801B65
:10BCD000910B8C179D07C8F3DF91CF911F910F91A6
:10BCE000089508950F931F9360918428709185287B
:10BCF000809186289091872800918428109185282A
:10BD00002091862830918728601771078207930752
:10BD100059F71F910F9108951F920F920FB60F922E
:10BD2000112410929E020F900FBE0F901F90189535
:10BD30001F920F920FB60F9211240BB60F922F93F2
:10BD40003F934F935F936F937F938F939F93AF93A3
:10BD5000BF93EF93FF93E0919402F091950280815D
:10BD6000E0919F02F091A002309709F00995FF91B0
:10BD7000EF91BF91AF919F918F917F916F915F9163
:10BD80004F913F912F910F900BBE0F900FBE0F90D0
:10BD90001F9018951F920F920FB60F9211241092B8
:10BDA000AB020F900FBE0F901F9018951F920F922D
:10BDB0000FB60F9211240BB60F922F933F934F9310
:10BDC0005F936F937F938F939F93AF93BF93EF9303
:10BDD000FF93E091A102F091A2028081E091AC0278
:10BDE000F091AD02309709F00995FF91EF91BF9165
:10BDF000AF919F918F917F916F915F914F913F9103
:10BE00002F910F900BBE0F900FBE0F901F901895A3
:10BE10009DE0899FF0011124EC56FD4FA281B38172
:10BE20001C92A481B5816C93A681B78188ED8C9317
:10BE3000A085B1854C9312861486138608959DE0E3
:10BE4000899FF0011124EC56FD4F81E08287A0818B
:10BE5000B1816C933A9680818111FDCF08951F9333
:10BE6000CF93DF93182FEB01FE016491662329F035
:10BE7000812F0E941F5F2196F7CFDF91CF911F91F5
:10BE800008951F93CF93DF93182FEB0188818823A8
:10BE900069F08A3021F46DE0812F0E941F5F699163
:10BEA0006D30A1F3812F0E941F5FF0CFDF91CF9102
:10BEB0001F910895CF93DF93CDB7DEB79E01285F22
:10BEC0003F4F4E815F8160E470E082E093E10E9429
:10BED0008D8C62E073E18D810E94415FDF91CF9193
:10BEE0000895CF93C82F8A3031F46DE080914213CA
:10BEF0000E941F5F02C08D3029F06C2F8091421389
:10BF00000E941F5F80E090E0CF9108959DE0899F9F
:10BF1000F0011124EC56FD4F748763870895682F54
:10BF200080E00C941F5F8093421386E892E0909328
:10BF3000F1308093F030089584B7877F84BF88E123
:10BF40000FB6F89480936000109260000FBE0895C1
:10BF50002FE088E190E00FB6F894A89580936000F8
:10BF60000FBE209360000895A895089588E10FB64C
:10BF7000F89480936000109260000FBE0895F894CA
:10BF800028E088E190E00FB6F894A89580936000CF
:10BF90000FBE20936000FFCF80918F2880918F2863
:10BFA00090E0089540E06FE181E491E00C94356504
:10BFB000E9E3F1E0808180818D7F80838DE090E0F6
:10BFC0000197F1F723E040E06FE182E491E00E9405
:10BFD0003F6583E090E00197F1F708959091390172
:10BFE00091FD0AC0282F803108F02FE040E06FE07B
:10BFF00085E491E00C943F6508958091390181FDBD
:10C000000EC040E06FE181E491E00E943565282F89
:10C010002F7E81E090E0213021F080E0089580E0E3
:10C0200090E008958091390181FD10C040E06FE1FA
:10C0300081E491E00E9435658F3131F0982F9F7E29
:10C04000915081E0923018F480E0089581E00895E5
:10C050000E9412608823E1F30895CF93DF93C82FE5
:10C060000E9428600E94D25FD82FC81789F1C8307B
:10C0700019F40E94D85F25C0C93121F4863189F4B2
:10C0800029E005C0C63169F4893159F426E040E061
:10C090006FE182E491E00E943F65E3E0F0E03197D8
:10C0A000F1F72C2F40E06FE182E491E00E943F65C0
:10C0B000D83019F4E9E6F1E002C0E3E0F0E03197AE
:10C0C000F1F70E94D25F8C1719F083E490E002C070
:10C0D00080E490E0DF91CF9108950E942860109253
:10C0E000242A0E94D85F80913901826080933901AF
:10C0F0008091A72A8823D9F180919400909195008E
:10C100004091B82A5091B92A84179507A0F48091DC
:10C11000842A9091852AA091862AB091872A8C57EB
:10C12000914EAF4FBF4F8093842A9093852AA0935E
:10C13000862AB093872A2091940030919500241B81
:10C14000350B8091842A9091852AA091862AB091FE
:10C15000872A820F931FA11DB11D8093842A90937B
:10C16000852AA093862AB093872A1092A72A8091C5
:10C17000A92A8823D9F1809194009091950040914B
:10C18000BC2A5091BD2A84179507A0F480918C2A6F
:10C1900090918D2AA0918E2AB0918F2A8C57914E22
:10C1A000AF4FBF4F80938C2A90938D2AA0938E2AF5
:10C1B000B0938F2A2091940030919500241B350B69
:10C1C00080918C2A90918D2AA0918E2AB0918F2AED
:10C1D000820F931FA11DB11D80938C2A90938D2AED
:10C1E000A0938E2AB0938F2A1092A92A0895809145
:10C1F000242A882381F08091C613811104C00E94F3
:10C200001260811106C081E08093C41381E090E048
:10C2100008950E946D6080E090E008958091940000
:10C22000909195009093BD2A8093BC2A21E02093A1
:10C23000A92A8091390181FD08C08091390181FDD1
:10C240001AC086E10E942D6016C02093232A809197
:10C250009400909195009093B92A8093B82A2093E6
:10C26000A72A809139018D7F809339018091232AFB
:10C270008111FCCFE2CF81E08093242A0895809140
:10C28000242A81110AC08091C613882321F081E0FD
:10C290008093C51302C00E940E6181E090E0089572
:10C2A0001F93CF93DF931F92CDB7DEB78FB78983EC
:10C2B0008091C613811126C0F8948091242A882386
:10C2C00051F08091390181FD1BC00E9412608823CA
:10C2D000B9F080E003C00E943F6181E020914701F6
:10C2E00091E02E3008F090E0192F119581110E94F5
:10C2F000F760107429F089818FBF81E090E004C05D
:10C3000089818FBF80E090E00F90DF91CF911F91E6
:10C3100008958091C513882321F00E940E61109228
:10C32000C5138091C413882321F00E946D60109280
:10C33000C4131092C61308950F931F93AB0121E00D
:10C340002093C6130091682A1091692A20916A2AC5
:10C3500030916B2A0F5F1F4F2F4F3F4F0093682A7A
:10C360001093692A20936A2A30936B2A22E0260FC1
:10C3700027FF0CC08091212A9091222A0196909348
:10C38000222A8093212A0FEF1FEF07C0BC0183E40C
:10C3900093E10E94528B00E010E00E948961C80185
:10C3A0001F910F9108958093C81308950E94D25F42
:10C3B000823011F0823111F480E0089581E0089517
:10C3C00008958FEF80934E0122E044E060EF8CE609
:10C3D00091E00E943F6525E041E06EE08CE290E054
:10C3E0000E943F6580E880936F01809146018093B1
:10C3F0006D0121E045E060E284E491E00C943F654A
:10C400008DEF93E00197F1F70E942B651092982829
:10C4100010921A2910929C2910929728109296280F
:10C42000E9E3F1E080818E7F808380818D7F80834E
:10C430008DE090E00197F1F7E9E3F1E08081816020
:10C44000808323E040E06FE182E491E00E943F6559
:10C450008DEF93E00197F1F780915D0180915E018E
:10C460000E94E16160E070E08EEA92E00E94DF4DA0
:10C470000E940E6181E090E008958091C7130895B5
:10C48000CF93DF931F92CDB7DEB789830E942860D8
:10C4900089818093C713282F40E06FE188E491E001
:10C4A0000F90DF91CF910C943F650E944062809184
:10C4B000390181FD03C086E00C942D600895FA01D6
:10C4C00080936201909363016093600170936101B6
:10C4D0003097C1F0808180936B01818180936A01E4
:10C4E0008281809369018381809368018481809334
:10C4F00067018581809366018681809365018781CC
:10C500008093640108958EEA92E00E94004E81E0DB
:10C5100080938F28809190289091912801969093F4
:10C5200091288093902881E090E008958091972849
:10C5300092E8899FF0011124E856F74D10828F5F31
:10C54000833018F48093972802C010929728E091C6
:10C55000972882E8E89FF0011124E856F74D808182
:10C5600081110C94836210928F2808951F93CF93AA
:10C57000DF932091972812E8129F90011124D9018E
:10C58000A856B74D4C91411103C00E94966293C0CA
:10C590005091390151FD8FC05091242A552309F43F
:10C5A0008AC047FF16C00E9496628091582A9091D7
:10C5B000592AA0915A2AB0915B2A0196A11DB11D5A
:10C5C0008093582A9093592AA0935A2AB0935B2AB1
:10C5D00072C04330B0F40E9496628091542A9091C8
:10C5E000552AA091562AB091572A0196A11DB11D36
:10C5F0008093542A9093552AA093562AB093572A91
:10C600005AC050E0EA0122976C177D07B0F40E94EF
:10C6100096628091502A9091512AA091522AB0910D
:10C62000532A0196A11DB11D8093502A9093512A3F
:10C63000A093522AB093532A3EC0B9016756774D52
:10C640000E94528BE09197281E9FF0011124E85E12
:10C65000F64D8081809388280E94966280914701E0
:10C660008093892890918E28992311F0891710F4CE
:10C6700080938E286091892870E084E00E948A551A
:10C680006091882870E083E00E948A5540916C2A6E
:10C6900050916D2A60916E2A70916F2A4F5F5F4FA3
:10C6A0006F4F7F4F40936C2A50936D2A60936E2A90
:10C6B00070936F2A02C0C0E0D0E0CE01DF91CF912D
:10C6C0001F910895CF93DF93EC01888199810097A2
:10C6D000E9F08730954021F01982188283E026C066
:10C6E0006238C1F410928F280E9411550E9478542C
:10C6F00060E870E00E94B662181619066CF40E9499
:10C700007354E0913D03F0913E03099587E095E075
:10C710009983888381E00AC080918C2890918D282C
:10C72000019690938D2880938C28F0CFDF91CF9144
:10C73000089591E09093C6130E94EE5F0C94896176
:10C740008091390181FD06C040E06FE085E491E011
:10C750000C94356580E108950F931F93CF93DF9379
:10C76000182F21E02093C6130091242A80913901CB
:10C7700081FF16C080919400909195009093B92A02
:10C780008093B82A2093A72A2093232A80913901E5
:10C790008D7F809339018091232A8111FCCF00E0A5
:10C7A0000E9428608091242A882309F43FC0809148
:10C7B000A92A8823D9F18091940090919500E09165
:10C7C000BC2AF091BD2A8E179F07A0F440918C2AB5
:10C7D00050918D2A60918E2A70918F2A4C57514E1C
:10C7E0006F4F7F4F40938C2A50938D2A60938E2AEF
:10C7F00070938F2A20919400309195002E1B3F0B4F
:10C8000040918C2A50918D2A60918E2A70918F2AA6
:10C81000420F531F611D711D40938C2A50938D2A26
:10C8200060938E2A70938F2A1092A92A80913901E1
:10C8300081FD03C089E10E942D6086E00E9495552C
:10C84000892B51F00E94A063C82F86E00E94955565
:10C8500081500E94EE5F02C0C0E0D0E020919400C1
:10C86000309195003093BB2A2093BA2A81E08093BF
:10C87000A82AF894809139018260809339018091CF
:10C8800039018D7F8093390162E0610F83E493E188
:10C890000E947065789420911E2A30911F2A2F5F84
:10C8A0003F4F30931F2A20931E2A0E94286045E0A4
:10C8B00060EE82E491E00E943565182F86E00E94C8
:10C8C0009555892B19F08C2F0E94EE5F002319F0EB
:10C8D0000E940E6102C00E946D608091A82A882388
:10C8E000D9F18091940090919500E091BA2AF0914D
:10C8F000BB2A8E179F07A0F44091882A5091892A5D
:10C9000060918A2A70918B2A4C57514E6F4F7F4FFE
:10C910004093882A5093892A60938A2A70938B2A9D
:10C9200020919400309195002E1B3F0B4091882A56
:10C930005091892A60918A2A70918B2A420F531F45
:10C94000611D711D4093882A5093892A60938A2A19
:10C9500070938B2A1092A82A8091242A882361F050
:10C9600020919400309195003093BD2A2093BC2AE9
:10C9700081E08093A92A07C023E040E06FE182E4D0
:10C9800091E00E943F650E9489611130E9F0133007
:10C99000A9F48091602A9091612AA091622AB091B5
:10C9A000632A0196A11DB11D8093602A9093612A8C
:10C9B000A093622AB093632A12E009C0153031F0C7
:10C9C000173029F411E003C010E001C013E0812FFB
:10C9D00090E0DF91CF911F910F910895CF93DF9356
:10C9E000EB010E949C61009729F4CE010E94AC6388
:10C9F000009751F02091212A3091222A2F5F3F4F3A
:10CA00003093222A2093212ADF91CF910895CF934A
:10CA1000DF938091242A811104C00E943F61D1E0FC
:10CA200001C0D0E00E94D25F863111F0813119F44B
:10CA3000C091470109C040E06FE186E491E00E94A7
:10CA40003565C82FCC0FC80FD1110E94F7608C2F0D
:10CA5000DF91CF9108951092CA131092C913EFE697
:10CA6000F0E08081806280830895FC0180818623CC
:10CA700090E002C0959587954A95E2F70895F8945D
:10CA8000FC015081362F30955323042E01C0220F14
:10CA90000A94EAF72623522B508378940895409104
:10CAA0007B01FC014193A0E8B1E050E8540F9D01E7
:10CAB0002F5F3F4F6C916193521711F0D901F7CF5F
:10CAC0004150E42FF0E0E058FE4F2181FC01E05896
:10CAD000FF4F2083FC01EF57FF4F21E02083089593
:10CAE00060938001E1E8F1E061589F012F5F3F4FC3
:10CAF000DC014D91CD014083621711F0F901F5CFB2
:10CB000008951F920F920FB60F9211240BB60F9239
:10CB10002F933F934F935F936F937F938F939F9345
:10CB2000AF93BF93EF93FF93809147018093892840
:10CB30008091962822E8829FC00111248856974D43
:10CB40000E944F65809196288F5F833018F4809300
:10CB5000962802C0109296280E948362FF91EF915E
:10CB6000BF91AF919F918F917F916F915F914F9105
:10CB70003F912F910F900BBE0F900FBE0F901F9003
:10CB800018951F920F920FB60F9211240F900FBE9F
:10CB90000F901F9018951F920F920FB60F921124AD
:10CBA0000F900FBE0F901F9018951F920F920FB607
:10CBB0000F9211240F900FBE0F901F9018951F9287
:10CBC0000F920FB60F9211241092232A0F900FBECE
:10CBD0000F901F9018951F920F920FB60F9211246D
:10CBE0001092232A0F900FBE0F901F9018951F923E
:10CBF0000F920FB60F9211248F9381E080938F28AC
:10CC00008F910F900FBE0F901F9018951F920F924B
:10CC10000FB60F9211241092232A0F900FBE0F907F
:10CC20001F9018951F920F920FB60F9211248F9399
:10CC30009F938091C9139091CA1301969093CA1340
:10CC40008093C9139F918F910F900FBE0F901F90EB
:10CC50001895CF92DF92EF92FF920F931F93CF938D
:10CC6000DF937C018B016A018BEC93E10E949F4E64
:10CC7000EC01009751F0EC81FD81309711F0C80173
:10CC80000995CE010E94474FF3CFA601B801C70115
:10CC9000DF91CF911F910F91FF90EF90DF90CF9098
:10CCA0000C94294C0F931F93CF93DF9300D0CDB7F3
:10CCB000DEB780912C2A90912D2AA0912E2AB09136
:10CCC0002F2A0196A11DB11D80932C2A90932D2A05
:10CCD000A0932E2AB0932F2A0E94BC688C018BEC63
:10CCE00093E10E949F4E009779F0DC011296ED913E
:10CCF000FC911397309729F089839A8309959A813B
:10CD000089810E94474FEFCF0115110549F0C801F5
:10CD10000F900F90DF91CF911F910F910C94204CA9
:10CD20000F900F90DF91CF911F910F9108950E9466
:10CD3000AF6D0E9411550E94E36689E293E09093E3
:10CD4000272A8093262A0E94BA682FEF31E040E01C
:10CD50005EE160E074E082E090E00C948368BC01E6
:10CD60008BEC93E10C94FF4EBC018BEC93E10C94A3
:10CD7000E44ECF93DF93EC014091282A5091292A69
:10CD800060912A2A70912B2A4F5F5F4F6F4F7F4F20
:10CD90004093282A5093292A60932A2A70932B2A99
:10CDA0000E94CF68009761F00E949154E0912D039A
:10CDB000F0912E03BE0189E296E6099581E090E0AC
:10CDC000DF91CF91089581ED93E10C949B4E0F93E9
:10CDD000CF93DF93EC017B836A8318865F834E8356
:10CDE000BC0181ED93E10E94FF4EE091CD13F091E3
:10CDF000CE13309749F04C815D8101E020E030E0B6
:10CE000068858A819B810995DF91CF910F91089563
:10CE1000BC0181ED93E10C94E44E0F93DC01189674
:10CE20001C921897E091CD13F091CE13309759F0E2
:10CE300000E020E030E040E050E060E012968D91AC
:10CE40009C91139709950F9108950F93DC01AB0105
:10CE500014962D913C91159781E018968C93189714
:10CE600015967C936E931497E091CD13F091CE13A9
:10CE7000309739F000E061E012968D919C91139704
:10CE800009950F9108950F93DC01E091CD13F09176
:10CE9000CE13309771F014964D915C91159701E087
:10CEA0009A0118966C91189712968D919C911397F0
:10CEB00009950F910895E091CF13F091D013309719
:10CEC00009F0099408959093D0138093CF13089597
:10CED0009093CE138093CD13089581ED93E10C943C
:10CEE0009F4EEF92FF920F931F93CF93DF938C018E
:10CEF000EB017A0181ED93E10E949F4E0097D9F0FA
:10CF0000DC0112962D913C9113972C173D0781F46B
:10CF10001696ED91FC911797309769F09701AE0145
:10CF2000B801DF91CF911F910F91FF90EF9009947D
:10CF30000E94474FE3CFDF91CF911F910F91FF9058
:10CF4000EF9008950895CF93DF93C4E0D4E1688112
:10CF5000798120E030E042EC57E68EEE93E10E94CA
:10CF60001F510E94AD6D688179810E94598520E032
:10CF700030E046ED57E6BC018EED93E1DF91CF91B5
:10CF80000C941F5180910414909105142091021467
:10CF900030910314880F991F2817390708F4C90125
:10CFA00090930514809304140C94A367CF93DF939C
:10CFB0000E9411550E947854EC01198218820E9437
:10CFC0006D6728813981009719F1FC014085442360
:10CFD000F9F0FC0142815381F901EE0FFF1FEE0FC2
:10CFE000FF1FEC0FFD1F53834283FC0144815581D9
:10CFF0002F5F3F4FF901EE0FFF1FEE0FFF1FEC0FEA
:10D00000FD1F51834083398328830E94474FD9CF26
:10D01000C901880F991F880F991F02960E947354A7
:10D0200088819981892B31F083ED93E1DF91CF9154
:10D030000C94F74BDF91CF910895AF92BF92CF92AE
:10D04000DF92EF92FF920F931F93CF93DF9300D065
:10D05000CDB7DEB76B010E947854FC0100811181CD
:10D060001A8309830C30110518F4E12CF12C0DC042
:10D070001F930F938DE099E09F938F930E94ED8B08
:10D080000F900F900F900F9021C0E016F106F1F075
:10D090000E947854F701EE0FFF1FEE0FFF1FE80FFD
:10D0A000F91FA280B3800E947854FFEFEF1AFF0AA5
:10D0B000F701EE0FFF1FEE0FFF1FE80FF91F408172
:10D0C0005181B501C6010E947167DFCF0F900F90AB
:10D0D000DF91CF911F910F91FF90EF90DF90CF9054
:10D0E000BF90AF9008950F93013059F48091FE13D3
:10D0F0009091FF1390930514809304140F910C9456
:10D10000A3670F910895EF92FF920F931F93CF9310
:10D11000DF938B01EA01790146E153E0BC0183ED25
:10D1200093E10E94DB4B1093FF130093FE13D09307
:10D130000114C0930014F0920314E092021483E7E8
:10D1400098E6DF91CF911F910F91FF90EF900C9493
:10D1500068678EEE93E10E94A3518EED93E10E94E9
:10D16000A35183ED93E10C94F54B809104149091BD
:10D17000051408950C94354CCF93DF93E0911A0376
:10D18000F0911B030995EC01009729F06A817B81DE
:10D1900081E00E948A55CE01DF91CF9108950F93CF
:10D1A0001F93CF93DF93EC01E0911C03F0911D03DB
:10D1B00009958C016A817B8181E00E948A5581E01A
:10D1C00090E0012B11F480E090E0DF91CF911F916E
:10D1D0000F910895E0911E03F0911F03099420E040
:10D1E00030E00296FC0132974081442331F0FC018B
:10D1F00031974081240F311DF4CFC9010895FC01FE
:10D20000208130E0322F22278181282B02C0220F7B
:10D21000331F6A95E2F7832F9927FA01E05EFC4FEE
:10D22000208130E08223932328E030E0241B350B5B
:10D2300002C0969587952A95E2F708956F927F929E
:10D240008F929F92AF92BF92CF92DF92EF92FF9216
:10D250000F931F93CF93DF938C01EB016A01790148
:10D260002830310524F4A901B601CE014AC0590184
:10D2700023E0B594A7942A95E1F74115510521F0D3
:10D280004801612C712C03C0D801FB0120C048E08B
:10D2900050E0B601CE01860D971D0E94FF68F40193
:10D2A00081934F01FFEF6F1A7F0A6A147B047CF3AE
:10D2B000C501B7FE02C080E090E0A7014770552786
:10D2C0004115510511F1080F191FB60118C0CF0102
:10D2D0008C1B9D0B8A159B051CF481918D93F7CFB8
:10D2E000C501B7FE02C080E090E0A7014770552756
:10D2F0004115510551F0080F191F60E070E08C0FC7
:10D300009D1F0E94FF68F8018083DF91CF911F91DC
:10D310000F91FF90EF90DF90CF90BF90AF909F90D4
:10D320008F907F906F9008958F929F92AF92BF924F
:10D33000CF92DF92EF92FF920F931F93CF93DF93E1
:10D3400000D0CDB7DEB70E9478548C0182E090E027
:10D350000E945654892B19F480E090E05DC0F801DA
:10D36000818190E0982F88272081820F911D0E9453
:10D37000464C7C01009781F30E9478544C01F701E0
:10D380002681822F86958695869590E0422F47705C
:10D3900021E030E011F420E030E0820F931F0E9482
:10D3A0005654892BC9F2F70104811581C12CD12C67
:10D3B000F8018081882379F1F801A180B12CB601B0
:10D3C00033E0759567953A95E1F7A60147705527C3
:10D3D000680D791D883168F09501CE0101960E9493
:10D3E0001E69BE016F5F7F4FF80180810E949E55CC
:10D3F0000DC01A8219829501CE0101960E941E6904
:10D4000069817A81F80180810E948A55CA0CDB1CEF
:10D410000E5F1F4FCDCFC7010F900F90DF91CF91BF
:10D420001F910F91FF90EF90DF90CF90BF90AF9042
:10D430009F908F900895DC0150E0E0E1F0E0E61B62
:10D44000F70BE21BF30B02C0440F551FEA95E2F7FE
:10D450008C91852B8C9311968C911197842B11961E
:10D460008C9308956F927F928F929F92AF92BF920A
:10D47000CF92DF92EF92FF920F931F93CF93DF93A0
:10D480008C016B01EA017901283031051CF44881D7
:10D49000C8015CC0390153E0759467945A95E1F76F
:10D4A0006115710521F04E01A12CB12C03C0D801EA
:10D4B000FE0127C0F40141914F0128E030E0B601A0
:10D4C000C8018A0D9B1D0E941B6AFFEFAF1ABF0A9D
:10D4D000A614B7047CF3C30177FE02C080E090E09D
:10D4E0009701277033272115310509F43FC0C80F74
:10D4F000D91F488150E0B601621B730B685F7F4FF4
:10D500001CC0CF018C1B9D0B861597051CF48191C7
:10D510008D93F7CFC30177FE02C080E090E09701C2
:10D52000277033272115310509F1C80FD91F48810C
:10D5300050E068E070E0621B730B02C055954795A0
:10D540006A95E2F760E070E0800F911FDF91CF9164
:10D550001F910F91FF90EF90DF90CF90BF90AF9011
:10D560009F908F907F906F900C941B6ADF91CF916A
:10D570001F910F91FF90EF90DF90CF90BF90AF90F1
:10D580009F908F907F906F9008956F927F928F926F
:10D590009F92AF92BF92CF92DF92EF92FF920F9342
:10D5A0001F93CF93DF9300D0CDB7DEB78C01FC0182
:10D5B0008681E82EE694E694E694F12C282F2770D5
:10D5C00081E090E011F480E090E0E80EF91EC701E0
:10D5D00002960E94DA54009709F445C00E947F54D5
:10D5E000F8012281FC012083F8012381FC012183C1
:10D5F0000E947F5402965C01A70160E070E00E94E7
:10D600005B8BF80104811581E12CF12CF8018081FC
:10D61000882339F1F8018180912C670163E0D5946A
:10D62000C7946A95E1F73701F7E06F227724CA0CB7
:10D63000DB1C883128F00E94A8559401AC0108C079
:10D640000E9495559A8389839401AE014F5F5F4F85
:10D65000B301C6010E94326AE80CF91C0E5F1F4F2D
:10D66000D5CF81E090E00F900F90DF91CF911F9187
:10D670000F91FF90EF90DF90CF90BF90AF909F9071
:10D680008F907F906F900895E0913B03F0913C0361
:10D690000994E0911403F09115030994E0913F037C
:10D6A000F09140030994E0914103F0914203099401
:10D6B00080E090E008950895E0910C03F0910D034F
:10D6C000099480E090E008950F931F93CF93DF9328
:10D6D000CDB7DEB7E0970FB6F894DEBF0FBECDBF73
:10D6E0000E94C5548C010E947854AE014F5F5F4F79
:10D6F000602F0E943473882309F446C088A99801DA
:10D70000281B3109C9010E945654892BE9F12E8149
:10D7100021110CC0BE016A5E7F4F88E10E949E55B8
:10D72000E0912F03F091300309952EC08A859B85E7
:10D730008D3C3BEA930711F0019631F5223019F048
:10D7400088E090E002C082E090E001979C012F5FAA
:10D750003F4F12161306F4F6E1E0F0E0EC0FFD1F68
:10D76000E80FF91F23852F3F81F3BE01645F7F4FD0
:10D7700089E10E949E5589E10E94A85565E378E2FF
:10D780000E94944B892B31F6E0960FB6F894DEBFD9
:10D790000FBECDBFDF91CF911F910F910895AF9232
:10D7A000BF92CF92DF92EF92FF920F931F93CF938E
:10D7B000DF93CDB7DEB7E0970FB6F894DEBF0FBEAC
:10D7C000CDBF8C016B01CE0101967C0180E3F70196
:10D7D00011928A95E9F781E089838CE00E94955542
:10D7E0008C831D821F828091081491E0980F909382
:10D7F0000814898783E0B82EB8868DEC9BEA9B8756
:10D800008A8789E10E94A85568EE72E00E94944BD5
:10D81000892B31F082E08E838FEF8C878D8709C052
:10D8200089E10E94A855BC01CE010C960E948B4B49
:10D83000BE828DEC9BEA9D8B8C8B65E378E2CE01FA
:10D8400046960E948B4B0E9478549FA78EA70E94F9
:10D85000C55488ABC7010E942D72B82E90E00E947B
:10D86000DA54892B31F10E947F54BC014B2DC70142
:10D870000E944B72E0900203F09003030E94CF5489
:10D880005C010E947F54B501F7010995011511054E
:10D8900081F0009739F0019761F441E050E064E0D5
:10D8A00070E004C041E050E060E070E0C601F801C3
:10D8B0000995E0960FB6F894DEBF0FBECDBFDF919D
:10D8C000CF911F910F91FF90EF90DF90CF90BF907D
:10D8D000AF9008950E94AD6D80930814E0910C0301
:10D8E000F0910D030994892B29F0E0910C03F0913C
:10D8F0000D0304C0E0910E03F0910F030994CF9340
:10D90000DF93EC0189919991009729F060E070E034
:10D910000E94DF4DF7CFDF91CF910895CF93DF9332
:10D92000EC0189919991009719F00E94314DF9CF3E
:10D93000DF91CF910895CF93DF93EC017B836A83CE
:10D940000E94445E99838883DF91CF910895FC0102
:10D950008081918122813381820F931F9183808303
:10D960000895CF93DF93EC010E94445E99838883EE
:10D97000DF91CF910895CF93DF93EC010E94445E35
:10D9800028813981821B930B9C012F5F3F4F81E0DF
:10D9900090E04A815B814217530710F080E090E0ED
:10D9A000DF91CF910895CF93DF93FC01C281D381A2
:10D9B00080819181C80FD91F0E94445E9E01281B5F
:10D9C000390BC901DF91CF910895CF93DF93EEEA30
:10D9D000FAE2C0E7DAE2A2EABAE2119211921992EF
:10D9E0001992199219921D928AE2E63CF807A9F75A
:10D9F000DF91CF910895CF93DF93FC01EE55F54D64
:10DA000040819C01220F331F220F331F442301F159
:10DA1000A0919400B0919500FC01EE0FFF1FE2551C
:10DA2000F54D80819181AD01481B590BCA01E90177
:10DA3000C059D54D488159816A817B81480F591F52
:10DA4000611D711D488359836A837B83B183A083E1
:10DA5000F901E059F54D6081718182819381DF91F7
:10DA6000CF91089560E070E0CB010895FC01EE0FC6
:10DA7000FF1FEE0FFF1FE059F54D40835183628376
:10DA800073830895CF93DF9322EA3AE2C0E7DAE2A4
:10DA9000EEEAFAE2D9018D919D018823B9F0409117
:10DAA00094005091950080819181BA01681B790B97
:10DAB00088819981AA81BB81860F971FA11DB11D05
:10DAC00088839983AA83BB835183408324963296AB
:10DAD000BAE22E3A3B07F1F6DF91CF9108950C940C
:10DAE000BC710F931F93FC01CB014091091450911D
:10DAF0000A14338322831583048371836083F09334
:10DB00000A14E0930914452B11F40E94D67180E0A9
:10DB100090E01F910F9108958091091490910A143B
:10DB20000097C1F010920A1410920914DC011496A7
:10DB30006D917C9115971296ED91FC911397099533
:10DB4000E0910914F0910A14309721F080819181BD
:10DB50000C94D67108950C94E5870C94E18780ECC1
:10DB600092E00E94164E88EB92E00C94164ECF93F2
:10DB7000DF930E948554892BA9F088EB92E00E94E4
:10DB8000344EEC01009721F10E94C554998388839B
:10DB90000E94C0549B838A83CE0104960E94015444
:10DBA0008CAB14C080EC92E00E94344EEC010097E4
:10DBB00079F002960E94135499838883BE016E54B3
:10DBC0007F4FCE018E579F4F0E946855CE0102C0F5
:10DBD00080E090E0DF91CF910895BC016E547F4FBB
:10DBE0008E579F4F0C946855CF93DF93EC01BC0187
:10DBF00080EC92E00E947E4EBE01892B19F080ECF1
:10DC000092E009C088EB92E00E947E4E892B39F0A9
:10DC1000BE0188EB92E0DF91CF910C94594EDF91D9
:10DC2000CF9108950F931F93CF93DF93EC01BC0125
:10DC300080EC92E00E947E4E892B91F0FE01619172
:10DC40007191CF010E942455BE016E547F4FCE01C9
:10DC50008E579F4FDF91CF911F910F910C94795563
:10DC6000BE0188EB92E00E947E4E892BD1F00E948B
:10DC70001155688179818A819B810E9424558CA9E4
:10DC800090E00E94DA540CA910E00E947F54BE017B
:10DC90006C5F7F4FA801DF91CF911F910F910C9482
:10DCA000528BDF91CF911F910F910895CF93DF9306
:10DCB000EC01BC0180EC92E00E947E4E892B19F0B1
:10DCC000CE0102960CC0BE0188EB92E00E947E4E0F
:10DCD000892B19F08A819B8102C080E090E0DF915E
:10DCE000CF910895FC01808191810895860F911D47
:10DCF000860F911D8E579F4F0895860F911D860F99
:10DD0000911D8E579F4FFC01808191810895089548
:10DD100088E69AE10E945850892B21F088E69AE122
:10DD20000C9445500895E091541AF091551A30978B
:10DD300009F0099480E00895EF92FF920F931F93EA
:10DD4000CF93DF937C01EA01FC01808191810097F0
:10DD500041F08C30934071F1F7011182108283E021
:10DD6000F2C080E024E0829FF0011124EA5AF54ECF
:10DD7000118210828F5F8430A8F38093531A8091B0
:10DD80008E1190918F119093671A8093661A0E945A
:10DD90002A4D8093C62A60E470E088E69AE10E94EA
:10DDA00031500E94AA748CE093E0F7019183808344
:10DDB00081E0C9C06230D9F48091C72A9091C82A05
:10DDC000892B89F38091D82A863029F48091F02A12
:10DDD00081FD0E94886E81E00E94E8758091C72ACB
:10DDE0009091C82A892BF9F20E94AC70DCCF633085
:10DDF00060F5611114C02097B1F2D093D52FC09374
:10DE0000D42F83E00E94E8758091C72A9091C82A98
:10DE1000892B11F00E94936E0E94886EC4CF6130EE
:10DE200011F6209709F4BFCFD093D12FC093D02FF4
:10DE300085E00E94E8758091C72A9091C82A892BB5
:10DE400009F4B1CF0E94936EAECF6738E9F5109216
:10DE5000521A06E51AE18091521A8430B8F4F8019A
:10DE6000828193818C179D0749F4808191810E9462
:10DE7000B575F80111821082138212820C5F1F4F58
:10DE80008091521A8F5F8093521AE5CFEFEEFFE236
:10DE9000838194818C179D0719F414821382108258
:10DEA000B09620E3EF36F20799F7ECE6F0E38185D0
:10DEB00092858C179D0711F4158214823D9680E39C
:10DEC000EE3EF807A1F76FCF683809F06CCFC8565F
:10DED000DA4109F068CF88E69AE10E945850892B10
:10DEE00009F461CF1092521AE091521AE43008F00E
:10DEF0005ACF20E2E29FF0011124EA52F04D818DC9
:10DF00008823D9F088E69AE10E9445508091521A00
:10DF1000E0E28E9FC00111248A52904D9093D52F3C
:10DF20008093D42F82E00E94E8758091C72A909157
:10DF3000C82A892B11F00E94936E8091521A8F5F2C
:10DF40008093521AD1CFDF91CF911F910F91FF9003
:10DF5000EF9008959093551A8093541A0895209144
:10DF60008E1130918F1160E0E6E5FAE1643098F4AB
:10DF7000408151814817590759F442815381421712
:10DF8000530731F46093511A118210820C94B575C5
:10DF900034966F5FEBCF6093511A089540E0E6E549
:10DFA000FAE14430A8F451E0540F20813181232B51
:10DFB00061F44093501A9183808320918E113091A7
:10DFC0008F11338322830C94CF753496452FE9CF7C
:10DFD0004093501A089520918E1130918F11FC01B9
:10DFE000358F248F778F668F089520918E11309111
:10DFF0008F11FC0132872187748763870895CF933F
:10E00000DF93EA010E945875009749F020918E1124
:10E0100030918F11FC0132872187D487C387DF912C
:10E02000CF9108950F931F93CF93DF9300D000D02B
:10E03000CDB7DEB78C01AB018FEF89838A838B83E9
:10E040008C83B801CE0101960E94FF6F009719F0F2
:10E05000FC01158304830F900F900F900F90DF91B8
:10E06000CF911F910F91089540E050E062E088EC5D
:10E0700092E00E94D04D1092C82A1092C72A0895AB
:10E08000AC0161E088EC92E00C94B24DAC0160E030
:10E0900088EC92E00C94B24D0F931F93CF93DF93D3
:10E0A0008A010E94D674EC01009759F080918E117C
:10E0B00090918F119D8F8C8F1F8F0E8FCE010E949C
:10E0C0004670CE01DF91CF911F910F910895CF93AC
:10E0D000DF93A091D42FB091D52F109719F0ED01B7
:10E0E0006C9605C0C091D02FD091D12F29968091E8
:10E0F000CF2F86FF22C010924F1A40E0E6E5FAE1EA
:10E100004430B8F42081318114968D919C911597FB
:10E110002817390759F482819381009739F0409389
:10E120004F1A998388831B821A8205C034964F5FE9
:10E13000E7CF40934F1A0E94886E8881998100979B
:10E1400041F04A815B816091C62ADF91CF910C94A6
:10E15000D04DDF91CF9108950F931F93CF93DF930D
:10E160008091D82A863009F071C08091C72A909199
:10E17000C82A8115954009F069C0C4E9D2E0D0935E
:10E18000C82AC093C72A02E00093D12A14E9109349
:10E19000D22A1092F42A1092F32A0E94A474809535
:10E1A00090959093F42A8093F32A1092DA2A109291
:10E1B000D92A0E949374809590959093DA2A80933F
:10E1C000D92A0E94936ED093C82AC093C72A00937D
:10E1D000D12A1093D22AA091D22FB091D32FFD0132
:10E1E000E459FD4F8CE692E001900D920197E1F722
:10E1F0006CE672E087EE9AE20E9452748091CB2A1C
:10E200008093E72A8091CC2A8093E82A8091CD2AB6
:10E210008093E92A8091CE2A8093EA2A1092F42AE8
:10E220001092F32A0E94A474809590959093F42AFA
:10E230008093F32A1092DA2A1092D92A0E949374BA
:10E24000809590959093DA2A8093D92ADF91CF9187
:10E250001F910F910C94936EFC01680F791F80E061
:10E2600048E1E617F70781F0219198E0322F38272F
:10E27000532F517030FD84278695513009F4806802
:10E280002695915099F7EDCF08951F920F920FB6F2
:10E290000F9211240BB60F922F933F934F935F93DE
:10E2A0006F937F938F939F93AF93BF93EF93FF935E
:10E2B00080919400909195009093B32A8093B22A14
:10E2C00081E08093A42A80917100807D8093710009
:10E2D0000E948C6D8091A42A8823D9F180919400AA
:10E2E000909195004091B22A5091B32A84179507D6
:10E2F000A0F48091782A9091792AA0917A2AB091FD
:10E300007B2A8C57914EAF4FBF4F8093782A9093C2
:10E31000792AA0937A2AB0937B2A20919400309195
:10E320009500241B350B8091782A9091792AA09131
:10E330007A2AB0917B2A820F931FA11DB11D809371
:10E34000782A9093792AA0937A2AB0937B2A109204
:10E35000A42AFF91EF91BF91AF919F918F917F91EF
:10E360006F915F914F913F912F910F900BBE0F9046
:10E370000FBE0F901F9018959FB7F894E1E7F0E05B
:10E380008081807D808388B38F6288BB10929000EB
:10E39000E1E9F0E010821092920010929500109244
:10E3A00094008081856080839FBF08952FB7F89483
:10E3B000909399008093980088B38F6288BBE1E7BF
:10E3C000F0E08081826080832FBF0895CF93DF9338
:10E3D000FC01DB0185E0EB0119928A95E9F7858163
:10E3E000837011F082E08C938781837021F082E04A
:10E3F00012968C9312978581837081F08781837048
:10E4000069F023893489818592852817390731F489
:10E4100081E0848312961C92129701C01482858138
:10E420008370823021F0833021F080E003C082E0ED
:10E4300001C088E011968C93119787818370823098
:10E4400021F0833021F080E003C082E001C088E049
:10E4500013968C93DF91CF910895CF93DF9300D0E3
:10E4600000D01F92CDB7DEB7BE016F5F7F4F0E9415
:10E47000E67189819A81890F8D5F9B81890F9C81CB
:10E48000890F9D81890F0F900F900F900F900F9023
:10E49000DF91CF9108954F925F926F927F928F920A
:10E4A0009F92AF92BF92CF92DF92EF92FF920F9323
:10E4B0001F93CF93DF9300D000D000D0CDB7DEB74D
:10E4C0008C017B01BE016F5F7F4F4E830E94E6711E
:10E4D000B981AA815B804C808B2F90E003962A2F14
:10E4E00030E0820F931F850D911D642D70E0860F23
:10E4F000971F5D81850F911D4E8150E04817590788
:10E500000CF49AC0F801818180FB662460F8712CBC
:10E5100043E0660C771C4A95E1F7828180FB8824F2
:10E5200080F8912C54E0880C991C5A95E1F78628C4
:10E5300080818770882A838180FBAA24A0F8B12C6F
:10E5400085E0AA0CBB1C8A95E1F78A28848180FBB0
:10E55000CC24C0F8D12C96E0CC0CDD1C9A95E1F7C8
:10E560008C28F7018082F80145814370F4E04F9FC9
:10E57000A0011124F80186818370F0E18F9FC00112
:10E580001124482BF8018781F0E48F9FC0011124EA
:10E59000482BF7014183F8018085F7018283B2306F
:10E5A00059F4F8018185F7018383F8018285F70129
:10E5B000848395E0C92E02C083E0C82EB0E080E0DD
:10E5C00090E0200F311FDB2EDC0C0197BA1761F0B1
:10E5D000A901480F591FFA01B384A7014D0D511D20
:10E5E000FA01B082BF5FEFCF9D2DF2E05F120EC047
:10E5F000D701AD0DB11DF80183898C9381E08D0D9C
:10E60000D701A80FB11D9E5F84898C9340E020E064
:10E6100030E0060F171F842F890F21503109441550
:10E6200061F0D801A20FB31F55965C91D701A80FD6
:10E63000B11D5C934F5FEFCF80E026960FB6F89444
:10E64000DEBF0FBECDBFDF91CF911F910F91FF9025
:10E65000EF90DF90CF90BF90AF909F908F907F9082
:10E660006F905F904F900895BF92CF92DF92EF929C
:10E67000FF920F931F93CF93DF937C01D62EEA0175
:10E6800082E0861708F0B2C0F701808186FBBB24C8
:10E69000B0F89181292F269526952370C92EC29412
:10E6A000C694C69453E0C522382F3770388383FB55
:10E6B000332730F9398384FB332730F93A8385FBDC
:10E6C000882780F98B83BC822D83892F8295837064
:10E6D0008E83CF8282818887222391F13381848146
:10E6E00090E0982F8827830F911D9A87898787014B
:10E6F0000B5F1F4F223079F468EE72E0CE010B966B
:10E700000E948B4BF70186818B8785818C878701DF
:10E71000095F1F4F20C02330F1F4F7013D9680E0E0
:10E7200090E03E2F2F2F4291DE01A80FB91F1B96BC
:10E730004C93019688309105B1F7032F122F0BC02F
:10E7400087010D5F1F4F68EE72E0CE010B960E94AD
:10E750008B4B1A861986CC20B9F1B1100DC0F80187
:10E760002081818190E0982F8827820F911D9C8BBA
:10E770008B8B0E5F1F4F04C089859A859C8B8B8B7A
:10E78000F2E0CF120EC068EE72E0CE0145960E9414
:10E790008B4BF80181818D8B80818E8B0E5F1F4F9B
:10E7A0001BC0F3E0CF1218C0085F1F4FF80180E0D4
:10E7B00090E02291DE01A80FB91F55962C93019687
:10E7C00088309105B1F708C068EE72E0CE01459639
:10E7D0000E948B4B1C8A1B8AC8018E199F092D2D04
:10E7E000281B2FA71EA70DA7D81608F480E0DF91DD
:10E7F000CF911F910F91FF90EF90DF90CF90BF903E
:10E800000895FB0141505109460F571FE417F507C2
:10E8100078F4208130E0322F22276181260F311DCC
:10E82000820F931F8217930708F401963296EECF5A
:10E83000E417F50751F4208130E0322F2227820FB0
:10E84000931F8217930708F401960895CF93DF93DF
:10E85000C091D22AD0E064972091D12A30E0322FA3
:10E860002227C20FD31F48E050E06BED7AE29E01F1
:10E87000280F311DC9010E940174AE0163EE7AE2D6
:10E880000E940174009721F098278927982702C0D9
:10E890008FEF9FEFDF91CF9108959093811A80932E
:10E8A000801A0895FC015381560F5093CE2A872F6A
:10E8B00099274281480F4093CD2AA181A093CC2A69
:10E8C000E081E093CB2A242F30E02817390748F461
:10E8D00081E08A0F8093CC2A811103C0EF5FE0931F
:10E8E000CB2A852F90E077278617970788F44F5F0C
:10E8F0004093CD2A41110CC08091CC2A8F5F809328
:10E90000CC2A811105C08091CB2A8F5F8093CB2ABE
:10E910000895AB01BC0180E090E00E94017498274B
:10E9200089279827089544E150E06FEC7AE280E06F
:10E9300090E00E940174009721F09827892798277A
:10E9400008958FEF9FEF089586E00C94267481E17F
:10E950000C94267480E0E82FF0E0EE0FFF1FEA5AD7
:10E96000FF4C118210828F5F8430A8F380E090E228
:10E97000899FF0011124EA52F04D118E8F5F84308F
:10E98000B0F380E094E090937B1A80937A1A80E051
:10E990009DE0989FF0011124E459FF4C15821482E8
:10E9A0008F5F8A30B0F38093791A0895CF932091C6
:10E9B0007A1A30917B1A2F5F3F4F21154DE73407AC
:10E9C00010F020E030E1522F432FE6EDFFE2C0E0EF
:10E9D000C43059F0A18DAA2329F0A481B581A417D0
:10E9E000B50749F3CF5FB096F3CF30937B1A2093EE
:10E9F0007A1A1092791A20E0E0E0F0E02430E8F48E
:10EA000030E2239FD0011124AA52B04D59963C9177
:10EA10005997311104C02093791AFD0110C0373085
:10EA200041F4309739F05A964C915A97328D3417F9
:10EA300008F0DF012F5FFD01E1CF2093791A3097B5
:10EA4000A1F122E0218F20917C1A248720917D1A48
:10EA5000258720917E1A268720917F1A278728ED07
:10EA600034E0338B228B358B248B21E030E0318BEB
:10EA7000208B138E21E0228F23E0208F168A20E145
:10EA8000278B20917A1A30917B1A3227232732273D
:10EA90003583248377836683DC014D915D916D918D
:10EAA0007C914083518362837383CF01CF9108951A
:10EAB000CF93DF9320917A1A30917B1A2F5F3F4FCB
:10EAC00021154DE7340710F020E030E1522F432F9D
:10EAD000E0E7F0E3C0E0CA3041F0A081B181CF5F50
:10EAE0003D96A417B507B9F7E9CF30937B1A209369
:10EAF0007A1A40E05DE04A30A0F4A1E0A40F549FF0
:10EB0000F0011124E459FF4C24813581232B39F481
:10EB10004093791A309741F480E090E023C04A2F67
:10EB2000EACF4093791AF8CF20917A1A30917B1A64
:10EB30003227232732273583248377836683009700
:10EB400029F4108211821282138209C0EC0188819B
:10EB50009981AA81BB8180839183A283B38380E45E
:10EB60008087CF01DF91CF91089540E04430A0F439
:10EB7000E42FF0E051E0540FEE0FFF1FEA5AFF4C74
:10EB8000208131812817390729F44093791A11829D
:10EB900010820895452FEACF4093791A089540E0F6
:10EBA000443098F4E42FF0E051E0540FEE0FFF1FD3
:10EBB000EA5AFF4C20813181232B29F44093791AA2
:10EBC000918380830895452FEBCF4093791A089560
:10EBD000AF92BF92CF92DF92EF92FF920F931F936B
:10EBE000CF93DF93C091D42FD091D52F843009F4E7
:10EBF000DCC127EF3AE23093D32F2093D22F30930A
:10EC0000CA2A2093C92A833059F4898D8F708330A2
:10EC100009F06BC088899989892B09F0DFC67FC00C
:10EC2000823009F080C080917F1A8F5F80937F1AB5
:10EC3000811113C080917E1A8F5F80937E1A81119B
:10EC40000CC080917D1A8F5F80937D1A811105C061
:10EC500080917C1A8F5F80937C1A1092C82A109240
:10EC6000C72A10926B3010926A30298D822F8D7FC7
:10EC7000853041F48A8D8F5F8A8F843109F0AEC66A
:10EC8000198EACC6222309F4A9C688899989892BD3
:10EC900009F441C08A8D9FEF980F9A8F81119EC60B
:10ECA0008B8D883031F09FEF920F923048F4853091
:10ECB00039F4198E80E88093CF2F0E94677047C582
:10ECC000853038F493E0082E01C0990F0A94EAF7D2
:10ECD00001C090E39A8F8F5F8B8F822F8F7083306C
:10ECE000A1F048F4813009F44FC3823009F076C6B0
:10ECF0001092F02A4CC3863009F4C8C4883009F455
:10ED0000C5C4843009F06AC6C1C484E08093CF2FA3
:10ED10000E9467704EC52F70233009F05FC688E0EF
:10ED20008093CF2F09C5853019F5E091D02FF09150
:10ED3000D12F84819581892B09F450C61092D52F4B
:10ED40001092D42F8BEE9AE29093D32F8093D22FF0
:10ED50009093CA2A8093C92A10926B3010926A301D
:10ED60001092C82A1092C72A88E08093CF2F1BC127
:10ED70008091CF2A853409F031C60091D12A10E064
:10ED8000102F00278091D22A080F111D8091C72AC9
:10ED90009091C82A8017910708F420C61093C82ABA
:10EDA0000093C72A8091D52A8F7309F017C68091E6
:10EDB000D62A811113C68091663090916730C09138
:10EDC0004503D09146038C179D0759F44091683054
:10EDD00050916930209147033091480342175307FF
:10EDE000A1F02091DF2A3091E02A2817390709F095
:10EDF000F5C52091E12A3091E22A80916830909106
:10EE000069302817390709F0E9C50E949374019603
:10EE100009F0E4C58091D82A863009F429C18131EE
:10EE2000E9F1813009F0DAC58091E32A883009F0F0
:10EE3000D5C51092E32A8091E52A9091E62A873F72
:10EE40003FEF930710F0099601C008969093E62AC9
:10EE50008093E52A8091DB2A9091DC2AA091DD2A1B
:10EE6000B091DE2A8093DF2A9093E02AA093E12AD2
:10EE7000B093E22A8091663090916730A09168301B
:10EE8000B09169308093DB2A9093DC2AA093DD2A2D
:10EE9000B093DE2A80E48093D72A7DC50C511109F6
:10EEA0001093C82A0093C72A8BEE9AE29093D32F2F
:10EEB0008093D22F8091E92A9091EA2A892B29F018
:10EEC0000E94A774019609F089C52091E52A309126
:10EED000E62A2115310509F481C58CE690E390936B
:10EEE000D12F8093D02FA090E32AB090E42A4091B4
:10EEF0004703509148036091490370914A03A091E0
:10EF00004B03B0914C030091DB2A1091DC2AE09076
:10EF1000DD2AF090DE2AE091D02FF091D12F80E30E
:10EF2000EE3EF80708F05AC584819581009721F1DB
:10EF30002817390709F586819781009719F0A816D7
:10EF4000B906D1F4808191818C179D0729F4C28084
:10EF5000D380C416D506B1F08617970729F4C2806E
:10EF6000D380CA16DB0671F00817190729F48281CD
:10EF70009381E816F90631F03D96F093D12FE09396
:10EF8000D02FC9CF1092D52F1092D42F82E080932A
:10EF9000CF2F8BEE9AE29093CA2A8093C92A1092BF
:10EFA0006B3010926A300E94677080916A30909145
:10EFB0006B30009709F412C59C01245E3F4F3093DB
:10EFC000C82A2093C72A3093D12A2093D22AE091CD
:10EFD000D02FF091D12F20852093D72A21E12093A3
:10EFE000D82A08969827892798279093E82A80930B
:10EFF000E72A1092EA2A1092E92A84819581909357
:10F00000E42A8093E32A868197819093E62A80936D
:10F01000E52A8091663090916730A0916830B09178
:10F0200069308093DB2A9093DC2AA093DD2AB09389
:10F03000DE2A80819181A281B3818093DF2A90931F
:10F04000E02AA093E12AB093E22A87EF9AE2909314
:10F05000D32F8093D22F0E94A7748095909500970C
:10F0600011F48FEF9FEF9093EA2A8093E92A93C4DB
:10F070000E94A474019609F0B1C48091E52A909190
:10F08000E62A009709F4AAC42091E32A3091E42AE1
:10F090002115310509F4A2C44091DB2A5091DC2AE4
:10F0A0006091DD2A7091DE2AEFEEFFE2C6EDDFE22D
:10F0B000F080FF20A9F0AC81BD818A179B0781F405
:10F0C000AE81BF812A173B0759F4A881B9814A173D
:10F0D0005B0731F4AA81BB816A177B0709F46FC112
:10F0E000A096B096A0E3C635DA0711F72091F02A72
:10F0F0002F732230D9F49093771A8093761A40E0D8
:10F10000443090F4E42FF0E0EE0FFF1FEA5AFF4C7A
:10F11000208131814F5F8217930791F71092791AFE
:10F1200020E0C0E0D0E07EC04093791A8091F02AC0
:10F1300082FD54C484E18093F02A88E290E09093A9
:10F14000C82A8093C72A80E58093EF2A8091EA2A13
:10F150009091EE2A9093EA2A3091E92A9091ED2A33
:10F160009093E92A3093ED2A2091E82A9091EC2A95
:10F170009093E82A2093EC2A9091E72A9093791AA9
:10F180004091EB2A4093E72A9093EB2A8F5F80937C
:10F19000EE2A81110FC081E0830F8093ED2A811147
:10F1A00009C081E0820F8093EC2A811103C09F5F28
:10F1B0009093EB2A8091E32A9091E42A9093771A16
:10F1C0008093761A2091E52A3091E62A3093E42A3A
:10F1D0002093E32A9093E62A8093E52A8091DB2A04
:10F1E0009091DC2AA091DD2AB091DE2A8093DF2A5B
:10F1F0009093E02AA093E12AB093E22A80916630AE
:10F2000090916730A0916830B09169308093DB2A8B
:10F210009093DC2AA093DD2AB093DE2AA1C3373075
:10F2200089F02F5F2430C0F430E2239FC001112405
:10F23000FC01EA52F04D318D3111F1CF2093791A52
:10F24000EF010CC0209721F0428D3A8D341748F71A
:10F25000EC01CA52D04DE5CF2093791A209709F4DA
:10F26000BDC3D093D52FC093D42F83E08A8F888FCE
:10F270001E8A84E08F8B1B8E8091E52A9091E62A6E
:10F280009D838C838091E32A9091E42A9F838E83CF
:10F290008091DB2A9091DC2AA091DD2AB091DE2AB0
:10F2A00088839983AA83BB8381E0898F80917C1AAC
:10F2B0008C8780917D1A8D8780917E1A8E878091B0
:10F2C0007F1A8F8781E090E0998B888B8091EA2A62
:10F2D0008B878091E92A8A878091E82A89878091A3
:10F2E000E72A888781E090E00E94527D8091EF2A92
:10F2F000282F207F30E0213531050CF445C0829560
:10F300008F7090E00597880F991F880F991F309193
:10F31000781A20E0E22FF0E0E817F9078CF5E153C6
:10F32000F54D30A5311105C02093791A1092781A45
:10F330002BC0313011F42F5FEDCF3230E1F441A515
:10F340004430C9F42093791A3093781A82A590E05A
:10F35000982F882723A5822B9093771A8093761A6B
:10F36000893DA4E09A0710F088ED94E09B8B8A8B8E
:10F370009D8B8C8B09C041A5442311F0240FCACF6B
:10F380002093791A3093781A80E18093F02A809143
:10F39000F02A82608093F02A82E08093F72A84E04A
:10F3A0008093F82A8093F92A88ED8093FA2A8CE2D8
:10F3B00090E09093C82A8093C72A80E67EC2D093BB
:10F3C000D52FC093D42F1092CF2F9091F02A92FF77
:10F3D00003C0198E80E21AC28091EF2A82958F7045
:10F3E000880F880F8093791A081B1109045111099D
:10F3F0001093C82A0093C72A8F2D8F70823029F46A
:10F40000892F8F73823139F41FC0813021F4892F05
:10F410008F738230C9F0012B19F4892F8370A1F00A
:10F420002091E72A888528133EC22091E82A898501
:10F43000281339C22091E92A8A85281334C22091E1
:10F44000EA2A8B8528132FC294FF4AC068897989DC
:10F450006115710509F444C0CE010C960E945274E6
:10F460003091EB2A8091CB2A38133AC02091EC2AB4
:10F470008091CC2A281334C09091ED2A8091CD2A16
:10F4800098132EC08091EE2A4091CE2A841328C072
:10F490003C872D879E878F878B8D81111AC02E897F
:10F4A000888D9A8D891B922F969596959695891B96
:10F4B000280F2E8B87FD81959F89392F369536959C
:10F4C000931B980F9F8B822F869586958695890F23
:10F4D000888F81E08093CF2F888D8A8F198A188A30
:10F4E000498D842F8F7090E0FC013197E830F10551
:10F4F00008F074C2E057FF4F0C941D878091CF2F06
:10F5000080FF14C083E0898F80E48093CF2F198A15
:10F51000188A8091C72A9091C82A009709F408C1D7
:10F5200022E42093CF2F0E94527D02C18091F02AC5
:10F530008F73823009F052C227CF8091CF2F80FF86
:10F5400070C08091F02A8F73823109F06AC0809177
:10F55000EF2A282F207F30E0213531050CF445C0FB
:10F5600082958F7090E00597880F991F880F991FDB
:10F570003091781A20E0E22FF0E0E817F9078CF5D7
:10F58000E153F54D30A5311105C02093791A109241
:10F59000781A2BC0313011F42F5FEDCF3230E1F407
:10F5A00041A54430C9F42093791A3093781A82A582
:10F5B00090E0982F882723A5822B9093771A809329
:10F5C000761A893D24E0920710F088ED94E09B8B39
:10F5D0008A8B9D8B8C8B09C041A5442311F0240F8D
:10F5E000CACF2093791A3093781A83E0898F80915B
:10F5F000E72A88878091E82A89878091E92A8A8783
:10F600008091EA2A8B8781E090E00E94527D82E41B
:10F610008093CF2F198A188A1092C82A1092C72A6D
:10F6200087C080E28093CF2F0E946770E091D42F33
:10F63000F091D52F118E7ACD8091F02A80FF28C0CD
:10F6400044FD26C088899989892B09F0C7C180911A
:10F65000C72A9091C82A01960E94527D2091CF2FEF
:10F66000822F80618093CF2F8091C72A9091C82AE2
:10F67000892B19F022612093CF2F0E94677081E0BF
:10F6800090E0998B888B88E0898F1B8E81E10CC17B
:10F6900085FF1CC08091F52A90E0982F8827209143
:10F6A000F62A822B2091D22F3091D32F280F391F89
:10F6B0003093D32F2093D22F2091C72A3091C82A7C
:10F6C000281B390B3093C82A2093C72A8091C72A58
:10F6D0009091C82A009749F044FD07C02091CF2F90
:10F6E00022602093CF2F0E94527D8091F12A90E0DA
:10F6F000982F88272091F22A820F911D9093771AD4
:10F700008093761A2C893D892817390710F0892BA8
:10F7100021F43093771A2093761A8091761A90917B
:10F72000771A9B8B8A8B8091CF2F837009F456C1F7
:10F7300010926B3010926A300E9467708091CF2FC8
:10F7400085FF07C010926B3010926A30198E84E1E9
:10F75000ABC084FF0AC010926B3010926A3081E017
:10F7600090E0998B888B84E08FCF20916A30309124
:10F770006B3021153105E1F080FF02C0198A188A2B
:10F7800088899989009781F48A899B8982179307D0
:10F7900020F490936B3080936A3080916A3090911E
:10F7A0006B30998B888B04C090936B3080936A3058
:10F7B0001B8E8091C92A9091CA2A9093D32F80934F
:10F7C000D22F80916A3090916B30892B59F08889C3
:10F7D0009989009739F088969093C82A8093C72A10
:10F7E00088E10BC08091CF2F81FFF8C088E290E0C4
:10F7F0009093C82A8093C72A80E18093F02A5CC046
:10F800008091CF2F80FFEAC0198E80E18093CF2FA7
:10F810000E946770E3C08091C72A9091C82A009720
:10F8200011F00E94527D9091F02A8091CF2F90FF8D
:10F830000BC080FF06C087E0898F1A8E198A188A4C
:10F8400019C086E0898F16C080FF1EC085E0898FB1
:10F85000198A188AC3C08091C72A9091C82A009734
:10F8600011F00E94527D8091F02A80FF0DC087E048
:10F87000898F1A8E81E090E00E94527D80E1809312
:10F88000CF2F0E9467700FC08091C72A9091C82A1D
:10F89000892B49F4A3C08091CF2F80FF9FC087E0C0
:10F8A000898F1A8E9BC080E18093F02A88E290E0D5
:10F8B0009093C82A8093C72A80E58093EF2A888591
:10F8C0008093EB2A89858093EC2A8A858093ED2AA0
:10F8D0008B858093EE2A8C858093E72A8D85809393
:10F8E000E82A8E858093E92A8F858093EA2A86E02C
:10F8F0008093D82A8C819D819093E42A8093E32A77
:10F900008E819F819093E62A8093E52A80916630CC
:10F9100090916730A0916830B09169308093DB2A74
:10F920009093DC2AA093DD2AB093DE2A8881998106
:10F93000AA81BB818093DF2A9093E02AA093E12AD9
:10F94000B093E22A898D84FF05C01092F22A1092AA
:10F95000F12A06C084E08093F12A88ED8093F22A90
:10F9600080E48093D72A8091C72A9091C82A9093E7
:10F97000D12A8093D22A1092F62A1092F52A109258
:10F98000F42A1092F32A0E94A47480959095909383
:10F99000F42A8093F32A85E48093CF2A1092D02A08
:10F9A0001092D62A1092D52A8091801A9091811AAD
:10F9B00001969093811A8093801A9093D32A809312
:10F9C000D42A1092DA2A1092D92A0E949374809530
:10F9D00090959093DA2A8093D92A04C01092C82A6D
:10F9E0001092C72A1092CF2FDF91CF911F910F91C4
:10F9F000FF90EF90DF90CF90BF90AF900895982741
:10FA00008927982708950E9423870895FC018091F3
:10FA1000C92A9091CA2A2FEC3FE2281B390BAB016F
:10FA2000261737070CF4A9011416150654F4509341
:10FA30006B3040936A30E817F90719F0BF010C9456
:10FA4000528B089580E880936100109261000E94BB
:10FA5000D85B0E94474D0E94B45F809176289091B8
:10FA60007728009729F0019790937728809376283C
:10FA7000C0907828D0907928E0907A28F0907B2860
:10FA80000E94725EC616D706E806F90611F30E94B8
:10FA9000725E609378287093792880937A28909387
:10FAA0007B28D7CF2091D42F3091D52FBC01C9010D
:10FAB00008960E945274E091D42FF091D52F809136
:10FAC000CB2A80878091CC2A81878091CD2A82871A
:10FAD0008091CE2A838708952F923F924F925F9212
:10FAE0006F927F928F929F92AF92BF92CF92DF924E
:10FAF000EF92FF920F931F93CF93DF93CDB7DEB7B3
:10FB000063970FB6F894DEBF0FBECDBF7C011B011B
:10FB10006A01FC0117821682838181FF66C3BE01E0
:10FB20006F5F7F4F4B01F7019381F10193FD859149
:10FB300093FF81911F01882309F453C3853239F45F
:10FB400093FD859193FF81911F01853239F4B701AF
:10FB500090E00E94BB8B56016501E5CF10E0512C6F
:10FB600020E02032A0F48B3269F030F4803259F07A
:10FB7000833269F420612CC08D3239F0803339F43E
:10FB8000216026C02260246023C0286021C027FD98
:10FB900027C030ED380F3A3078F426FF06C0FAE07F
:10FBA0001F9F300D1124132F13C06AE0569E300D95
:10FBB0001124532E20620CC08E3221F426FD11C375
:10FBC000206406C08C3611F4206802C0883641F4E7
:10FBD000F10193FD859193FF81911F018111C1CFA7
:10FBE0009BEB980F933018F42061805E06C09BE970
:10FBF000980F933008F0AAC12F7E26FF16E02F73CE
:10FC0000722E853621F4F22FF0647F2E08C08636DE
:10FC100021F4622F6068762E02C01111115077FE18
:10FC200007C01C3348F444244394410E27E00BC022
:10FC3000183030F4212F06C027E04CE3442E03C0D7
:10FC400027E017E0412C560174E0A70EB11CF60125
:10FC50006081718182819381042DA4010E945A8A5E
:10FC60006C01098100FF02C003FF06C071FC07C0E0
:10FC700072FC08C0612C08C03DE2632E05C02BE277
:10FC8000622E02C090E2692E802F8C7099F166205E
:10FC900011F084E001C083E0851510F0512C0BC0F9
:10FCA000581A73FC08C0B70180E290E00E94BB8B39
:10FCB0005A94C9F7F3CF662029F0B701862D90E05A
:10FCC0000E94BB8B03FD03C00BE010E102C007E004
:10FCD00010E1F72DF0717F2EF8018491882309F44B
:10FCE00076C271108052B70190E00E94BB8B0F5F0B
:10FCF0001F4FF2CF77FE0FC04C0C04FF04C08A8167
:10FD0000813309F44A94141474F5F8E0F41578F585
:10FD100088E0482E2CC076FC2AC0812F90E08C15FC
:10FD20009D059CF06CEFC6166FEFD60674F0772D2C
:10FD30007068772E0AC0E2E0F0E0EC0FFD1FE10FE3
:10FD4000F11D8081803319F411501111F4CF77FE29
:10FD50000EC044244394410E812F90E0C816D9066A
:10FD60002CF41C1904C04424439401C010E077FE15
:10FD700007C01C141D043CF496012F5F3F4F05C0C3
:10FD800025E030E002C021E030E0662011F02F5F76
:10FD90003F4F112331F0412F50E04F5F5F4F240F51
:10FDA000351F452D50E02417350714F4521A01C0B1
:10FDB000512C872D897049F4552039F0B70180E224
:10FDC00090E00E94BB8B5A94F7CF662029F0B701D0
:10FDD000862D90E00E94BB8B73FC09C0552039F042
:10FDE000B70180E390E00E94BB8B5A94F7CF77FE77
:10FDF0005FC09C2D8D2DD7FE02C090E080E0692E63
:10FE0000782E40E050E0C601841991099D878C87C7
:10FE1000960126193709280D391D812F90E0EE270C
:10FE2000FF27E81BF90BFF87EE87FFEF6F167F06B2
:10FE300069F4B7018EE290E02B8B3A8B488B598B9B
:10FE40000E94BB8B598948893A892B89C614D704EB
:10FE500054F06C857D85661577052CF4F901E40F67
:10FE6000F51F818101C080E371E0671A71084F5F5F
:10FE70005F4FEE85FF856E167F066CF0B70190E050
:10FE80002B8B3A8B488B598B0E94BB8B2B893A89E1
:10FE900048895989CACF6C147D0439F49A81963304
:10FEA00018F4953311F404FF81E3B70190E04BC0DF
:10FEB0008A81813309F00F7EB70190E00E94BB8BED
:10FEC000111105C074FE18C085E490E017C0B70199
:10FED0008EE290E00E94BB8B82E066246394680E01
:10FEE000F401E80FF11D8081B70190E00E94BB8B07
:10FEF000115041F3862DF1CF85E690E0B7010E94C5
:10FF0000BB8BD7FC05C0C114D10439F404FF05C074
:10FF1000D194C194D1088DE201C08BE2B70190E089
:10FF20000E94BB8B80E36AE0C616D1042CF08F5F81
:10FF3000FAE0CF1AD108F7CFB70190E00E94BB8B4F
:10FF4000B701C601C0960E94BB8B41C1833631F018
:10FF5000833779F0833509F058C021C0560172E02B
:10FF6000A70EB11CF6018081898301E010E06401D5
:10FF700014C05601F2E0AF0EB11CF601C080D18072
:10FF800026FF03C0612F70E002C06FEF7FEFC60154
:10FF90002B8B0E94818B8C012B892F7715C05601EA
:10FFA000F2E0AF0EB11CF601C080D18026FF03C085
:10FFB000612F70E002C06FEF7FEFC6012B8B0E94B4
:10FFC000438B8C012B892068722E23FD1AC0852D4E
:10FFD00090E008171907A8F4B70180E290E00E94AA
:10FFE000BB8B5A94F4CFF60177FC859177FE819113
:10FFF0006F01B70190E00E94BB8B51105A940150E1
:020000021000EC
:1000000011090115110579F7E2C0843611F089361E
:1000100051F5560127FF09C0F4E0AF0EB11CF601FF
:1000200060817181828193810AC0F2E0AF0EB11CC0
:10003000F60160817181882777FD8095982F022FC6
:100040000F7697FF08C090958095709561957F4FCA
:100050008F4F9F4F00682AE030E0A4010E94C68CB9
:10006000C82EC8183EC0022F853721F40F7E2AE023
:1000700030E01DC0097F8F3691F018F4883559F0B3
:10008000B0C0803719F0883711F0ABC0006104FFB1
:1000900009C0046007C024FF08C0066006C028E04D
:1000A00030E005C020E130E002C020E132E056013E
:1000B00007FF09C0F4E0AF0EB11CF6016081718149
:1000C0008281938108C0F2E0AF0EB11CF60160811D
:1000D000718180E090E0A4010E94C68CC82EC818EF
:1000E0000F7706FF0BC0202F2E7FC11650F404FFA0
:1000F0000AC002FD08C0202F2E7E05C0DC2C202F58
:1001000003C0DC2C01C0D12E24FF0DC0FE01EC0D7C
:10011000F11D8081803311F4297E09C022FF06C0C1
:10012000D394D39404C0822F867809F0D39423FD0E
:1001300013C020FF06C01C2DD51418F4150D1D1971
:10014000D52CD51468F4B70180E290E02B8B0E9487
:10015000BB8BD3942B89F5CFD51410F45D1801C057
:10016000512C24FF12C0B70180E390E02B8B0E943A
:10017000BB8B2B8922FF17C021FF03C088E590E0CD
:1001800002C088E790E0B7010CC0822F867859F052
:1001900021FD02C080E201C08BE227FD8DE2B701A4
:1001A00090E00E94BB8BC11638F4B70180E390E069
:1001B0000E94BB8B1150F7CFCA94F401EC0DF11DD6
:1001C0008081B70190E00E94BB8BC110F5CF552014
:1001D00009F4C2CCB70180E290E00E94BB8B5A9434
:1001E000F6CFF7018681978102C08FEF9FEF63966C
:1001F0000FB6F894DEBF0FBECDBFDF91CF911F9138
:100200000F91FF90EF90DF90CF90BF90AF909F90B5
:100210008F907F906F905F904F903F902F900895B8
:100220005058BB27AA270ED04EC23FD230F044D23E
:1002300020F031F49F3F11F41EF4FFC10EF4E0955D
:10024000E7FBF5C1E92F50D280F3BA1762077307B5
:100250008407950718F071F49EF568C20EF4E095D6
:100260000B2EBA2FA02D0B01B90190010C01CA0170
:10027000A0011124FF27591B99F0593F50F4503E1B
:1002800068F11A16F040A22F232F342F4427585F0D
:10029000F3CF469537952795A795F0405395C9F725
:1002A0007EF41F16BA0B620B730B840BBAF09150DD
:1002B000A1F0FF0FBB1F661F771F881FC2F70EC07C
:1002C000BA0F621F731F841F48F48795779567954F
:1002D000B795F7959E3F08F0B3CF9395880F08F038
:1002E0009927EE0F979587950895DFD158F080E80C
:1002F00091E009F49EEFE0D128F040E851E059F494
:100300005EEF09C09AC112C2E92FE078EDD168F31F
:10031000092E052AC1F3261737074807590738F071
:100320000E2E07F8E02569F0E025E0640AC0EF63CF
:1003300007F8009407FADB01B9019D01DC01CA014D
:10034000AD01EF9347D0BFD10AD05F91552331F073
:100350002BED3FE049E450FD49EC63CF0895DF9376
:10036000DD27B92FBF7740E85FE316161706480769
:100370005B0710F4D92FE1D19F938F937F936F93F5
:1003800046D3E0E3F1E06CD19ED12F913F914F91A4
:100390005F919AD2DD2349F09058A2EA2AED3FE01E
:1003A00049EC5FE3D0785D274DDFDF918CC11BD135
:1003B00008F481E008950CD086C17ED140F075D15B
:1003C00030F021F45F3F19F032C15111B0C135C195
:1003D0008BD198F39923C9F35523B1F3951B550B92
:1003E000BB27AA2762177307840738F09F5F5F4F08
:1003F000220F331F441FAA1FA9F333D00E2E3AF049
:10040000E0E830D091505040E695001CCAF729D062
:10041000FE2F27D0660F771F881FBB1F26173707B1
:100420004807AB07B0E809F0BB0B802DBF01FF27E1
:1004300093585F4F2AF09E3F510568F0F8C077C18E
:100440005F3FECF3983EDCF3869577956795B7951B
:10045000F7959F5FC9F7880F911D9695879597F936
:100460000895E1E0660F771F881FBB1F62177307AF
:100470008407BA0720F0621B730B840BBA0BEE1FC4
:1004800088F7E095089519F40EF0D1C04FC1D5C09A
:1004900033D1C8F39638C0F707F80F92E8942BE3EE
:1004A0003AEA48EB5FE712D20F920F920F924DB7E4
:1004B0005EB70F92CAD1EDE5F1E0D2D04F915F91D6
:1004C000EF91FF91E595EE1FFF1F49F0FE57E068A1
:1004D0004427EE0F441FFA95E1F74195550B36D1AD
:1004E0000F9007FE2AC1089597FB0EF4A9D03EC0D5
:1004F000E89409C097FB3EF49095809570956195BE
:100500007F4F8F4F9F4F9923A9F0F92F96E9BB2773
:100510009395F695879577956795B795F111F8CFEF
:10052000FAF4BB0F11F460FF1BC06F5F7F4F8F4F5A
:100530009F4F16C0882311F096E911C0772321F050
:100540009EE8872F762F05C0662371F096E8862FE8
:1005500070E060E02AF09A95660F771F881FDAF73F
:10056000880F9695879597F90895E894F92F96EB5B
:10057000FF2381F0121613061406440B9395F6958B
:1005800087957795679557954040FF23B9F71BC02E
:1005900099270895882351F49850D2F7872B762F06
:1005A000652F542F432F322F20E0B1F3121613067C
:1005B0001406440B88233AF09A95440F551F661F82
:1005C000771F881FCAF755234AF4440F551F11F4AB
:1005D00060FF04C06F5F7F4F8F4F9F4F880F9695CE
:1005E000879597F90895990F0008550FAA0BE0E831
:1005F000FEEF16161706E807F907C0F012161306E5
:10060000E407F50798F0621B730B840B950B39F424
:100610000A2661F0232B242B252B21F408950A268A
:1006200009F4A140A6958FEF811D811D089597F9CA
:100630009F6780E870E060E008959FEF80EC089588
:100640009095809570956095509540953095219541
:100650003F4F4F4F5F4F6F4F7F4F8F4F9F4F0895CB
:10066000DF93CF931F930F93FF92EF92DF927B0163
:100670008C01689405C0DA2EEF0126D1FE01E894C2
:10068000A5912591359145915591AEF3EF01DADDB4
:10069000FE019701A801DA9479F7DF90EF90FF90BF
:1006A0000F911F91CF91DF91089500240A9416169F
:1006B000170618060906089500240A941216130650
:1006C000140605060895092E0394000C11F48823DE
:1006D00052F0BB0F40F4BF2B11F460FF04C06F5FFA
:1006E0007F4F8F4F9F4F089557FD9058440F551FD0
:1006F00059F05F3F71F04795880F97FB991F61F0A4
:100700009F3F79F087950895121613061406551F1A
:10071000F2CF4695F1DF08C0161617061806991F86
:10072000F1CF86957105610508940895E894BB277B
:1007300066277727CB0197F908959B01AC0160E00C
:1007400070E080E89FE337CE72CF64C1D5DFE8F375
:100750009923D9F3940F511DBBF39150504094F05D
:1007600059F0882332F0660F771F881F9150504050
:10077000C1F79E3F510544F7880F911D96958795C7
:1007800097F908955F3FACF0983E9CF0BB278695A3
:1007900077956795B79508F4B1609395C1F7BB0F4E
:1007A00058F711F460FFE8CF6F5F7F4F8F4F9F4F77
:1007B000E3CFBDCF0AD029ED3BE54EED5EE378C037
:1007C0000EF028C13ACF689432CF96DFC8F3992350
:1007D000D1F3C6F3DF93CF931F930F93FF92C92FEB
:1007E000DD2788232AF02197660F771F881FDAF705
:1007F00020E030E040E85FEB9FE3883920F0803E66
:1008000030F021968F770DDDE5E8F1E003C009DDDA
:10081000E2EBF1E025DF8B01BE01EC01FB2E6F570F
:1008200071097595771F880B990B64DE28E132E713
:1008300041E35FE349D0AF2D9801AE01FF900F91E6
:100840001F91CF91DF91FEDC3ECFFA01DC01AA0FB0
:10085000BB1F9B01AC01BF5728F422273327442735
:1008600050781FC0B75188F4AB2F002446953795B8
:100870002795011CA395D2F3002069F0220F331FA6
:10088000441FB395DAF30DD0CBCC61307105A0E8ED
:100890008A07B94630F49B01AC0166277727882781
:1008A0009078309621F020833183428353830895DA
:1008B0000BD009CFFADE28F0FFDE18F0952309F0FF
:1008C000B6CEBBCE112433CF0FDFA0F3959FD1F36B
:1008D000950F50E0551F629FF001729FBB27F00DEE
:1008E000B11D639FAA27F00DB11DAA1F649F662743
:1008F000B00DA11D661F829F2227B00DA11D621F92
:10090000739FB00DA11D621F839FA00D611D221F4B
:10091000749F3327A00D611D231F849F600D211D2F
:10092000822F762F6A2F11249F5750408AF0E1F0D2
:1009300088234AF0EE0FFF1FBB1F661F771F881F1B
:1009400091505040A9F79E3F510570F070CEEFCE08
:100950005F3FECF3983EDCF3869577956795B79506
:10096000F795E7959F5FC1F7FE2B880F911D969530
:10097000879597F90895FA01EE0FFF1F309621052C
:10098000310599F16115710561F48038BFE39B076A
:1009900049F168949038810561F08038BFEF9B077A
:1009A00041F0992342F5FF3FE1053105210511F1A1
:1009B000E8940894E795D901AA2329F4AB2FBE2F18
:1009C000F85FD0F310C0FF5F70F4A695E0F7F73939
:1009D00050F019F0FF3A38F49F779F930CD00F90A6
:1009E00007FC905808953EF028CE60E070E080E863
:1009F0009FE308954FE79F775F934F933F932F9324
:100A0000E4DE2F913F914F915F9152DF41CD9B01E9
:100A1000AC014ECF9F3F31F0915020F487957795F0
:100A20006795B795880F911D9695879597F90895C5
:100A30000E942085332312F48A1B9B0B0C94318572
:100A4000A29FB001B39FC001A39F700D811D11240F
:100A5000911DB29F700D811D1124911D08950E945A
:100A60002085B7FF0895821B930B08950E9420856F
:100A7000A59F900DB49F900DA49F800D911D1124F2
:100A80000895B7FF0C9436850E943685821B930B20
:100A90000895DB018F939F930E943685BF91AF919C
:100AA000A29F800D911DA39F900DB29F900D1124C8
:100AB0000895AA1BBB1B51E107C0AA1FBB1FA617A5
:100AC000B70710F0A61BB70B881F991F5A95A9F7F7
:100AD00080959095BC01CD01089597FB072E16F4E3
:100AE000009407D077FD09D00E94598507FC05D0F6
:100AF0003EF4909581959F4F0895709561957F4F35
:100B00000895A1E21A2EAA1BBB1BFD010DC0AA1F4E
:100B1000BB1FEE1FFF1FA217B307E407F50720F066
:100B2000A21BB30BE40BF50B661F771F881F991FE1
:100B30001A9469F760957095809590959B01AC012A
:100B4000BD01CF010895052E97FB1EF400940E946D
:100B5000CE8657FD07D00E94818507FC03D04EF456
:100B60000C94CE8650954095309521953F4F4F4F30
:100B70005F4F0895689401C0E894F92FF12B12F0AB
:100B80000C94EE85A0E0B0E0E8ECF5E80C94EC867F
:100B9000092E059422F40E94D686112392F4F0E8DF
:100BA0000F26FFEFE094F09400951095B094C09458
:100BB000D094A194BF0ACF0ADF0AEF0AFF0A0F0BF5
:100BC0001F0B0E947D8607FC0E94D686CDB7DEB73C
:100BD000ECE00C940887689401C0E8948F929F928F
:100BE000CF93DF930E947D86DF91CF919F908F906E
:100BF0000895DF93CF931F930F939A9DF02D219F1C
:100C0000F00D8B9DF00D8A9DE02DF10D039FF00DF1
:100C1000029FE00DF11D4E9DE00DF11D5E9DF00D5A
:100C20004F9DF00D7F936F93BF92AF925F934F9361
:100C3000D5010E9420858B01AC01D7010E9420853F
:100C4000EB01E80FF91FD6010E9449862F913F91D1
:100C5000D6010E942085C60FD71FE81FF91FAF914C
:100C6000BF910E9449862F913F910E942085C60F17
:100C7000D71FE81FF91FD6010E942085E60FF71F36
:100C80009801BE01CF0111240F911F91CF91DF91E7
:100C900008950E942085460F571FC81FD91F08F4CA
:100CA00031960895E894DF93CF93FC01DB010E9415
:100CB00020857F936F93E9019A01AC01BF93AF93B5
:100CC0003F932F93DF010E94208526F46C1B7D0B40
:100CD000820B930B9E01EB01FC010E944986AF91B0
:100CE000BF912F913F910E944986BE01CF01F9012A
:100CF0002F913F91CF91DF91089588249924F40199
:100D0000E401B0E49F93AA279A158B049C04ED0597
:100D1000FE05CF05D007A10798F4AD2FDC2FCF2F0C
:100D2000FE2FE92D982C892E982F872F762F652F4F
:100D3000542F432F322F2227B85031F7BF9127C0AD
:100D40001B2EBF91BB27220F331F441F551F661F49
:100D5000771F881F991F881C991CEE1FFF1FCC1F2F
:100D6000DD1FAA1FBB1F8A149B04EC05FD05CE05E1
:100D7000DF05A007B10748F08A189B08EC09FD09B8
:100D8000CE09DF09A00BB10B21601A94E1F62EF415
:100D90009401AF01BE01CD01000C0895909580959E
:100DA000709561957F4F8F4F9F4F08956095709517
:100DB0008095909530954095509521953F4F4F4F98
:100DC0005F4F6F4F7F4F8F4F9F4F08952F923F92EE
:100DD0004F925F926F927F928F929F92AF92BF924B
:100DE000CF92DF92EF92FF920F931F93CF93DF93F7
:100DF000CDB7DEB7CA1BDB0B0FB6F894DEBF0FBE54
:100E0000CDBF09942A88398848885F846E847D84A0
:100E10008C849B84AA84B984C884DF80EE80FD80A2
:100E20000C811B81AA81B981CE0FD11D0FB6F89418
:100E3000DEBF0FBECDBFED010895EE0FFF1F059081
:100E4000F491E02D09946927962769277827872749
:100E5000782708950F93083090F0982F872F762FDA
:100E6000652F542F432F322F22270850F4CF220F03
:100E7000331F441F551F661F771F881F991F0A9530
:100E8000B2F70F91089597FB10F8169400080F938E
:100E9000083098F00850232F342F452F562F672FF6
:100EA000782F892F902DF4CF059497958795779576
:100EB000679557954795379527950A95AAF70F9106
:100EC00008952A0D3B1D4C1D5D1D6E1D7F1D801F4D
:100ED000911F08950024A7FD00942A0F301D401D86
:100EE000501D601D701D801D901D08952A193B091D
:100EF0004C095D096E097F09800B910B08952A1535
:100F00003B054C055D056E057F058007910708953B
:100F10000024A7FD00942A17300540055005600500
:100F200070058005900508958F929F92AF92BF92B1
:100F3000CF92DF92EF92FF92CF93DF93EC01688123
:100F400079818A819B81611571058105910521F463
:100F500064E279ED8BE597E02DE133EF41E050E07D
:100F60000E94A38549015A019B01AC01A7EAB1E4A3
:100F70000E9436856B017C01ACEEB4EFA5019401B3
:100F80000E944485C60ED71EE81EF91EF7FE06C055
:100F900081E0C81AD108E10880E8F80AC882D9823D
:100FA000EA82FB82C6019F77DF91CF91FF90EF909D
:100FB000DF90CF90BF90AF909F908F9008950C944A
:100FC000948782ED92E00C949487A0E0B0E0809347
:100FD000D2029093D302A093D402B093D502089585
:100FE0002F923F925F926F927F928F929F92AF92D9
:100FF000BF92CF92DF92EF92FF920F931F93CF9306
:10100000DF938B01EA016115710521F0DB018C93FF
:1010100011969C93209739F09E012250310923327A
:10102000310508F0FBC07C016701BFEFCB1ADB0A7A
:101030005601F7016080862D90E00E94328B892B4B
:1010400011F07601F1CFFDE26F120AC0570182E084
:10105000A80EB11CD70111966C90772473940BC025
:10106000BBE26B1207C05701E2E0AE0EB11CD70124
:1010700011966C90712CCE018F7E892B89F4B0E390
:101080006B1222C0F50180818F7D883541F561802A
:10109000F2E0AF0EB11C872D8260782EC0E1D0E067
:1010A000C830D105F1F04CF4C230D10511F5C12C96
:1010B000D12CE12CB0E4FB2E2FC0CA30D10531F089
:1010C000C031D10521F115C0209751F7CAE0D0E019
:1010D000ACECCA2EDC2CEC2CACE0FA2E1DC0209718
:1010E000F9F6C8E0D0E0C12CD12CE12CF0E1FF2EC4
:1010F00013C060E070E080E090E89E01442737FD77
:101100004095542F0E94818569017A0105C0C12C48
:10111000D12CE12CE8E0FE2EF50160E020E030E08B
:10112000A9014E01AA2497FCA094BA2C1F0170EDCE
:10113000572E560CA9E0A51570F48FEB860D8A3159
:1011400018F499EC592E06C08FE9860D8A3130F5D6
:1011500089EA582E560C852D90E08C179D07F4F4E3
:1011600067FD18C0C216D306E406F50680F0C50177
:10117000B4010E9449859B01AC01250D311D411D23
:10118000511D213031054105B0E85B0710F06FEFCC
:1011900001C061E03196D1016C90C8CF872D81707C
:1011A0000115110571F0662329F03197D801ED93EF
:1011B000FC9307C071FE19C03297D801ED93FC93E0
:1011C00014C067FF12C0882329F020E030E040E01F
:1011D00050E804C02FEF3FEF4FEF5FE782E290E06F
:1011E0009093F5308093F43016C0882341F05095E9
:1011F0004095309521953F4F4F4F5F4F0CC057FFA3
:101200000AC082E290E09093F5308093F4302FEFA3
:101210003FEF4FEF5FE7B901CA0104C060E070E043
:1012200080E090E0DF91CF911F910F91FF90EF90C0
:10123000DF90CF90BF90AF909F908F907F906F90F6
:101240005F903F902F9008952F923F925F926F9200
:101250007F928F929F92AF92BF92CF92DF92EF9246
:10126000FF920F931F93CF93DF938B01EA016115D8
:10127000710521F0DB018C9311969C93209739F036
:101280009E01225031092332310508F0D8C07C017B
:101290006701BFEFCB1ADB0A5601F7016080862D8C
:1012A00090E00E94328B892B11F07601F1CFFDE2A4
:1012B0006F120AC0570182E0A80EB11CD701119627
:1012C0006C90772473940BC0BBE26B1207C057017C
:1012D000E2E0AE0EB11CD70111966C90712CCE01DC
:1012E0008F7E892B89F4B0E36B1237C0F5018081C2
:1012F0008F7D8835D1F46180F2E0AF0EB11C872D6F
:101300008260782EC0E1D0E0CA30D10551F1C03101
:10131000D10521F0C830D10599F409C0CC24CA9474
:10132000DC2CEC2CAFE0FA2E22C0209769F7C8E045
:10133000D0E0CC24CA94DC2CEC2CFFE1FF2E17C0AB
:101340006FEF7FEFCB019E01442737FD4095542F6F
:101350000E94818569017A010AC02097A9F6CAE036
:10136000D0E0E9E9CE2EDC2CEC2CE9E1FE2EF501F3
:1013700060E020E030E0A9014E01AA2497FCA0948F
:10138000BA2C1F0170ED572E560CA9E0A51570F46C
:101390008FEB860D8A3118F499EC592E06C08FE92F
:1013A000860D8A3148F589EA582E560C852D90E035
:1013B0008C179D070CF56F3FD9F0C216D306E406D3
:1013C000F50698F0C501B4010E9449859B01AC0166
:1013D000852D90E0A0E0B0E0280F391F4A1F5B1F69
:1013E000281739074A075B0710F46FEF01C061E067
:1013F0003196D1016C90C5CF0115110551F06623CE
:1014000011F0319703C071FE04C03297D801ED93FB
:10141000FC9370FE07C050954095309521953F4F45
:101420004F4F5F4F67FF10C082E290E09093F5301E
:101430008093F4306FEF7FEF8FEF9FEF07C060E096
:1014400070E080E090E002C0B901CA01DF91CF9165
:101450001F910F91FF90EF90DF90CF90BF90AF90D2
:101460009F908F907F906F905F903F902F90089506
:10147000662777270C945F8DFC0188279927E894CD
:1014800021912032E9F3293010F02E30C8F32B32AD
:1014900041F02D3239F4689404C00E94B38B820F5E
:1014A000911D219120532A30C0F31EF4909581950F
:1014B0009F4F0895283008F027E03327DA01990F6D
:1014C000311D87FD916000966105710539F4326028
:1014D0002E5F3D9330E32A95E1F708959F3F30F06A
:1014E00080387105610509F03C5F3C5F3D939130A8
:1014F00008F08068911DDF93CF931F930F93FF92A5
:10150000EF92192F987F9695E92F96959695E90F6A
:10151000FF27E759FF4E99273327EE24FF24A70121
:10152000E70105900894079428F4360FE71EF81E8B
:10153000491F511D660F771F881F991F0694A1F739
:101540000590079428F4E70EF81E491F561FC11D89
:10155000770F881F991F661F0694A1F705900794BF
:1015600028F4F80E491F561FC71FD11D880F991F59
:10157000661F771F0694A1F70590079420F4490F82
:10158000561FC71FD81F990F661F771F881F069405
:10159000A9F784911095177041F0D695C795579586
:1015A0004795F794E7941A95C1F7EFE0F0E1689456
:1015B0001590159135916591959105907FE2739500
:1015C000E118F10A430B560BC90BD009C0F7E10C27
:1015D000F11E431F561FC91FD01D7EF4703311F436
:1015E0008A95E6CFE894015030F0080F0AF40027FE
:1015F000021708F4202F2395022F7A3328F079E37D
:101600007D932A95E9F710C07D932A9589F6069473
:1016100097956795379517951794E118F10A430B3D
:10162000560BC90BD00998F023957E9173957A33A8
:1016300008F070E37C932013B8F77E9170617D937E
:1016400030F0839571E37D9370E32A95E1F71124DF
:10165000EF90FF900F911F91CF91DF91992787FD18
:10166000909508959111A8C3803219F08950855042
:10167000D0F70895FB01DC018D91059080190110D0
:10168000D9F3990B0895FC01059061507040011049
:10169000D8F7809590958E0F9F1F089542E85AE1E4
:1016A0000C948C8BFB01DC0102C001900D92415027
:1016B0005040D8F70895DC0101C06D93415050406F
:1016C000E0F70895FB01DC018D9101908019011074
:1016D000D9F3990B0895FB01DC0101900D920020D4
:1016E000E1F70895FB01DC014150504048F00190C2
:1016F0000D920020C9F701C01D9241505040E0F703
:101700000895FC016150704001900110D8F7809558
:1017100090958E0F9F1F0895FA01A191B0810097B7
:1017200019F41097E1F0CD01DC01CD010D900020FE
:1017300011F4C00113C0FB012191222319F02015DF
:10174000D9F7F3CFFB012191201519F41E921196C0
:1017500006C02223C1F70D900020A1F7D001FA01A5
:10176000A193B08308957AE0979F902D879F802D55
:10177000910D112408950F931F93CF93DF93182F8A
:10178000092FEB018B8181FD03C08FEF9FEF20C0FC
:1017900082FF10C04E815F812C813D81421753072B
:1017A0007CF4E881F9819F012F5F3F4F39832883C3
:1017B000108306C0E885F985812F0995892B29F7C3
:1017C0002E813F812F5F3F4F3F832E83812F902FAC
:1017D000DF91CF911F910F910895CF93DF93CDB7F4
:1017E000DEB7FE01359661917191AF018091F030C5
:1017F0009091F1300E946C7DDF91CF9108950F930D
:101800001F93CF93DF93CDB7DEB7FE01379661917B
:10181000719100EF10E3D8018D919C91DC0113963A
:101820002C911397286013962C93AF010E946C7D26
:10183000D801ED91FC912381277F2383DF91CF9104
:101840001F910F9108950F931F93CF93DF93E09112
:10185000F030F091F130238121FF1BC0EC0100E05A
:1018600010E089916091F0307091F130DB011896B1
:10187000ED91FC911997882331F00995892B89F313
:101880000FEF1FEFEECF8AE00995892B11F4C80105
:1018900002C08FEF9FEFDF91CF911F910F910895BD
:1018A0000F931F93CF93DF93CDB7DEB72E970FB66D
:1018B000F894DEBF0FBECDBF0D891E898F89988D2C
:1018C00026E02C831A83098397FF02C080E090E80A
:1018D00001979E838D83AE01455E5F4F698D7A8D42
:1018E000CE0101960E946C7D4D815E8157FD0AC03C
:1018F0002F813885421753070CF49A01F801E20F43
:10190000F31F10822E960FB6F894DEBF0FBECDBF28
:10191000DF91CF911F910F9108950F931F93CF9354
:10192000DF93CDB7DEB72E970FB6F894DEBF0FBEAC
:10193000CDBF8C01CA0146E04C831A83098377FF2F
:1019400002C060E070E8615071097E836D83A90177
:10195000BC01CE0101960E946C7D4D815E8157FDD8
:101960000AC02F813885421753070CF49A01F801F9
:10197000E20FF31F10822E960FB6F894DEBF0FBE53
:10198000CDBFDF91CF911F910F910895FA01AA2742
:10199000283051F1203181F1E8946F936E7F6E5FB2
:1019A0007F4F8F4F9F4FAF4FB1E03ED0B4E03CD060
:1019B000670F781F891F9A1FA11D680F791F8A1F43
:1019C000911DA11D6A0F711D811D911DA11D20D0AA
:1019D00009F468943F912AE0269F11243019305D64
:1019E0003193DEF6CF010895462F4770405D419355
:1019F000B3E00FD0C9F7F6CF462F4F70405D4A33A2
:101A000018F0495D31FD4052419302D0A9F7EACF69
:101A1000B4E0A6959795879577956795BA95C9F798
:101A200000976105710508959B01AC010A2E06948B
:101A30005795479537952795BA95C9F7620F731F44
:101A4000841F951FA01D0895DC01CB01FC01F999AD
:101A5000FECF06C0F2BDE1BDF89A319600B40D92FA
:101A600041505040B8F70895F999FECF92BD81BD1D
:101A7000F89A992780B50895A8E1B0E042E050E0D7
:101A80000C94268DDC01CB0103C02D910E944D8D5D
:101A900041505040D0F70895262FF999FECF1FBA34
:101AA00092BD81BD20BD0FB6F894FA9AF99A0FBE87
:101AB000019608950E944C8D272F0C944D8D4F92C6
:101AC0005F926F927F928F929F92AF92BF92CF92CE
:101AD000DF92EF92FF920F931F93CF93DF938B01CF
:101AE0006115710521F0DB018C9311969C93EC013B
:101AF0005E01BFEFAB1ABB0A7501C8808C2D90E068
:101B00000E94328B892B11F0E501F2CFEDE2CE126B
:101B100008C07E01F2E0EF0EF11CC980DD24D394F1
:101B200009C02BE2C21205C07E0142E0E40EF11CA6
:101B3000C980D12CE701219743E050E061E171E1D8
:101B4000CE010E94DF8E892BD1F4E701229645E079
:101B500050E06CE071E1CE010E94DF8E892B11F420
:101B6000E70127960115110519F0D801CD93DC93F3
:101B7000D11008C160E070E080E89FE70CC143E04D
:101B800050E069E071E1CE010E94DF8E892B59F4AB
:101B90000115110509F4FBC0B2E0EB0EF11CF801D0
:101BA000F182E082F4C0F70160E070E0CB01C0E0B8
:101BB000D0E07F01A0EDAA2EAC0C29E02A1530F16F
:101BC0004D2D4260B42E2D2D2870D2FE04C021115F
:101BD00025C0219623C021112197A5E0B0E09B01EB
:101BE000AC010E943685660F771F881F991F6A0D0A
:101BF000711D811D911D6839A9E97A078A07A9E13C
:101C00009A0760F0BD2DB660BB2E08C02EEFA21261
